:020000040800F2
:10000000F0FF022065DA0508ADDA0508ADE6010863
:10001000ADDA0508ADDA0508ADDA05080000000024
:10002000000000000000000000000000ADDA05083C
:10003000ADDA050800000000ADDA0508A19500085A
:10004000ADDA0508ADDA0508ADDA0508ADDA050860
:10005000ADDA0508ADDA050841B1000849B100087C
:1000600051B1000859B1000861B10008ADDA0508C6
:10007000ADDA0508ADDA0508ADDA0508ADDA050830
:10008000ADDA0508ADDA0508ADDA0508ADDA050820
:10009000ADDA0508ADDA0508ADDA050869B1000882
:1000A0001DDF00082DDF000855DF00089DDE000879
:1000B000ADDE0008BDDE0008CDDE000865EA000800
:1000C0004DA500086DEA000859A50008ADDA05083D
:1000D000ADDA05089D420508694305085544050841
:1000E00071B10008ADDA0508ADDA050865DF000872
:1000F00075DF000885DF00080DDF0008ADDA0508B0
:10010000ADDA0508ADDA0508DDDE0008ADDA050870
:10011000414505082D460508EDDE0008FDDE000816
:10012000CDAD0008E1AD0008F5AD000809AE00084E
:100130001DAE0008ADDA0508ADDA0508ADDA050830
:10014000ADDA0508ADDA0508ADDA050809CE000814
:1001500031AE000845AE0008000000001947050850
:1001600075EA000865A50008000000000000000016
:10017000ADDA0508ADDA0508ADDA050800000000C3
:1001800000000000ADDA050805480508F14805083B
:10019000ADDA0508000000000000000000000000CB
:1001A000000000000000000000000000ADDA0508BB
:1001B000ADDA050800000000ADDA05080000000017
:1001C000000000000000000000000000000000002F
:1001D0000000000000000000ADDA0508ADDA0508F7
:1001E000ADDA05081DCD0008ADDA050895DF000879
:1001F00059AE00086DAE000881AE000895AE00084B
:0C020000A9AE0008BDAE0008D1AE000899
:1080000010B40C4B4FF0E02C1A68DCF8180019681B
:108010008A42F9D159688842F6D89C684FF47A713F
:1080200001FB04F31B1AB3FBF4F35DF8044B01FBF3
:1080300002307047A0180020002A4FEA014C30B5EA
:1080400003460ABFE6468E468C4600F1C005002472
:1080500019689A6841EA0C0142EA0E029A60C3E983
:1080600000140C33AB42F3D1D0F8C030C0F8C44098
:1080700043EA0E03C0F8C030C0F8C84030BD00BFAE
:1080800030B4436919690A6822F001020A609A68EB
:10809000B3F80CC01468E26822EA0C02E2600468DB
:1080A00090F810C02068082202FA0CF2024039D180
:1080B0002248057B022000FA0CF06060002D2FD0D2
:1080C000187E01282FD0D3F8A0100131C3F8A010DA
:1080D000EFF31180502181F312885C68DD6B216819
:1080E00021EA05011D6C2943C0B2216080F311888B
:1080F00098681969DC6A00680C601C6B4C605C6BEA
:108100008C609C6BCC604262B3F87C20C2620A68CF
:10811000012422430A601C76C2689B891343C36012
:1081200030BC7047FEE7D3F8A4000130C3F8A400C8
:108130000B6862F300030B60F2E700BFA018002099
:1081400010B40C4C2369002B11DD002004F1140C39
:108150000146DCF8743003F1C00259600C339342DD
:10816000FBD12369013083420CF1AC0CF1DC5DF8EA
:10817000044B7047A018002070B5474C04EB401327
:1081800093F8E02202B970BD072800F282804C22E9
:1081900002FB004294F8245694F825E692F8C66350
:1081A00083F8C66275454FF000034FEA401C82F821
:1081B000C6330CD00EEB4E0304EBC30393F8282612
:1081C000561E012E4FEA4E0355D9032A4DD004EB1B
:1081D0000C00A0F8C412EFF31182902383F31288ED
:1081E00090F8C632B0F8C41243EA41030021D2B27B
:1081F0009BB280F8C61282F31188217BD0F8DC4252
:108200001A0982EA13225A40B9B1D0F8C812646F31
:10821000D2431B019BB202F00F020120884013439E
:1082200004F1C0011D0402D46268024362600C3490
:108230005B00A1429BB2F5D170BDD0F8C812646F4B
:108240001B0110319BB202F00F0201208840134342
:1082500004F1C0011A0402D46268024362600C3463
:108260005B00A1429BB2F5D170BD0EF1010202F09C
:108270000302AA42ABD0734404EBC303034493F854
:1082800035160029A3D004EB0C03012283F8C62283
:108290009DE700239B78FFDEA0180020704700BFF9
:1082A000704700BF024B03EB401393F8E1027047A5
:1082B000A01800204368826C10B49A61EFF3118219
:1082C000502383F312884168C46B0B6823EA0403CC
:1082D000446C2343D2B20B6082F31188D0E907418A
:1082E0008268036912681C605960D0E909419C608A
:1082F000D960B0F85C10D16200235DF8044B0376BE
:10830000704700BF026890F810C01168022303FA9A
:108310000CF3194200D1704710B4074C41684FF07C
:10832000000C84F888C608686CF3000008605DF8EB
:10833000044B5360704700BFA01800200B4890F812
:10834000891689B101EB4101002310B4490000F204
:108350008C601C4650F82320063302B114608B4217
:10836000F8D15DF8044B7047704700BFA01800209B
:108370000B4890F8891689B101EB4101002310B434
:10838000490000F28C601C4650F82320063302B1ED
:1083900014608B42F8D15DF8044B7047704700BF02
:1083A000A0180020204B1B78002B3BD12DE9F04179
:1083B0001E4C94F889269AB31D4F04F28C62502605
:1083C0004FF02C0E1D4607E094F8891652F8180B52
:1083D00001338B42056023DA117C0029F4D0516807
:1083E0004FEA912CACF5801CBCF1530F4FF0FE000E
:1083F00098BF17F80C00EFF3118C86F31288D1F8B0
:1084000024800EFB004008F10108C0F87487486919
:1084100040F001005FFA8CFC48618CF31188D3E7CF
:10842000BDE8F081704700BF00000020A0180020C8
:10843000D8F5050800EE100AB8EE400A704700BFF4
:10844000BCEEC00A10EE103A98B27047704700BFF9
:10845000704700BF704700BF704700BF01207047E2
:10846000094A0A4BD2F8E829D3F8BC02526AD3F879
:10847000C01292F85330012B08BFB2F85030A0EB75
:10848000010008BFC0187047A018002098290020DC
:10849000012380F85130704710B4EFF3118180232D
:1084A00083F312880C4AC9B2D2F8C432D2F8C84257
:1084B000D2F8C402D2F8C82281F31188904203F1A5
:1084C000FF33A3EB04038CBF0020012003EBC0208B
:1084D0005DF8044B704700BF98290020074BD0F887
:1084E00094105B68D0F8A0205B1A9A42B8BFC0F81D
:1084F000A030012380F8CC3000207047001000E04D
:10850000072809D8054B4C2202FB0033B3F8C403FB
:10851000B0FA80F04009704700207047A018002092
:10852000072806D8034B4C2202FB0033012283F8B4
:10853000C6237047A0180020374A38B54C2303FBE8
:10854000002393F8D33303B938BD92F824C692F8C8
:1085500025369C450ED003EB430402EBC40494F88B
:1085600028E60EF1FF35012D4FEA430445D9BEF14F
:10857000030F3DD04FF04C0C0CFB002CACF8C41397
:10858000EFF31181902383F31288BCF8C4439CF865
:10859000C63343EA44030024C9B29BB28CF8C643F5
:1085A00081F31188190A147B81EA1311594004B12F
:1085B000C9434C2404FB00241B0118489BB201F062
:1085C0000F021A43D0F8CC52D4F80C040121A8476A
:1085D000D4F80814B4F8D0C3CA88D4F8043442EAF2
:1085E0000C02CA8058601A6842F001021A6038BD55
:1085F0005D1C05F003056545BCD01C4402EBC404BA
:10860000044494F835160029B4D04C2303FB00230E
:10861000012483F8C643ADE7A01800209829002064
:1086200010B584464FEA810E102312F4004F14BF98
:108630000E2407245200013BCCF8004092B2F444CF
:10864000F3D100EB81128C01035142F8213012204A
:1086500010BD00BF10B584464FEA810E0424130BF1
:1086600003EB430318331201013CCCF8003092B203
:10867000F444F4D100EB01130A01845043F8214083
:10868000062010BD704700BF704700BF034B00EBD2
:10869000400003EBC00393F89D067047A01800202C
:1086A000074B93F8D032834207D9064B00EB4000CA
:1086B00003EBC003D3F8A00670470020704700BF4B
:1086C00098290020A018002036E700BF072808D806
:1086D000044B03EB401393F8E02212B1012283F81C
:1086E000C6227047A0180020072808D8054B03EBC6
:1086F0004013B3F8C402B0FA80F04009704700207C
:10870000704700BFA0180020054B93F8D032834279
:1087100083BF044B03EB4013D3F8D0020020704713
:1087200098290020A018002003689A69D10508D56F
:108730004FF4807213218177DA611A6822F0800287
:108740001A609A69920508D54FF400721321817757
:10875000DA611A6822F080021A609A69510508D518
:108760004FF4806213218177DA611A6822F0800267
:108770001A609A69120508D54FF4006213218177B7
:10878000DA611A6822F080021A609A69D10408D569
:108790004FF4805213218177DA611A6822F0800247
:1087A0001A609A69920408D54FF400521321817718
:1087B000DA611A6822F080021A607047194B1A4A6F
:1087C0001968D2F8D432CB1A322B05DCD2F8E83251
:1087D000CB1A002B11DC7047D2F8D81249B192F8AD
:1087E000E4328888096803F001031B0100FA03F3EF
:1087F0008B610023C2F8E8327047D2F8D8326BB1EF
:1088000018689B8810B44469234218BF1B04323196
:108810005DF8044B8361C2F8E81270473231C2F848
:10882000E8127047A018002098290020D0E90920FC
:10883000131A58425841704790F84F3830B53BB939
:1088400090F84D1890F84E380124DAB2914200D8D1
:1088500030BDB0F8565804FA03F22A43A0F856285F
:108860000133F2E70379024613F0010006D0D2E9A2
:108870000731D2685B1A013A03EA0200704710B56B
:10888000037913F0010304460ED0FFF7EBFF034614
:1088900050B1226A6369E1689B5C0132B2FBF1F07E
:1088A00001FB1022DBB22262184610BD03799B0740
:1088B0000AD5436A8269D154436A02690133B3FB22
:1088C000F2F102FB11334362704770470171704748
:1088D0000379014613F0020007D00B69D1E90921A1
:1088E000013B521A1A40D2B2981A7047074AD2F87E
:1088F000D8324BB192F8E4229988186802F001024C
:10890000130101FA03F383610020704798290020C6
:108910004FF40070034B1060D3F8F8320B60002066
:10892000704700BF98290020002070470120704741
:1089300001207047002070470123437700207047D3
:1089400008B503468269006BD96A02449A6101B195
:108950008847002008BD00BF436A1B681B6A5B682C
:108960005B78024613F0010008BF5077704700BFE4
:10897000F0B5214C214A224B95B0054604F10C007C
:10898000CDE90002049304F110000023CDE90503B2
:10899000CDE90E331B4A09920B93221D10931393BA
:1089A00011936B6A2F7F0A921868012302228DF8B7
:1089B0000C3007938DF820308DF834308DF8483026
:1089C0003B1D02920E460C9353F02CF98FB1330EDF
:1089D00063710634320C330A22706370A670686AC1
:1089E00069464AF0B5FF6B6A186853F01BF915B079
:1089F000F0BD0534EEE700BF00000020C02C0020D1
:108A0000598900083989000810B5044694B05022ED
:108A10000649684656F04CFB606A69464AF098FF82
:108A2000636A186853F0FEF814B010BD2CF6050800
:108A3000C2628161704700BF2DE9F0410446406A7F
:108A400000681E460F46904653F0ECF8237FA0695D
:108A5000002B35D0234D030E6B75052205F116034F
:108A60009870EA64020C000A58701A703B68AB6593
:108A70000020D8F800302B66012E2363286724D00D
:108A8000022E1BD1D8F80420A866796885F8640006
:108A9000E966134414496A670120236385F8780066
:108AA000E967124B627F606AA3F11401002A08BFD4
:108AB00019464AF04DFFE36A73B1206BBDE8F081BF
:108AC0000B4B0422A3F11505CAE7074B85F8646038
:108AD000C5E91A306867E4E7636A186853F0A2F8DA
:108AE000EBE700BF000000204189000830000020B3
:108AF0001500002000B583B081610192049A0093B3
:108B0000C26201236A4601A9FFF796FF03B05DF830
:108B100004FB00BF043070470D4B93F83023D3F8AB
:108B20002C130244D2B283F8302393F8302301444B
:108B30001206C3F82C1305D593F8302382F0800277
:108B400083F83023034B012283F89420704700BF41
:108B500098290020000000202DE9F047154FD7F894
:108B60003453ED0A20D00026B14607F55B7874191E
:108B7000D7F838331048D3F828A0C7F8649304EB2B
:108B8000D474641010234246E102D0470F280BDD55
:108B90000A4B03F1100153F8042B013207D18B4229
:108BA000F9D12546B542E2DCE802BDE8F087661C53
:108BB000F8E700BF98290020D02C0020042D0020C9
:108BC00030B585B068464CF089F91048104AD0F8A5
:108BD000FC10009B0F4D4FF0604441F08071C0F8D5
:108BE000FC10002100F1C840C4F8B05FA0F565009A
:108BF00051601168084CA0F67D60A0FB030341F0B2
:108C000001019B0CA360116005B030BD00ED00E0D8
:108C1000001000E055CEACC5A018002010B54FF4F0
:108C20004010104C82B04CF0C9F9002301210222FF
:108C3000CDE9002120461A464FF4C05152F0ACFF56
:108C4000636A23F470236362636A43F420236362DC
:108C5000636A23F470436362636A43F4204363628C
:108C600002B010BD0000024010B5044655F024FDCE
:108C700081B22046BDE81040FFF77EBA38B50B4DF3
:108C800000EB400005F28C6303EBC00393ED027A26
:108C9000D3ED037AE7EE007AC4002544B0EE670A0C
:108CA00055F00AFDD5F88C36186038BDA0180020A4
:108CB00010B5044655F000FD81B22046BDE81040D5
:108CC0003AE400BF38B5194B93F8242693F82536BB
:108CD0009A4226D1164A92F87C530DB34FF0000CFD
:108CE00002F560726146136859621868083261F3D0
:108CF000C710186032F8040CD862186840F0800081
:108D00001860186861F341001860DC6832F8020CE2
:108D10000CF1010C20436545D86022F8021CE2DC0E
:108D200038BD53F033FA0028D4D138BDA018002044
:108D300098290020F8B50C4B1D685A69154005406C
:108D40005D617DB1094F0126B5FA85F4C4F11F04B8
:108D500007EB840306FA04F4D3F8C00303689847CA
:108D6000A543F1D1F8BD00BF003C01409829002087
:108D70002DE9F8430269C36812EA030828D00546C2
:108D80000E464FF00047B8FA88F327FA03F2D243B1
:108D90001B3B2A6108EA0208042B16D8DFE803F01F
:108DA000332A221A0300B36A002B35D003F1FF39AE
:108DB00000231FFA89F9B362746A34B1236820462C
:108DC000494698476468002CF8D1B8F1000FDAD111
:108DD000BDE8F8837068A98E03689847B8F1000F62
:108DE000D1D1F5E7B068298F03689847B8F1000F33
:108DF000C9D1EDE7F068E96B036889B29847B8F12B
:108E0000000FC0D1E4E73069296C036889B2984744
:108E1000B8F1000FB7D1DBE7EB6A1FFA83F9CBE7B4
:108E200038B51E4CD4F8BC3273B1D4F8C022D4F893
:108E3000BC329A4208D0D4F8C032E218013392F81A
:108E40000004C4F8C03238BD154AD2F8E82900231E
:108E5000526AC4F8C03292F8531001F0FF05B1B164
:108E6000B2F8505082F853305DB10E49D01C10F862
:108E700001CF01F801CB0133B2F850C09BB29C4541
:108E8000F5D809484023043201214DF05BF9C4F8BC
:108E9000BC52D4F8BC020028CDD1D4E798290020D8
:108EA000A0180020982D00208422002090F8503037
:108EB0005A1C0344D2B280F8502083F83C1090F83A
:108EC00051300BB1132A01D954F0C0B8704700BF1C
:108ED000002280F8512054F0B9B8F8B5A0F6680423
:108EE0002379DB0727D5657994F84C3805F001071D
:108EF0003D460BB3D4F848341A68D36A5B08536212
:108F000094F8503823B1B4F85A380133A4F85A38D9
:108F1000636C85F001025979186852F0FBFB01235C
:108F200084F84F38002384F84D3884F84E38A4F87C
:108F3000563884F84C38F8BD94F84F68012E04BFB9
:108F400094F84D3884F84E382046FFF775FC636C72
:108F50004EB9012284F84F287A4059791868BDE843
:108F6000F84052F0D7BB002284F84F283A46F4E785
:108F700070B5094C05460926013E00D170BD94F933
:108F8000000017F0F3FC031E04DBEA18617811728D
:108F9000A278EA540434EFE77CF605082DE9F8439B
:108FA000DDF820800F4615460021202204461E468B
:108FB00056F0D6F8B8F1000F0CD0D8F80030E381A5
:108FC0001B0C2382D8F80430B8F80A20E3821B0C6B
:108FD00062822383384654F05DF8EB0619D4431EB1
:108FE000B8B107EB000C01E0013B12D31CF801ED16
:108FF000BEF12E0FF8D1C01A421E032AA8BF0322C9
:10900000082B03F10109A8BF08239046B9441A466A
:1090100006E008280246B946A8BF08224FF000081B
:109020004FF02033394623606360204656F040F805
:1090300004F10800154B238142464946837056F0DF
:1090400037F8611EE21D11F801CFACF16103192B55
:109050009CBFACF1200C81F800C09142F3D104F127
:109060000A0011F8013FA3F16102192A9CBF203BBD
:109070000B708142F5D118232373330CA382E57260
:10908000099B6683E361BDE8F88300BF20202000D0
:109090002DE9F04FD648DFF888B3006887B0CBF8E9
:1090A000D402002B5ED09C18A046154601F5FE7632
:1090B0000C461DE0002D62D0DBF80433AB4200F01B
:1090C000C580DBF80033AB4200F0F780DBE9C2314A
:1090D000AB424BD8A94200F27281691A204650F087
:1090E00089F90135454504F5007406F5007639D057
:1090F000DBF81033AB42DDD8DBF82073EB1A396BA9
:10910000DA0802328A4203F0070A02D3BB6B9A42A2
:109110000BD939461046039250F03CF9039A0746A2
:10912000002800F08681CBF820033B79002B40F02B
:109130001D81D7F82890B9F1000F00F073813B6BC7
:10914000D21AFB680AEBC20203EB422220463B46DE
:109150004FF400710135C847454504F5007406F524
:109160000076C5D1002007B0BDE8F08FA942B4D980
:109170004FF400720021204655F0F2FFB1E74FF4A2
:1091800000722946204655F0EBFF802384F8BE315B
:109190000C2384F8C231DBF80013964ADBF8F8326E
:1091A000C4F8C6119142C4F8CA3100F30D81924A45
:1091B000924F82FB010287FB01070A44C817C0EBEC
:1091C0006212C0EB27308E4F84F8C10187FB02C7C3
:1091D000C2EB821C8010A1EB0C01013120F03F009A
:1091E00017440843D117C1EBE7110A4484F8BF21A3
:1091F000804A84F8C001013B934200F3F1807E4A2B
:109200007E4882FB031280FB03101A44D917C1EB7E
:109210006212C1EB20317A4884F8C51180FB0270DC
:10922000C2EB82178910DB1B013321F03F01104490
:109230001943D317C3EBE0131A4484F8C41184F81C
:10924000C3214AF65523A4F8FE314AE74FF0FF3315
:1092500084F8EC3184F8ED3184F8EE3184F8EF31A4
:109260005223237063706123A37084F8E731412394
:10927000E37084F8E6317223002784F8E43184F83F
:10928000E531DBF81833C4F8E8314FF4F0723946B1
:10929000201D55F065FF552384F8FE316FF055030E
:1092A000C4F8F071C4F8F471C4F8F87184F8FC7172
:1092B00084F8FD7184F8FF3113E74FF40072002148
:1092C000204655F04DFF4F4B03CB45F6EB03238073
:1092D00090230222C4F80710A3700821F823C4F8D1
:1092E0000300617322746375DBF8F8322273A27392
:1092F00084F82C20DBF800239B1A2362DBE9C223CD
:109300009B1A63620023E372E3736377A377E377C7
:1093100084F82D3084F82E3084F82F3084F83130E2
:10932000394BA361394BC4F842303E2323770123E4
:1093300084F83030364A802384F8403084F8461070
:109340004AF65521A4F8FE1103CA324BC4F847006F
:10935000C4F84B1003CB1388A4F84F309378C4F8AB
:109360005200C4F8561084F85130BAE64FF4007237
:109370000021204655F0F4FEBAF1000F60D13B6C9D
:1093800004F12009002B00F097803B6B2249112249
:10939000CDE900AA2046FFF701FE3B6C1A6C002ABB
:1093A00000F099801B6B1D49CDE900AA48461122A7
:1093B000FFF7F4FD04F140094FF4E07387E0E91A88
:1093C000204650F017F88CE6FF2284F8C1214FF6B2
:1093D000FF72A4F8BF21074A013B93427FF70FAF0A
:1093E000FF2384F8C5314FF6FF73A4F8C33128E793
:1093F000A0180020FF03FB008320088297554541F9
:1094000081808080FC7006083F00FF0029940E0DCB
:109410000871060814710608F4700608F87006084A
:109420009829002049464FF40072204655F098FED6
:1094300057E62D4A231F43F8042F9E42FBD150E6E6
:10944000D7E910274FEA0A13002A42D0023B002F27
:109450003FF447AE013BBF6CF9D1A1464FF4007316
:10946000002F3FF43EAECDE9035609EB030A059405
:1094700008E00024CDE90064FFF790FDBF6CBFB1A8
:10948000D14515D03C7939683B6B484607F11C063D
:10949000112209F12009002CEBD17A793C6942F0C4
:1094A0002102CDE90064FFF779FDBF6C002FE7D101
:1094B000DDE90356059C14E6CDE900AA5346DBF826
:1094C000FC1208222046FFF769FD4FF4F0737F6C11
:1094D000C6E7013BBBE7CDE900AA0449534648462D
:1094E0001122FFF75BFD65E7DEADBEEFF870060801
:1094F00038B590F82830012B044606D0407F08B9D3
:10950000012038BD0023637738BD406A03681A7BA9
:1095100092B9637F002BF3D00A4D0B49022305F566
:1095200040624AF0CFF995F8013CD84303F00103BB
:1095300000F001006377E7E71B6A002BE9D0002009
:1095400038BD00BF982900209800002038B5044697
:1095500094F82830012B07D0637F0BB10023637789
:10956000012038BD1B6A23B1606A03681A7B002A98
:10957000F8D1637F002BF3D0074D0849022305F58E
:1095800040624AF09FF995F8013C03F00102DB07C5
:109590006277E5D5DCE700BF98290020980000201D
:1095A00010B4EFF31183102282F31288094A0A4C97
:1095B00011684FF0E0200131116081695160002293
:1095C000C4F8042C0269DBB283F311885DF8044B04
:1095D000704700BFA01800209829002030B4EFF396
:1095E0001183102282F312884FF0E0220E48946912
:1095F0001169C90344BF0121C0F8041C0B4948BFCD
:1096000094690D68D0F8042CDBB283F31188896863
:109610004FF47A702A4400FB01F31B1B30BCB3FBF0
:10962000F1F300FB0230704798290020A0180020B9
:10963000224B5B68C3F3080330B4D3B9EFF3118353
:10964000BBB91F4B4FF0E02C1A68DCF81800196802
:109650008A42F9D159688842F6D89C684FF47A71E9
:1096600001FB04F3181AB0FBF4F030BC01FB02005C
:109670007047EFF31182102383F312884FF0E02339
:1096800010489C691969C90344BF0121C0F8041C32
:109690000B4948BF9C690D68D0F8043CD2B282F3F4
:1096A000118889684FF47A722B4402FB01F0001B89
:1096B00030BCB0FBF1F002FB0300704700ED00E0AE
:1096C000A0180020982900202DE9F047FFF7B0FFEF
:1096D000214D224F2C6906464FF000094FF0AC088F
:1096E000002C2DDD00231A4608FB0351013391F8AD
:1096F000B1109C4242EA0102F6D142EA090A5FFA3D
:109700008AFA91467B68C3F30803B3B9EFF3118378
:109710009BB9FEF775FC801BB0F5FA6F02DCB9F15E
:10972000000FDDD1BAF1000F04D00D4B93F8082CD7
:10973000542A09D05046BDE8F087FFF74FFFEAE70B
:10974000CA464FF00009DDE7B3F8102C0132A3F848
:10975000102C5046BDE8F087A018002000ED00E076
:1097600098290020AD4B1B7B0BB901207047AB48FB
:10977000AB490268AB4B2DE9F04FA1FB0212520935
:10978000A3FB0213DB08A84903EB8303A2EB43030B
:1097900085B0DAB201F61C44039204EB830791F81A
:1097A000D022029201F6FC63002500F5317BA84629
:1097B0009946029B984500F00E81DBF81820DBF8F3
:1097C0000460D2F89430D2F898500093B600FFF7B6
:1097D0002FFF009B019006F1085606EB4316934BB2
:1097E00013F8F4CC904B93F8082C05F180603938CD
:1097F000542A06EB801006EB8C1302D18A49A1F89B
:1098000012CC984240F281811968002900F07681DB
:10981000196C002900F08B81D3F88010002900F02A
:109820008881D3F8C01003F580730029E9D19E1B0D
:1098300098424FEAA61640F26881A91B45294FF0CD
:10984000000528BF45212846AE4603EB81119A4604
:1098500015460DE01A6C002A40F0F080D3F8802005
:10986000002A40F01B81D3F8C02003F580732AB989
:10987000994206D91A68002AECD04033994200F286
:10988000E1802A467546112D40F24781DEF115012F
:1098900000F14381664BD3F89C309E423CBF644B41
:1098A000C3F89C60614B019E53F8F03CF61A002E01
:1098B0001CDB019E03F5F42303F590739E4288BFE1
:1098C00033465A4E88BF053346F8F03C584B574E46
:1098D000D3F89C30052B86BF053BDBB2002306F88E
:1098E000F43C534E4FF0FF33C6F89C3031B100FAD0
:1098F00001F1C5F114050120A84008434D4BC0F308
:10990000C43103EB8101D1F8C45000F01F0103EB17
:109910008101D1F8C41041EA0531C0F3441503EBCD
:109920008505C0F3842003EB8003D5F8C400D3F889
:10993000C43041EA001141EA032181EA112383EA9C
:10994000131303F00F00384BD3F8043F0F2803F133
:10995000010340F0C080B1F5803F80F0BC80542A04
:109960004FEA11113ED0304AB1F5606FC2F8043FA2
:1099700044D0A9F80C1094F85830039883420CD0C6
:10998000BA6823689B1A23603A6B63689B1A63600A
:109990000023BB603B6384F85800236801332360D5
:1099A000BB680133BB604FF6FF73994205D1636812
:1099B000013363603B6B01333B6308F10108B8F18D
:1099C000080F04F15C0407F15C0709F114090BF1BD
:1099D000200B7FF4EEAE184B012201201A7005B067
:1099E000BDE8F08F1048B0F80C2C0132A0F80C2C18
:1099F0000D4AB1F5606FC2F8043FBAD1074A92F838
:109A0000253603EB430302EBC303434493F8353697
:109A10000D2BAED1802389F81E30ACE7A0180020B2
:109A20001F85EB51CDCCCCCC98290020903A00205A
:109A300000000020D8F505089839002080339942AD
:109A40007FF61FAFA3EB0A0C3E4A4FEAAC1C0CF1A9
:109A5000010C82FB0CA2A2EBEC72012AB8BF01221E
:109A600090404FF0010C9644013A0CFA02F2104378
:109A70009C46DCF800209AB1DCF84020002A5AD03D
:109A8000DCF88020002A59D0DCF8C0200CF5807C5E
:109A900042B16145EDD89A466346E9E6C033EDE64A
:109AA0000CF1400C6145F6D9ACEB03029211254B49
:109AB000013283FB02A3A3EBE273012BB8BF0123A6
:109AC00098409E440122013B02FA03F31843634687
:109AD0009A466346CCE6542A05D11B49B1F80C2CB2
:109AE0000132A1F80C2C184AC2F8043FD2F8003F0A
:109AF0000133C2F8003F4FF6FF713CE740339E1B35
:109B000098424FEAA6163FF698AEBCF1000F04D07B
:109B10000E4B0CF1FF3C03F8F4CC542A7FF44DAF0C
:109B2000094AB2F80E3C0133A2F80E3C45E78033F7
:109B30007DE6C0337BE60CF1800CB3E70CF1C00C82
:109B4000B0E700BF5655555598290020903A00209F
:109B500070B51E4C94F8242694F825369A422FD1DD
:109B60002569002D10DD1A48267B0024FEB1037EF6
:109B7000012B1FD002691368013443F00103A54291
:109B800000F1AC001360F1D1FFF752FD114B53F817
:109B9000EC4C002C0ADDE83B03EBC40419689A88FE
:109BA000C86808330243A342CA60F7D170BDFEF70C
:109BB00081FBDFE7002380F89C30FEF77BFBD9E7D1
:109BC00052F0E4FA0028CBD170BD00BFA0180020ED
:109BD000B4180020903A00202DE9F04FD0F8009002
:109BE000057CD9F800304FF0020A0AFA05F52B423D
:109BF00083B002D103B0BDE8F08F4169DFF888B2CD
:109C00009F4B4FF04C0808FB01B804465868D8F841
:109C1000CC33B8F8D0231F68D8F80464FB6823EA73
:109C20000203984AFB6042F8C80C336823F0010332
:109C300033609BF80C3023B9C9F8045003B0BDE879
:109C4000F08F304601914BF0C7F98E4A01990123FC
:109C500088F8F03352F8C03C002B00F005813B68D7
:109C600023F080033B604C2303FB01B34FF0FF3034
:109C700093F80034F862062B2FD8DFE813F0CD00FC
:109C80002E00A5002E0007002E0083003B6A23F45F
:109C900080733B624C2303FB01B33C6A93F80104DD
:109CA00060F349243C623C6AC0F3400060F3CB247B
:109CB0003C62F86993F8024464F30100F86193F898
:109CC0000304FB6960F30713FB61FB6923F00C03DA
:109CD000FB613B6A43F480733B624C2303FB01B39B
:109CE00031684BF6EF7421400024A3F8E44331605F
:109CF0003068B3F8E41301433160316893F8ED0341
:109D000060F30D313160316893F8EB0360F38B2120
:109D10003160316893F8EA0360F3092131603168FA
:109D200093F8E90360F3C7113160316893F8E803F1
:109D300060F38611316093F8EC03316860F34511EC
:109D40003160B3F8E603716860F30F017160D3F816
:109D5000DC03D3F80414B060D3F8E003F0601620FD
:109D60004860086840F001000860D3F8CC13B3F8ED
:109D7000D03309684248CC682343CB60436842F83B
:109D8000C43C59E73B6A23F480533B624C2303FBFA
:109D900001B3386A93F8014464F34D303862F869CE
:109DA00093F8024464F30920F86193F80304FB6913
:109DB00060F30F33FB61FB6923F44063FB613B6A93
:109DC00043F480533B6288E73B6A23F010033B6215
:109DD0004C2303FB01B33C6A93F8010460F3451480
:109DE0003C623C6AC0F3400060F3C7143C62B8694F
:109DF00093F8024464F30920B86193F80304BB6943
:109E000060F30F33BB61BB6923F44063BB613B6A02
:109E100043F010033B6260E73B6A23F001033B62BF
:109E20004C2303FB01B33C6A93F8010460F3410443
:109E30003C623C6AC0F3400060F3C3043C62B86912
:109E400093F8024464F30100B86193F80304BB691A
:109E500060F30713BB61BB6923F00C03BB613B6A72
:109E600043F001033B6238E7FFF7E2FB054A257C3C
:109E7000D4F80090019942F8C00C0AFA05F5EEE614
:109E8000001000E0903A0020A01800202DE9F047D3
:109E90000546FFF7CDFB244E244B254F04464FF0DB
:109EA00010084FF0E02C4FF47A7E4FF001097268F1
:109EB000C2F30802CAB9EFF31182B2B91A68DCF82A
:109EC000180019688A42F9D159688842F6D8D3F83F
:109ED00008A00EFB0AF1091AB1FBFAF10EFB0212FF
:109EE000121BAA42E3D3BDE8F087EFF3118288F397
:109EF0001288DCF81800DCF81010C90344BFC7F85A
:109F0000049CDCF818001968D7F804ACD2B282F3CC
:109F100011885144D3F808A00EFB0AF2121AB2FBC2
:109F2000FAF20EFB0122DBE700ED00E0A0180020B2
:109F3000982900202DE9F0473C4B3D4D3D4E00F166
:109F4000FF3810274FF0E0204FF47A7C6A68C2F3A4
:109F50000802002A54D1EFF31182002A50D11A6866
:109F6000846919688A42FAD159688C42F7D899688D
:109F70000CFB01FEAEEB040E4FF00109BEFBF1FE3F
:109F80000CFB02EE6A68C2F30802EAB9EFF3118231
:109F9000D2B91A68846919688A42FAD159688C4220
:109FA000F7D8D3F808A00CFB0AF1091BB1FBFAF1B2
:109FB0000CFB0212A2EB0E02B2F57A7FE2D3B8F1EB
:109FC0000108C3D2BDE8F087EFF3118287F312884E
:109FD00084690169C90344BFC6F8049C846919688F
:109FE000D6F804ACD2B282F311885144D3F808A059
:109FF0000CFB0AF2121BB2FBFAF20CFB0122D9E7AE
:10A00000EFF3118187F3128884690269D20303D5C3
:10A010000122C6F8042C8469D3F800E0D6F8042C99
:10A02000C9B281F311887244A1E700BFA0180020D3
:10A0300000ED00E0982900202DE9F04F01308E4C12
:10A040008E4D8F4E83B001F1FF385FFA80FA1027F2
:10A050004FF016FF4FF4FA7B4FF0E0224FF47A7C7A
:10A06000C1466B68C3F30803002B40F0CB80EFF3CD
:10A070001183002B40F0C6802368916920688342D9
:10A08000FAD160688142F7D8D4F808800CFB08F058
:10A09000A0EB010EBEFBF8FE0CFB03EE4FF0010837
:10A0A000CDF804906B68C3F30803002B40F08E805A
:10A0B000EFF31183002B40F08980236891692068B9
:10A0C0008342FAD160688142F7D8D4F808900CFB3B
:10A0D00009F0411AB1FBF9F10CFB0313A3EB0E03DA
:10A0E000B3F57A7FDED3BBF1010BDDF80490B8D174
:10A0F00050464FF47A7B50F07BFB4FF0E022DC4679
:10A100006B68C3F30803002B40F09980EFF31183D1
:10A11000002B40F094802368916920688342FAD133
:10A1200060688142F7D8D4F808800CFB08F0A0EBF7
:10A13000010EBEFBF8FE0CFB03EE4FF00108CDF85C
:10A1400004906B68C3F3080323BBEFF311830BBBCD
:10A150002368916920688342FAD160688142F7D808
:10A16000D4F808900CFB09F0411AB1FBF9F10CFB93
:10A170000313A3EB0E03B3F57A7FE2D3BBF1010B1C
:10A18000DDF80490BCD1B9F10108BFF461AF03B0B0
:10A19000BDE8F08FEFF3118387F31288906911699E
:10A1A000C90344BFC6F8048C90692168D6F8049CA2
:10A1B000DBB283F311884944D4F808900CFB09F30F
:10A1C0001B1AB3FBF9F30CFB0133D2E7EFF3118356
:10A1D00087F3128890691169C90344BFC6F8048CDB
:10A1E00090692168D6F8049CDBB283F31188494456
:10A1F000D4F808900CFB09F31B1AB3FBF9F30CFB22
:10A2000001336BE7EFF3118087F3128891691369CB
:10A21000DB0303D50123C6F8043C91692368D6F813
:10A2200004ECC0B280F31188A06873440CFB00FEFC
:10A23000AEEB010EBEFBF0FE0CFB03EE2EE7EFF3E0
:10A24000118087F3128891691369DB0303D5012319
:10A25000C6F8043C91692368D6F804ECC0B280F3D8
:10A260001188A06873440CFB00FEAEEB010EBEFB30
:10A27000F0FE0CFB03EE60E7A018002000ED00E00C
:10A28000982900202DE9F043144CDFF8549083B056
:10A2900004F520764FF0020802E00834B4421AD0E8
:10A2A00094F90650002DF8D1276807F13F4303F5D4
:10A2B0007E0309EB9323083493F8440150F062FEC7
:10A2C00034F8041C0123CDE900582A46384651F0E1
:10A2D00063FCB442E4D103B0BDE8F083D43900207C
:10A2E000D8F5050830B50C4683B00546D8B10368EB
:10A2F00003F13F4303F57E039B0A0C4A134493F892
:10A30000440150F03FFEC4F3810204F00303CDE9A1
:10A310000032C4F34113A9882868C4F3001251F035
:10A320003BFC03B030BD4FF0FF33E6E7D8F505083E
:10A3300000B1D7E7704700BF70B50E4B93F8D062FD
:10A34000AEB10D4C002504E00135B54204F1200406
:10A350000DD0237F002BF7D0E0680028F4D0217DBA
:10A360000135FFF7BFFFB54204F12004F1D1012010
:10A3700070BD00BF98290020641B002070B40D4AF6
:10A380000D4E0E4C0E4D4FF0010C36F8020F00230F
:10A3900040FA03F1C90704D50CFA03F11460918067
:10A3A00008320133102BF3D104F58064AC42ECD1B8
:10A3B00070BC7047D439002022F705080000024025
:10A3C0000020024038B50409013C072C1AD80F4D73
:10A3D00005EB440200F00F03B2F84C0140FA03F21F
:10A3E00012F0010210D0012202FA03F3013B1840DF
:10A3F000254454F049FF95F85C31054A034402EBCB
:10A40000C30038BD002038BD104638BDD8F505085A
:10A41000D4390020F8B50268017C04460223106894
:10A420008B40184206D1106808238B40184218BF91
:10A430005360F8BD6569536004238B405360EFF3AC
:10A440001183502282F312882A6C1168C9070BD538
:10A45000DBB283F3118895F86C3013B195F87D6009
:10A46000FEB12268217CDEE7506880B288B9D5E968
:10A4700009618E422BD0AF690F44D76089B222D8D0
:10A4800006462869401A80B250600021AE6285F805
:10A490006C10116841F00101DBB2116083F3118887
:10A4A000D9E795F87A00FFF78DFFAB6EDA680121E6
:10A4B00066F3C302DA6085F87D100028D1D0282128
:10A4C000FFF710FFCDE7711A89B25160DDE7012275
:10A4D00085F86C20BCE700BF174A1849D2F88830CD
:10A4E00030B443F47003C2F888300B6843F00103C2
:10A4F0000B600B689B07FCD58B68104A23F00303A5
:10A500008B60936813F00C0FC3F38101F9D1916054
:10A51000136809480A4D23F0867323F480331360CF
:10A520004FF41F044FF000635560C2F8A010D460D0
:10A5300030BC8360704700BF00ED00E0003802408F
:10A5400002300300704700BF002070470148FEF74B
:10A55000EBB800BF6C3C00200148FEF7E5B800BF37
:10A56000C03C00200148FEF7DFB800BF143D0020CA
:10A5700030B1036882881B691A4214BF0120002091
:10A58000704700BF10B1036882889A62704700BFAD
:10A5900010B1036882889A61704700BF2DE9F04FBF
:10A5A000076889B07D680790D7E904607168AA6878
:10A5B00012F08002FBD1BB69347C93F80EE0069266
:10A5C0000EF0030ECDF814E093F80DE0326893F826
:10A5D000119093F80F8001920EF0010A93F80CE0AD
:10A5E0005A8903920EF0010E4FF0020CCDF810E0E4
:10A5F00093F810E01A6802920CFA04F40EF0010BC2
:10A6000044F00C04B3F808E05B6809F0030908F0B3
:10A610000308002800F08680019A079E466146687C
:10A620005460047C0068069A0CFA04F444F00C04AC
:10A630004460086862F300000860306862F300005C
:10A640003060326842EA0C0232600A684BF6EF7002
:10A6500002400A600A684EEA02020A600A6869F368
:10A660000D320A600A6868F38B220A600A68059C4A
:10A6700064F309220A600A686AF3C7120A600A686A
:10A68000049C64F386120A600A686BF345120A6040
:10A690004A68039C64F30F024A60029A8A60CB60A6
:10A6A0003268FB690240326030681A8902433260C6
:10A6B0003268587C60F30D3232603268D87B60F3C8
:10A6C0008B2232603268987B60F3092232603268F4
:10A6D000587B60F3C71232603268187B60F38612D1
:10A6E0003260187C326860F34512326058897268B3
:10A6F00060F30F027260D3E90023B260F360336845
:10A7000043F0010333600B6843F001030B606B6897
:10A7100043F001036B606B6843EA0C036B6009B0A4
:10A72000BDE8F08F079A7261019A54600A6860F37D
:10A7300000020A600A684BF6EF7002400A600A687D
:10A740004EEA02020A600A6869F30D320A600A687A
:10A7500068F38B220A600A68059860F309220A6090
:10A760000A686AF3C7120A600A68049860F38612DE
:10A770000A600A686BF345120A604A68039860F33E
:10A780000F024A60029A8A60CB600B6843F00103B3
:10A790000B600B6843F002030B606B6843F002032D
:10A7A0006B6009B0BDE8F08F70B4046890F8385061
:10A7B0006368012284F824201A6822F040021A609B
:10A7C000B0F804C02289624516D0BCF5807F61468E
:10A7D000A8BF4FF480710229B8BF02211A6891FA0C
:10A7E000A1F1B1FA81F122F03802013942EAC10245
:10A7F00092B21A60A4F808C0027BA17A914209D0F3
:10A80000196872B321F002011960196821F0010181
:10A810001960A2721A6842F040021A60226A267B0E
:10A820009368C3B100218C4614329C449368013173
:10A83000002BF9D196B18DB1012909D8BCF1070FD0
:10A8400006D801EB81018B00226A13441B7B2BB9D4
:10A8500070BC49F091BC0EB1002DF5D170BC49F02F
:10A86000BBBC41F002011960196841F00101196097
:10A87000A272CFE738B52C4AD0F890305268D0F8A1
:10A880008810044673B1501A83420BDC94F8803070
:10A89000C4F88820012B10D0D4F884300133C4F8D8
:10A8A000843038BDD4F89430C4F888200B44C4F800
:10A8B0008C3094F88030012BEED16168201D04F1BA
:10A8C0009805EFF3118C102383F3128863681B6AD9
:10A8D0000BB3D4F8A0302A461BB1D3691432002B35
:10A8E000FBD10B6A6BB1996839B9934209D01968E9
:10A8F00029B15B6899680029F7D01433F3E7C3E9FD
:10A9000000055FFA8CFC8CF31188D4F88430013395
:10A91000C4F8843038BD0D625FFA8CFC8CF311886A
:10A92000FFF742FFB8E700BF001000E02DE9F0415B
:10A93000826992F88C30012B8AB0054649D0023BDF
:10A94000012B50D892F8FC30D26C2D4C63F07F0371
:10A95000137087693B6DD7F8108003F1010E0FCC9F
:10A96000EC46ACE80F00FB6CCDE9003E0FCCACE848
:10A970000F0094E8030007F110068CE80300EFF3E2
:10A980001180102383F312883B691B6A002B2ED0A1
:10A99000029B6A461BB1D3691432002BFBD1D8F855
:10A9A000203073B1996839B99A420AD0196829B12F
:10A9B0005B6899680029F7D01433F3E71E60C3F889
:10A9C00004D0C0B280F31188AA6911690B6A002B08
:10A9D000FCD1136D5A8852BAEA819A8852BA2A82F7
:10A9E000DB885BBA6B8201200AB0BDE8F081C8F851
:10A9F00020D0C0B280F311883046FFF7D5FEE3E7E0
:10AA00003CF705082DE9F04190F88C30056D012BDD
:10AA10008AB004466FD03ED9023B012B67D890F82C
:10AA2000FD30C26C5A4E63F07F031370036DD0F893
:10AA3000108003F1010E00F110070FCEEC46ACE8D8
:10AA40000F00E36CCDE9003E0FCEACE80F0096E8B6
:10AA500003008CE80300EFF31180102383F31288C6
:10AA600023691B6A002B00F08A80029B6A461BB197
:10AA7000D3691432002BFBD1D8F8203023B3996866
:10AA800039B9934220D01968D9B15B689968002917
:10AA9000F7D01433F3E7C36C4FF0FF321A605A60FB
:10AAA0009A60DA60D0F890300522B3F57A7FC0F86A
:10AAB000A0203BD8032380F88C3001200AB0BDE8E9
:10AAC000F0811F60C3F804D0C0B280F311882269FE
:10AAD000136A002BFCD16B885BBAA4F88030AB887A
:10AAE0005BBAA4F88230EB885BBAA4F8843001200A
:10AAF0000AB0BDE8F08190F8FC2090F8FD309B1A78
:10AB00005B100133DBB205EB430235F813305BBA5F
:10AB1000A0F8803053885BBAA0F8823093885BBA83
:10AB2000A0F8843001200AB0BDE8F08103691A7BE7
:10AB30000AB35B69FBB190F84830E3B190F8FC30A0
:10AB4000C26C606563F07F03137090F8FC1090F89E
:10AB5000FD30026D0F48C4F8B4005B1A07330121C1
:10AB6000C4F8AC30E36C84F8B0100A44C4E929326C
:10AB700084F88C10BBE7022384F88C30B7E7C8F860
:10AB800020D0C0B280F311883846FFF70DFE9EE753
:10AB90003CF70508DD840008F8B54569002D70D044
:10ABA0002C68236A1B7B002B77D1D4E90467317CA6
:10ABB0006368022202FA01F1D6E9006041F00C015B
:10ABC000002F35D0D0F800C0D7F804E02CF0010CED
:10ABD000C0F800C0DEF8000020F00100CEF8000050
:10ABE0007160397C8A40396842F00C024A605A68C8
:10ABF00022F002025A605A6822F001025A60236A67
:10AC00001B6943B1236A686C1B699847012800F0EF
:10AC10008D80022837D0236ADA69FAB9586900288A
:10AC200042D099692162C3E90522BDE8F840BBE53D
:10AC30009A681706FCD49A68D2070DD4026822F0ED
:10AC40000102026071605A6822F002025A60236AAF
:10AC50001B69002BD6D1DEE7DA68ECE7226A94F8AC
:10AC60002410127B1433D2B22362002937D1002A78
:10AC700055D12846FFF792FC2B681A6AD169002942
:10AC800014DCF8BD2362236ADA691433002AF9D18F
:10AC9000236ADA69002AE1D1C0E7AB68002B84D0CF
:10ACA0001A689B88936180E72062F8BDD06951697A
:10ACB0009C69002963D0012565736160596980B280
:10ACC00060810029DDD092693349DB69002A0ABF1F
:10ACD0000A460121002159735A605881F8BD276A3C
:10ACE0002E68B9683B68B069002B4ED04FF0010C5C
:10ACF00080F80DC043608BB27169438151B1F06936
:10AD000079684381244B00290ABF19460123002397
:10AD100041604373002384F82430002AA9D0AB6833
:10AD2000002BA6D01A689B889362A2E7236A2A6840
:10AD3000143B2362136AD96900297FF76CAFDE697F
:10AD400059699769A1B1844687F80DC07960B1B29D
:10AD500056697981002E3FF45EAFD2699B695181BB
:10AD60000D49002B04BF00200B465073536052E77F
:10AD70008C460A494FF0FF0E01F8A0EFE4E70D46BC
:10AD80000649FF2601F8A06F96E79C46034B4FF05B
:10AD9000FF0E03F8A0EFABE7A43D00200000002069
:10ADA00008B51D20FFF70EFB10B190F9063053B126
:10ADB0001E20FFF707FB10B190F9063003B108BD64
:10ADC0005523C38008BD5523C380F1E70348D0F85D
:10ADD000B0300BB1A4301847704700BF000000200E
:10ADE0000348D0F8D4300BB1C8301847704700BFC3
:10ADF000000000200348D0F8F8300BB1EC301847C1
:10AE0000704700BF000000200348D0F81C3113B188
:10AE100000F5887018477047000000200348D0F8FC
:10AE2000403113B100F59A701847704700000020B8
:10AE30000348D0F8643113B100F5AC70184770477F
:10AE4000000000200348D0F8883113B100F5BE702F
:10AE500018477047000000200348D0F8AC3113B108
:10AE600000F5D07018477047000000200348D0F864
:10AE7000D03113B100F5E270184770470000002090
:10AE80000348D0F8F43113B100F5F4701847704757
:10AE9000000000200348D0F8183213B100F5037009
:10AEA00018477047000000200348D0F83C3213B127
:10AEB00000F50C7018477047000000200348D0F8D8
:10AEC000603213B100F5157018477047000000207C
:10AED0000348D0F8843213B100F51E70184770474C
:10AEE000000000200F4B1049013800EBC00003EBBD
:10AEF0008003086BD3F8A4200C4B9A4214BF4FF088
:10AF000080734FF48003184382B00863096B0B40D1
:10AF10000193019BD2F8003143F00103C2F80031E4
:10AF200002B0704700000020003802400064024078
:10AF30002DE9F0410138124C00EBC00004EB800415
:10AF40001048D4F8A480804514BF382036200F461E
:10AF500015461E4650F016F8D8F8003143F00103AC
:10AF6000C8F8003194F9B500C4F8B070C5F3011207
:10AF7000A909C4F8B860BDE8F0414AF0F3BA00BFCF
:10AF80000000002000640240D3B20D2B2BD800B586
:10AF9000164B4FF0000C06E00CF1010CBCF1200F39
:10AFA00003F103031CD093F800E08645F4D193F835
:10AFB00001E08E45F0D10E4B0E480CEB4C0C02EB31
:10AFC0004202634400EB820193F88E31C1F8A4324F
:10AFD00000F5277000EB820081F89C325DF804FBDD
:10AFE00000205DF804FB0020704700BF64F70508EF
:10AFF000D8F505080000002010B40C4C002304F51F
:10B00000467C01E0152B0CD003EB430201331CF806
:10B0100002108142F6D1144494F91A035DF8044BEE
:10B0200070474FF0FF305DF8044B7047903A0020B6
:10B0300030B5134C002304F5F67C02E001331C2BE1
:10B040001BD05CF833508542F8D10CEBC30EDD0009
:10B050009EF804E08E45F1D10A4B02EB42022C44EB
:10B0600003EB820194F8F141C1F8A44203F5277380
:10B0700003EB820081F89C4230BD002030BD00BF50
:10B08000D8F5050800000020F0B110B504460F48BF
:10B0900094F804E0002300F5467C01E0152B11D064
:10B0A00003EB430201331CF802107145F6D18318FB
:10B0B000617993F91A232068D3B20D2B02D8BDE829
:10B0C0001040B5E7002010BD00207047903A0020E6
:10B0D000800AA0F58010532806D8044B1B5C0E2B69
:10B0E00002D8034AD056704700207047D8F50508AB
:10B0F000A871060808B5084849F060FF40220748D3
:10B10000002154F02DF8064B4FF0FF32C3F85823BE
:10B11000C3F85B2308BD00BF0E004400582D00207B
:10B12000903A002048B182880449B2FA82F2086855
:10B130004FF00043D34003430B607047003C014095
:10B140000120FDF7F7BD00BF0220FDF7F3BD00BFF2
:10B150000420FDF7EFBD00BF0820FDF7EBBD00BFE9
:10B160001020FDF7E7BD00BF4FF47870FDF7E2BD9A
:10B170004FF47C40FDF7DEBD40B338B505461446BC
:10B18000FFF7B0F8AB882968B3FA83F3C3F11F0364
:10B1900003F00700800013F0F80F04FA00F20AD061
:10B1A0004B6A0F2404FA00F023EA00034B624B6A57
:10B1B0001A434A6238BD0B6A0F2404FA00F023EAEE
:10B1C00000030B620B6A1A430A6238BD704700BF66
:10B1D0002DE9F047DFF854A2542303FB00A384B009
:10B1E000D3F8C481B8F1000F08D0D3E973490746FA
:10B1F000002C00F0D58094F9063013B104B0BDE8FE
:10B20000F087B9F1000F00F0DB8099F90630002BD0
:10B21000F4D1431CDBB21522E371A27189F8073027
:10B22000162389F8063098F828004FF0ABFE204628
:10B23000FFF7AEF94846FFF7ABF919212046FFF7B3
:10B2400077F819214846FFF773F80926332524B902
:10B250009CE0013D06D04FF0DDFD2368A28819690E
:10B260000A42F6D09A624FF031FE2368A2889A61B2
:10B270004FF02CFE013EE9D1332524B98DE0013D8C
:10B2800006D04FF0C7FD2368A2881B691A42F6D08A
:10B290002046FFF777F94FF019FE4846FFF772F99D
:10B2A0004FF014FE2046FFF773F94FF00FFE4846AB
:10B2B000FFF76EF94FF00AFE2046FFF759F9002814
:10B2C0007AD12046542407FB04F40AEB040595F8D0
:10B2D000D63195F8D421002B0CBF162636263146E0
:10B2E000FFF74AFF95F8D52131464846FFF744FF5E
:10B2F00046483C220021204453F032FFD5F8C431A7
:10B3000068465C68C5F8DC4149F0E8FDB5F8D8113D
:10B3100003984EF095FC3E4B9C42054655D03D4B64
:10B320009C425DD03C4B9C4265D0542303FB07A359
:10B33000D3F8DC21136843F001031360236823F082
:10B34000010323602561236843F470632360A368CD
:10B3500023F48063A360A3686FF30903A360A36869
:10B3600043F40043A3600022114698F92A004AF0F2
:10B37000F9F8002298F9290011464AF0F3F82368F9
:10B3800043F00103236039E74FF044FD013DFBD159
:10B390004FF09CFD6CE74FF03DFD013DFBD177E7A1
:10B3A000B9F1000F3FF43FAF99F90630002B7FF45D
:10B3B00025AF7B1CDBB231E74846FFF7D9F880E7C1
:10B3C0001523A371431CE3712DE7144849F0F6FDE2
:10B3D000134AD2F8203823F40013C2F82038A4E727
:10B3E000104849F0EBFD0E4AD2F8203823F48003D0
:10B3F000C2F8203899E70C4849F0E0FD084AD2F835
:10B40000203823F40003C2F820388EE76C3C00207B
:10B410000054004000580040005C0040150020002F
:10B42000003002401600200017002000903A002053
:10B430002DE9F047794D05EB0013D3F86043002C5C
:10B4400000F0A58093F86A7306464FEA0018384664
:10B450004FF098FD7B09012207F01F07013BBA401E
:10B46000042B09D8DFE803F09B03A1A795006C49E2
:10B470004B6923EA02034B6105EB0803013693F89D
:10B480006403FEF79FFFF6B2824610B11223C67125
:10B49000837105EB080393F86503FEF793FF81467C
:10B4A00010B11323C671837105EB080393F866038B
:10B4B000FEF788FF074610B11423C6718371454417
:10B4C000504695F867232621FFF756FE95F8682326
:10B4D00048462621FFF750FE95F869230621384695
:10B4E000FFF74AFE4F4B9C4276D04F4B9C4268D0B0
:10B4F0004E4B9C427BD04E4B9C4200F08380636855
:10B5000002210B436360636843F001036360E369F6
:10B5100023F40063E361236823F40043236023687A
:10B5200023F480432360236823F48063236023682B
:10B5300043F400732360236843F48073236023681B
:10B5400043F004032360636823F40073636063685B
:10B5500023F480736360236861F3C5032360236869
:10B5600023F080032360236823F4006323602368AF
:10B570000B432360236843F0010323602369072200
:10B5800062F30F032361236843F040032360BDE8A7
:10B59000F08723490B6A23EA02030B626CE7204918
:10B5A0000B6923EA02030B6166E71D498B6923EAF5
:10B5B00002038B6160E71A494B6A23EA02034B627C
:10B5C0005AE71C4849F0FAFC1B4AD2F8203823F409
:10B5D0008043C2F8203892E7184849F0EFFC164A39
:10B5E000D2F8243823F48053C2F8243887E714486B
:10B5F00049F0E4FC104AD2F8203823F40043C2F8A2
:10B6000020387CE70F4849F0D9FC0B4AD2F824389F
:10B6100023F40053C2F8243871E700BF903A0020A9
:10B62000003802400030014000380040003C00403B
:10B63000003401400E002000003002400C002400C5
:10B640000F0020000D0024002DE9F04F8FB00023E3
:10B650000793A74BA74CA84FA3F53376A44D4FF003
:10B660000009A64BD5F800B093F8B2234FEA9B230C
:10B67000A3F58013532B00F2CD80F35C0E2B00F268
:10B68000C980012A17F903A000F00581022A02D11E
:10B69000BAF1080F32D14FF001081FFA88F1504675
:10B6A00012F07AFA12F004FB90F9003013B1542B27
:10B6B00040F0018208F10108B8F1050FEDD1079BB8
:10B6C0000021002B00F0B0808A4A09E0F35C0E2BC9
:10B6D0000DD8FB5653450DD0AC32944200F0A180FA
:10B6E000906803689B0AA3F58013532BEED90023BF
:10B6F0005345F1D1437968799842EDD109F10109B7
:10B70000B9F1080F05F11C05ABD1079B0133042BE0
:10B71000079304F1AC04A1D10123DFF8F8B19A46F4
:10B72000774B93F8D0220AF1FF339A426FDD734BC7
:10B73000DBF80C609BF8102093F8C6330892002EBB
:10B7400000F0D583B2883068B2FA82F200F13F404F
:10B75000C2F11F0200F57E000792800A694A15694E
:10B76000002D40F3A8801432002705E00137AF42D6
:10B7700002F1AC0200F09C8011688142F6D1079B77
:10B780005C4ACBF80430AC2303FB0727CBF81870D6
:10B7900026B15FFA8AF3F3710323B371079D7B6CC3
:10B7A000F96B680001220324844002FA00F003438D
:10B7B0007B64544B1B7B2143F96302FA05F4B96C9B
:10B7C000002B00F05C812143B9646EB14B4BB28811
:10B7D00093F8581B3368490141F0050101F0E50178
:10B7E0009A613046FEF77EFD786FA1B20122FCF728
:10B7F00023FC38460AF1010AFCF75CFD40F2011314
:10B80000BAF1090FABF81C300BF1200B88D10FB047
:10B81000BDE8F08F013A012A7FF670AF4FF0000AC1
:10B8200039E700297FF46AAFA8683749002205E0AC
:10B8300001320E2A01F10C0100F06B834B68984233
:10B84000F6D1697952B25846FFF7F2FB2F4A4068A9
:10B8500051680023884203F1010309D00E2B02F145
:10B8600024023FF44BAF5168884203F10103F5D144
:10B87000DBB2274A013B03EBC30302EB830393F9DB
:10B88000BC30002B7FF43AAF194BC9EBC90903EB6D
:10B890008903A36039E7BAF1010F3FF4FCAE09F167
:10B8A0000109B9F1080F05F11C057FF4DAAE2CE7A8
:10B8B000042F00F006811349AC2202FB0512D16966
:10B8C0000991002900F00A83506154210130C4B26B
:10B8D00082F8BC100B4982F8BD406A1C0A61099AC3
:10B8E000094817685179D2F808E09C46002219E00F
:10B8F000A4F80508B4180020A8710608903A0020A2
:10B9000098290020A01800209C020020A4000020FC
:10B9100000000020641B002001320E2A00F10C0000
:10B9200000F0F78243689E45F6D152B23846CDF812
:10B930002CC00A91FFF77CFBDFF8C892A44BD0E93A
:10B940000180AC22CC4602FB0532C2E90980DCF85A
:10B95000040000228045DDE90A1302F101020AD049
:10B960000E2A0CF1240C3FF452AFDCF804008045A1
:10B9700002F10102F4D1D2B29648013A02EBC202BE
:10B9800000EB820292F9BC0000287FF440AFAC20AB
:10B9900082F8BD4000FB05F4601000EBA400C0EB92
:10B9A000C0100A9400EB803084010A9804EBA004D4
:10B9B000640004EBA0044FF08C0C542082F8BC000F
:10B9C0000CFB04F204EB4400834C00EB001004EB8E
:10B9D000800004F54C7404EB420E7D4A0A9C141955
:10B9E0003268A2613322C4F88C207A4AC4F88800F5
:10B9F000062BC4E92AECD2F8442369D07748784C66
:10BA0000072B784B18BF0346774818BF20460139EB
:10BA10006F4CB2FBF0F0B2FBF3F3421EC8B2AC21A4
:10BA200001FB0541013BA1F8903092B20023A1F83F
:10BA300070200B90FA62BB627A6942F001027A616F
:10BA40003A6863F309223A603A6863F306123A608F
:10BA50003B6843F080033B603B6843F080033B60FE
:10BA60004300D9B20C93072935D8DFE811F0540010
:10BA70003400A901340014023400DA01F701079BF5
:10BA8000103302FA03F30B43BB6476B1574B3268B1
:10BA900093F8581BB388490141F005011B0401F0DC
:10BAA000E50193613046FEF71DFC786FA1B20022DC
:10BAB000FCF7C2FA9DE6079B0121002B7FF404AE40
:10BAC0001CE64A4A032382F8C7330FB0BDE8F08F63
:10BAD000474B48489BE73B6823F001033B60012448
:10BAE00000230493029300930622234638460394CE
:10BAF00001940D914FF0E0FF0D99224638464AF02F
:10BB00002FF90D990439032920D8DFE811F0DC0161
:10BB10001F00A201BF013B6823F001033B6000212D
:10BB200001240A237B6306222346CDE90341CDE9A4
:10BB30000141009138464FF0BFFF224600213846B0
:10BB40004AF00EF9BB6943F00803BB61099B187901
:10BB5000002840F056813B6843F001033B6000231E
:10BB6000D9F80420904503F1010300F0B3810E2BB6
:10BB700009F12409F4D100234FF0FF340993154A49
:10BB80001D4804EBC40302EB83034FEAC409D3F856
:10BB9000A480804514BF382036204FF0F3F9D8F840
:10BBA000002142F00102C8F800210B9B032B00F298
:10BBB0008F81124B0C9A1344B3F8AC13044A10480B
:10BBC000AC2303FB05234FF0000C1984634622E0ED
:10BBD000A018002000000020583E002044950800D6
:10BBE000D0DD06001055220040771B00903A00205F
:10BBF000882A1100A0BB0D0000640240D8F505089A
:10BC0000A8390020A4000020974200F06E81013383
:10BC1000042B00F07B8150F83320002AF4D1B64A7F
:10BC20009C46134652F8EC2C013243F8EC2C03EB03
:10BC3000CC024FEACC0342F8E87C03440A9FAF4AA7
:10BC4000099817449A88114399809022AC493B4641
:10BC5000FFF76EF9AB4BAC49A14403EB8903AC226F
:10BC600002FB0512D3F8C430916A186861F306002C
:10BC70001860536A196841F0020119604FF480742A
:10BC80004FF440781021A7F86C40A7F87080A7F80F
:10BC90006810B2F88CE0A7F86AE09069022100F120
:10BCA000180C87F86E10C7F860C0D2F8885087F873
:10BCB0006F101030099018687D664BF6EF7900EA36
:10BCC00009001860186840F010001860186840F407
:10BCD00040501860186861F38B201860186861F391
:10BCE00009201860196841F080011960196821F075
:10BCF00040011960196821F02001196059686EF33C
:10BD00000F015960C3F808C0DD601968F96159680E
:10BD10003962996879620020D968B962A7F88C40C5
:10BD2000A7F89080A7F888000999B2F8AC40C7F846
:10BD30008010012187F88E10A7F88A40D2F8A85009
:10BD400087F88F101A68C7F8845002EA09021A604F
:10BD50001A681A601A6842F440521A601A6861F34D
:10BD60008B221A601A6861F309221A601A6842F07D
:10BD700080021A601A6860F386121A601A6860F30B
:10BD800045121A605A6864F30F025A600999996063
:10BD9000DD601A68FA625A683A639A687A63DA6808
:10BDA000BA631A6842F002021A60089B8BF81030DE
:10BDB000079BCBF80430CBF80C60CBF81870E8E4A4
:10BDC0003B6823F001033B60012400230A22BA638D
:10BDD0000221CDE90343CDE9003402930622234634
:10BDE00038464FF069FE38462246022149F0B8FF36
:10BDF000BB6943F40063BB61099B187900283FF4D9
:10BE0000AAAEFEF7DFFA099B0446DA790A21FFF7AA
:10BE1000B3F90CB15423E3807B6C43F400437B649F
:10BE200099E60A233B643B6823F001033B6001244D
:10BE3000002306221146049302930093384603948C
:10BE4000019423464FF038FE22460621384649F039
:10BE500087FFFB6943F40063FB6177E60A237B6796
:10BE60003B6823F001033B60012400230493029309
:10BE700000930622072138460394019423464FF08D
:10BE80001BFE22460721384649F06AFF3B6F43F00C
:10BE900008033B675AE60A23FB633B6823F0010370
:10BEA0003B600124002304930293009306220421A3
:10BEB00038460394019423464FF0FEFD22460421A8
:10BEC000384649F04DFFFB6943F00803FB613DE64E
:10BED000002173E6DBB209935C1E50E6064A02239A
:10BEE00082F8C7330FB0BDE8F08FDB00A5E64FF056
:10BEF000FF320792104631E4903A0020B418002037
:10BF00008180000800000020A018002000239B88EA
:10BF1000FFDE00235B68FFDE70B590F87A301C0905
:10BF2000013C072C0FD8194E06EB44020546B2F827
:10BF30004C0103F00F0340FA03F2D20703D595F842
:10BF40007D20012A01D0012070BD9A40013A1040A5
:10BF5000264453F099F996F85C310D4A034402EBFC
:10BF6000C30452F83320A38810691840ECD0002392
:10BF700095F87B2085F87D300A212046FFF7FCF8F4
:10BF8000AA6ED36843F00803D360DCE7D8F5050850
:10BF9000D439002038B505461446FEF7A3F9AB881E
:10BFA0002A68B3FA83F3C3F11F0303F00701890082
:10BFB00013F0F80F04FA01F40AD0536A0F2000FAC4
:10BFC00001F123EA01035362536A1C43546238BDF2
:10BFD000136A0F2000FA01F123EA01031362136AC6
:10BFE0001C43146238BD00BFF8B50D4B93F8D072F6
:10BFF00097B10C4DC7F109070924013C0ED0AE687A
:10C000003079FEF7DFF9297DF27908B1FFF7C2FF39
:10C01000A74205F14C05F0D10120F8BDA368FFDE71
:10C0200098290020641C00202DE9F04FDFF89CA225
:10C030009AF859BB8BB0BBF1000F03D100200BB0B5
:10C04000BDE8F08F00222F21584611F085FE0746EB
:10C050000028F3D00568CAF85C5BFFF715F8804646
:10C060000028EBD04468CAF8604B002CE6D08F4E15
:10C070000023324601E00E2BE0D051688C4202F1E1
:10C08000240203F10103F6D1DBB2DFF84492013B55
:10C0900003EBC30309EB830393F9BC20002ACDD142
:10C0A00058464FF02F0BA3F8BCB0FEF78BF9CAF837
:10C0B000640B08B1A0F806B0FA790A21FFF75CF822
:10C0C0007B4A002302F56D7151F83320954200F050
:10C0D000D58101330F2BF7D100204EF053FF2B6891
:10C0E000744A23F001032B60D9F844339342C0F023
:10C0F000B58103F1B772704902F55852A1FB0221D4
:10C10000890D013989B24A1C0139B3FBF2F36B4A3C
:10C110006B481B0AA2FB03321309A0FB03035B0855
:10C120001209AAF86A3B013A5B00EA62AAF8683B86
:10C13000A9626B6943F001036B612B6823F44073C0
:10C140002B602B6823F070032B6097F806A00AF091
:10C1500001021AF0020A40F084811046D646524687
:10C1600001237979089101F1FF3B5FFA8BFB4FEADC
:10C170004B010991C9B20791072909D8DFE811F0ED
:10C18000550108003C010800230108000A012200B3
:10C19000CDE901020022039300920799CDF810E047
:10C1A000062228464FF088FC2B6843F080032B6062
:10C1B000079B043B032B1DD8DFE813F019011C007B
:10C1C000000118004FF0000CC5F874C00721CDE93C
:10C1D00001020393CDF810E0CDF800C006222846F6
:10C1E0004FF06AFC2B6843F080032B602B6F43F009
:10C1F00008032B67BBF1030F00F23E81099B2C4A19
:10C200001344B3F8AC33EA681343EB60BAF1000FA0
:10C2100000F02C81089B59000139C9B2012228463F
:10C2200049F09EFD3246002351688C4202F12402FF
:10C2300003F1010300F02D810E2BF5D14FF0FF33F8
:10C2400003EBC30309EB83031E48D3F8A4A0824584
:10C2500014BF382036204EF095FEDAF8002142F067
:10C260000102CAF800210023324651688C4202F1D3
:10C27000240203F1010300F007810E2BF5D1002009
:10C28000114900236022FEF753FE236823F00103C7
:10C290002360204648F0A0FE7B79013B032B00F28F
:10C2A000FB80DFE803F074716E1700BFA40000206C
:10C2B000D8F50508006CDC02819F5E16598B4F0192
:10C2C000ABAAAAAA0064024005830008903A0020A5
:10C2D0000000002005F1400223684BF6EF710B408F
:10C2E0002360236843F0100323602368012161F376
:10C2F0000D3323602368022161F38B2323602368BD
:10C3000061F309232360236843F0800323602368DB
:10C3100023F040032360236823F020032360636835
:10C3200040F62A0161F30F0363605E4BA260E36095
:10C3300000237268944206F1240603F1010300F021
:10C34000A5800E2BF5D14FF0FF3303EBC30309EBB0
:10C350008309D8F80810D9F8C4301A6861F30602C6
:10C360001A60236843F0020323602368012003431B
:10C3700023606B6C43F400436B642B6803432B60B6
:10C380005DE605F13C02A7E705F13802A4E705F1F7
:10C390003402A1E74FF0000CC5F840C0CDE901021E
:10C3A00006220393CDF810E0CDF800C011462846D0
:10C3B0004FF082FB2B6843F080032B60EB6943F462
:10C3C0000063EB6116E74FF0000CC5F83CC0042198
:10C3D000CDE901020393CDF810E0CDF800C00622AC
:10C3E00028464FF069FB2B6843F080032B60EB6914
:10C3F00043F00803EB61FDE64FF0000CC5F838C0D0
:10C400000221CDE901020393CDF810E0CDF800C080
:10C41000062228464FF050FB2B6843F080032B6028
:10C42000AB6943F40063AB61E4E64FF0000CC5F880
:10C4300034C06146CDE901020393CDF810E0CDF898
:10C4400000C0062228464FF037FB2B6843F08003DC
:10C450002B60AB6943F00803AB61CBE64FF0FF31D3
:10C4600055E600204FF0010E03467AE607990122B7
:10C47000284649F075FCD5E60023C4E60A4A02EBDB
:10C48000C30393F8B80328E6D8B2F9E6DBB2013B60
:10C490005BE7DBB2013BD3E605F1340202EB83023A
:10C4A0001AE700BFFC840020D8F5050810B40C4939
:10C4B000D1F8603B1A6822F001021A60D1F85C2BB7
:10C4C00040F62A0400205C605062116841F00101CE
:10C4D00011601A6842F001021A605DF8044B70475F
:10C4E000903A002030B40B4A0B4B82B0CA2553243B
:10C4F00002EB800200205D625C62019001925D624D
:10C500005C620198FF2201605A625A6202B030BC3C
:10C51000704700BF5028004000280040F0B50E468C
:10C5200064493468D1F84413B1FBF2F1013B9BB28A
:10C53000013987B0E362A1626369BDF830C09DF83C
:10C54000342043F001036361236823F440732360C4
:10C55000236823F0700323607579B37907460AB125
:10C5600083F0010313F0020203F001010DD108462C
:10C5700001231146013D6D00EDB2072D09D8DFE81A
:10C5800005F01A084B085D086F8100200122034660
:10C59000F0E704920022CDE90101009229460393BD
:10C5A00006222046043D4FF087FA032D13D8DFE81A
:10C5B00005F052126476C4F834C0CDE902130021AC
:10C5C000049201900091062220464FF075FAA3696B
:10C5D00043F00803A361636C43F40043636423687E
:10C5E00043F0010323607379013B032B5CD8DFE840
:10C5F00003F0100D0A0204F140030022C7E90034E1
:10C600001A6007B0F0BD04F13C03F6E704F138030B
:10C61000F3E704F13403F0E7C4F838C004920022D1
:10C62000CDE90213019000920221062220464FF02C
:10C6300043FAA36943F40063A361CCE7C4F83CC0A8
:10C6400004920022CDE902130190009204210622F7
:10C6500020464FF031FAE36943F00803E361BAE79B
:10C66000C4F840C00492002200920622CDE90213D1
:10C670000190114620464FF01FFAE36943F400632E
:10C68000E361A8E7C4F874C004920022CDE9021364
:10C69000019000920721062220464FF00DFA236FE9
:10C6A00043F00803236796E704F1340202EB8303A7
:10C6B000A3E700BF000000202DE9F0478368046C69
:10C6C00093F8059093F806801E68054686B02046CC
:10C6D00048F082FC09F1FF3A002385F82C305FFA1C
:10C6E0008AF35F00FFB208F00208072F0DD8DFE8D9
:10C6F00017F0F9000C0002010C000B010C000800FF
:10C700001401F26922F40062F261B8F1000F14D052
:10C71000022B28D84FEA490909F1FF395FFA89F855
:10C7200000224146304649F01BFBBAF1030F00F2EC
:10C730000381DFE80AF0A59E951DA9F10203022BF3
:10C74000EED84FEA49010239424601F0FE01304677
:10C75000A9F1030949F004FBB9F1010F00F2878048
:10C76000DFE809F07C044FF00008D9E74FF0060835
:10C77000F36923F44073F3614FF0060995F83B30F9
:10C78000049395F83A30039395F83930029395F86D
:10C790003830019395F83730009395F8363095F896
:10C7A0003520394630464FF087F9B9F1040F00F0D3
:10C7B000BD80B9F1060F00F0BC800023B363414691
:10C7C0000122304649F0CCFA072F09D8DFE807F0FC
:10C7D000850880087B080476F36943F40063F361FD
:10C7E00023684BF6EF7110220B402A8423602368E4
:10C7F00013432360236895F8292062F30D332360E7
:10C80000236895F8272062F38B232360236895F82B
:10C81000262062F309232360236895F8252062F31C
:10C82000C7132360236895F8242062F386132360DE
:10C83000236895F8282062F34513236063686A8CA7
:10C8400062F30F036360D5E90623A260E360236807
:10C8500043F00203236006B0BDE8F0874FF0040800
:10C86000F36923F00303F3614FF0040986E74FF007
:10C870000208B36923F44073B3614FF002097DE706
:10C88000B36923F00303B36195F83B30049395F843
:10C890003A30039395F83930029395F83830019384
:10C8A00095F83730009395F8363095F8352000210B
:10C8B00030464FF001F90023736380E7336F43F094
:10C8C000080333678CE7F36943F00803F36187E7F4
:10C8D000B36943F40063B36182E7B36943F00803CB
:10C8E000B3617DE7B26922F00802B261B8F1000FCE
:10C8F0003FF423AF0CE7B26922F40062B261B8F1F1
:10C90000000F3FF41AAF03E7F26922F00802F26168
:10C91000B8F1000F3FF411AFFAE6326F22F00802CF
:10C920003267B8F1000F3FF408AFF1E60023F3637C
:10C9300045E70023336442E795F83B30049395F8CC
:10C940003A30039395F83930029395F838300193D3
:10C9500095F83730009395F8363095F835203946FC
:10C9600030464FF0A9F8A6E72DE9F04FA94D2B7BF3
:10C9700087B01BB9012007B0BDE8F08FA64E2C6828
:10C98000FCF756FE96F8D0120491002900F037818A
:10C99000A24BA34FA3FB04235B09A7FB0327FF08BC
:10C9A00007EB8707A3EB47079E4B53F8C03C05F501
:10C9B000717406F61C48A0EB030BFBB206F6FC698B
:10C9C000039308EB870700268A460594019410E03C
:10C9D000019C2046FFF770FE013623464C33564536
:10C9E000019308F15C0807F15C0709F1140900F0F4
:10C9F000BB80BBF1000F04DB019B1B6B5B4500F3AD
:10CA0000EA80844A4C2303FB062393F8F033002B7F
:10CA1000DED00198836881891A68036C5C68D368EA
:10CA2000A4B2C4F1160423EA0103072CD360CFD9C2
:10CA3000794A856CD2F8043F02960133C2F8043F6C
:10CA400000222868AE469446012115E0BCF1140F7F
:10CA50001EDC13F1080648BF03F1170633110CEB77
:10CA6000261C5E1E02FA03F30122114402FA06F6A6
:10CA70008C4246EA03020BD303465EF8040FA14240
:10CA8000A0EB0303E2D3CCF115034FF0150CE8E75C
:10CA9000BCF1150F029E5DD1634CC2F3842304EBFD
:10CAA000830302F01F00D3F82C14C2F3441304EBE9
:10CAB000830304EB8000D3F82C34C2F3C4320902A0
:10CAC00004EB820241EA0311D0F82C34D2F82C2472
:10CAD0000B4343EA023383EA132282EA121202F082
:10CAE0000F020F2A36D1C3F30F134FF6FF72934292
:10CAF00030D0B3F5606F72D0A9F80C3098F8582098
:10CB00000398824210D0B968D8F80020521AC8F8A9
:10CB10000020396BD8F80420521AC8F804200022EB
:10CB2000BA603A6388F85800D8F800200132C8F893
:10CB30000020BA680132BA604FF6FF7293427FF468
:10CB400047AFD8F804300133C8F804303B6B0133E9
:10CB50003B633DE7304AD2F8003F0133C2F8003F63
:10CB60009EB34FF6FF73C9E7304B059C049F01222B
:10CB70001A702C4B002643F8C06C03250FE05B00B5
:10CB8000BCF1020F03F1FF331DD900210122013650
:10CB900049F0E6F8B74204F14C043FF4EBAEA36869
:10CBA0001868426865F306124260217C5B7911F0D7
:10CBB000020103F1FF3CA3F10202E0D15B00022A73
:10CBC000A3F10203E2D8D9B2E0E729465822184877
:10CBD00052F06EFAC5E7002007B0BDE8F08F0D49AE
:10CBE00091F8252602EB420201EBC202324492F890
:10CBF00035260D2A80D1802289F81E207EE7064B3B
:10CC0000084A03F5805301211970049B42F8C03C87
:10CC1000B0E600BFA0180020982900201F85EB5126
:10CC2000CDCCCCCC903A0020D8F50508983900201E
:10CC3000403900202DE9F047884600294AD046189F
:10CC4000DFF89890DFF898A0451E013E8024EFF3AE
:10CC5000118184F31288D9F8C432D9F8C802D9F8FE
:10CC6000C422D9F8C8C2C9B281F31188624512E062
:10CC70000120FDF75FF9EFF3118184F31288D9F8F1
:10CC8000C432D9F8C802D9F8C422D9F8C872C9B2D6
:10CC900081F31188BA428CBF002201221B1A03EBD8
:10CCA000C223012BE4D0EFF3118284F31288D9F868
:10CCB000C83215F8011F5344D2B283F86C1BD9F85F
:10CCC000C8320133C3F30A03C9F8C83282F31188AA
:10CCD000B542BCD14046BDE8F08700BF982900208E
:10CCE000903A0020F8B50C4E96F8C83C032B00D0C3
:10CCF000F8BD37680D46144608E0FFF79BFF336820
:10CD0000DB1B322BA4EB00040544F1D8002C214698
:10CD10002846F2DCF8BD00BFA0180020344BD3F841
:10CD2000E839596A91F85230012B56D170B5314C1F
:10CD3000314AD4F8740260BBD2F8C402D2F8C832C7
:10CD4000984221D0D2F8C402D2F8C832984249D8C9
:10CD5000D2F8C832D2F8C4021B1AD2F8C42291F811
:10CD6000520088B1B3F5007F28BF4FF400731D4611
:10CD7000002381F85230214921480A44ABB2812175
:10CD800049F0F2F8C4F874521E4B6FF001021A61B8
:10CD900070BDD2F8C45200F03F032844C2F8C40268
:10CDA000D2F8C402B0F5006F04BF0020C2F8C4027C
:10CDB0000020C4F87402002BBED1D2F8C42291F82E
:10CDC00052000028E4D00D4881F852300244BDE8FA
:10CDD00070400B48812149F0C7B80A4B6FF001023F
:10CDE0001A617047D2F8C432C3F50063B5E700BFDB
:10CDF000A0180020884B002098290020FC45002026
:10CE000084220020004C01402DE9F04FA94DD5F8B7
:10CE1000E089D8F81460D8F81820D8F81430DB0767
:10CE200085B026D41640B70744BF0223C8F8143093
:10CE3000740300F19880300300F12A81F20400F1BC
:10CE40005F81310708D5D5F8E839DB690BB19A481D
:10CE500098470823C8F81430B2040DD4F30640D420
:10CE6000F70257D4B40262D4002EC0F2BB81300561
:10CE70006BD405B0BDE8F08FD5F8E4498F49D4F8FC
:10CE800000396FF30A03C4F80039D4F8043823F4E6
:10CE90008073C4F80438E368052262F38D23E360ED
:10CEA0004FF0400901272046C5F8589BA5F8527B52
:10CEB00048F082FF00238249A5F8F2392046C5F8E0
:10CEC000F89948F079FFD5F8E83985F8C87C5B68AF
:10CED0000BB1794898474FF40053C8F81430F30663
:10CEE000BED5D5F8E4399A6922F010029A611A6A1F
:10CEF000C2F343410229C2F30A1702F00F0200F005
:10CF00004582062900F0CA839A69F70242F01002AE
:10CF10009A61A7D5D5F8E8391B6A13B1664805218F
:10CF200098474FF48013B402C8F814309CD5D5F854
:10CF3000E8391B6A13B16048062198474FF4001383
:10CF4000002EC8F8143092DA4CE1D5F8E439D3F861
:10CF50000828D10700F13E824FF40063C8F814306E
:10CF600005B0BDE8F08FD5F8E439D3F81878D3F8D8
:10CF70001C281740BFB203F50061002F3FF45BAFE0
:10CF80004FF0000ACDE901864E4C03F5106B564672
:10CF9000884608E07F0806F1010604F12C040BF135
:10CFA000200B00F04081F907F4D5D8F81020D8F80C
:10CFB000343023FA06F94FEAC919DBF808305FFA72
:10CFC00089F949EA020909EA030919F0010F40F059
:10CFD0003E8119F0080F1CBF0823CBF8083019F068
:10CFE000100F1CBF1023CBF8083019F0400F1CBFE6
:10CFF0004023CBF8083019F0020F1CBF0223CBF8F6
:10D00000083019F0800FC5D0D5F8E499A26AE36A18
:10D01000A16909F5106A0AEB461AA2EB030E8E45C8
:10D02000DAF8180028BF8E4680B20EF10301B0EB8B
:10D03000910F40F2FF8009F5805C0CEB063C0396F3
:10D0400011468B4280F0F580A269C91A914228BF2F
:10D05000114688B20330CE1C8010626A8E464FEAB9
:10D06000960609D00023013352F8041BCCF80010B7
:10D070009842F8D1626AE36A72446262DAF8182070
:10D0800092B273449642E36280F0D380A16AD8E7FB
:10D09000D5F8E479D7F81848D7F81C381C40240C88
:10D0A00007F5006C3FF4CAAE07F530674FF0000992
:10D0B000E34610E0A018002084220020F023002086
:10D0C0009022002080220020640809F1010907F164
:10D0D00020073FF4B3AEE307F6D5BA68DBF81430A7
:10D0E00002EA030A1AF0010F40F011811AF0080F4A
:10D0F00040F0D5801AF0100F1CBF1023BB60E3E78F
:10D10000D5F8E449D4F8043823F00103C4F804380E
:10D110004CF03CFB2269C14B102161F38A12226161
:10D12000226942F0200204F50067226101E0013B20
:10D1300002D022699006FAD404F5106304F5206148
:10D14000FF229A60C3F8082220338B42F9D14FF0B6
:10D15000FF33BB614FF00113FB617B6943F00103B7
:10D160007B617B6943F002037B617B6943F00803C9
:10D170007B613B6943F001033B613B6943F0020380
:10D180003B613B6943F008033B61D4F8003823F46A
:10D19000FE63C4F800380023C4F8103BD4F8103BF9
:10D1A000012161F3DC43C4F8103BD4F8103B182292
:10D1B00062F31203C4F8103BD4F8103B43F0C043B1
:10D1C000C4F8103BD5F8E83985F8C81C1B6A0BB1C8
:10D1D000934898474FF480533107C8F814307FF5CF
:10D1E0003BAE30E6D5F8E439D3F8042822F001024A
:10D1F000C3F80428D3F8002E22F00102C3F8002E51
:10D2000095F8C92CD5F8E83985F8C82C1B6A13B1F4
:10D210008348032198474FF000433005C8F8143085
:10D220007FF527AE91E6DDE9018630037FF506AE96
:10D230002EE7039EBEF1000F7FF4ACAED9F8343870
:10D240000122B24023EA0203C9F83438A2E6D8F832
:10D250003430012202FA06F123EA0103C8F834301F
:10D26000CBF80820002E72D195F8C43C022B7FF435
:10D27000B0AED5F8141AD5F8F839994240F2508278
:10D28000C91A8B42C5F8141A88BF8BB2D5F8042A84
:10D29000634898BF9BB2002148F066FE99E60823D8
:10D2A000BB60B5F8B82CB5F8BE3CD5F8BA1CA5F8EB
:10D2B000B02C02F01F0C0120BCF1010F85F8C40C4A
:10D2C000A5F8B63CB5F8BC0CA5F8C63CC5F8B21C30
:10D2D0005FFA82FE00F0C481BCF1020FC2F30722A4
:10D2E00000F07B81BCF1000F00F0898095F8CA3C0A
:10D2F000002B3FF4FFAED5F8E429D2F80018002047
:10D3000063F30A11C2F8001885F8CA0CF2E601238B
:10D31000BB60B9F1000F29D195F8C43C032B7FF411
:10D32000E5AED5F8741BD5F8583B994240F2CF8151
:10D33000C91A8B42C5F8741B88BF8BB2D5F8642B11
:10D34000374898BF9BB2002148F0FCFECEE6D5F8E6
:10D35000E8395B69002B3FF43CAE95F8C82C032AF2
:10D360007FF437AEF1B22E48984732E6D5F8E83967
:10D370009B69002B3FF4BAAE95F8C82C032A7FF4C2
:10D38000B5AE5FFA89F126489847AFE6002F3FF423
:10D39000BBAD2C2101FB025107F1030CD1F8649BBA
:10D3A0004FEAAC0C03F5805E484600210131DEF8FF
:10D3B000004040F8044B6145F8D12C2101FB02529A
:10D3C00009EB0700D2F86C1BC2F8640B3944C2F8B1
:10D3D0006C1B99E595F8C82C85F8C92C042285F8B2
:10D3E000C82CD3F80828D2071CD4D5F8E8391B6A12
:10D3F000002B3FF4B1AD022109489847ACE51EF07F
:10D40000600F40F0778189B2092A12D8DFE802F074
:10D410005D3B11BC11D29211791500BF420D030082
:10D4200084220020D3F8002E42F00102C3F8002E1F
:10D43000DBE7B44848F05AFD58E7CAB2B2490343A3
:10D4400081F878220193F4D195F8C83C022B00F0C2
:10D45000F481032BEDD1002A40F0D881D5F8E839CA
:10D4600085F8CD2C022185F8C81C5B68A54801927F
:10D470009847019AA348042385F8C43C11461346F3
:10D4800048F072FD32E795F8C83C023B012BD0D83A
:10D4900001297FF42BAFD5F8D03CD5F8E8299B497A
:10D4A00023F00203C5F8D03C002385F8CB3C9268FA
:10D4B000A1F533709047042285F8C42C00239148CD
:10D4C0001A46194648F050FD10E795F8C83C023B53
:10D4D000012BAED895F8CB3C2BB1D5F8D03C43F01E
:10D4E0000203C5F8D03C8A4A02230021A2F53B7012
:10D4F000C5F8183AC5F8143A85F8C43C48F034FD2C
:10D50000F4E6012B95D195F8C82C022A00F0C981C8
:10D51000032A8ED17F4AC5F8183A02216FF43A7C6B
:10D5200085F8C41C02EB0C000021C5F8143A48F041
:10D530001BFDDBE60B0A022B00F0E281032B00F05F
:10D54000D681012B7FF475AFD5F8EC391B6898476D
:10D5500000283FF4CBAE0388002B3FF4C7AEB5F8EC
:10D56000B61C00293FF4C2AE8B4228BF0B460221F5
:10D57000426885F8C41C6348C5F8183A0021C5F80C
:10D58000143A48F0F1FCB1E601297FF4AFAE85F81A
:10D59000CB1CD5F8E8395D499B68A1F533709847F5
:10D5A0000023042285F8C42C56481A46194648F030
:10D5B000DBFC9BE603437FF43CAF95F8C82C032AC1
:10D5C00001F07F013FF435AF00290CBF0122022298
:10D5D00085F8CA1C85F8C82CE3E70EF0600E0B0C2A
:10D5E000BEF1200F0193C1F307430AD1D5F8E82912
:10D5F000464992680293A1F53370904795F8B12C93
:10D60000029B012A00F0CC80032A00F0AC80002AA3
:10D610007FF40FAF95F8C82C022A00F09C80032AF3
:10D620007FF407AF019A100600F1E8803A4A2C21F6
:10D6300001FB032202F5B872537B3248A3F10103C8
:10D64000B3FA83F35B0942F8103F00210223C5F8C7
:10D65000183AC5F8143A85F8C43C48F085FC45E60C
:10D6600095F8C83C032B7FF4E4AE264BD5F8E829A7
:10D670000193926803F5337118469047B5F8B62CBC
:10D68000019B002A7FF432AE18460422002385F85D
:10D69000C42C19461A4648F067FC27E607F1030C2C
:10D6A0005FEAAC0C0AD01D4803F5805E0021013111
:10D6B000DEF8004040F8044B8C45F8D12C2101FBEA
:10D6C0000252D2F86C1B3944C2F86C1B1CE4D5F82A
:10D6D000E8391A690B4B1AB1184601939047019B20
:10D6E00018460422002385F8C42C19461A4648F02F
:10D6F0003BFCFBE4D5F8E83904499B68A1F533709D
:10D700009847F3E584220020884B00205025002014
:10D71000702500206D250020802200205825002043
:10D72000D5F8102A93424CD0D5F8E839DB68002BA5
:10D730005FD095F8C82CDFF810A2032A01D150461B
:10D7400098470023052285F8C42C50461A461946EE
:10D7500048F0F8FC3DE459063FF4C8AD7A48194654
:10D7600048F094FBC2E595F8C82C022AF3D0032AAE
:10D770007FF45FAEB5F8B22C002A3DD15A063BD0FB
:10D780001946714B0193184648F080FB019BD5F870
:10D79000E8290193184692686C499047019B73E70A
:10D7A00095F8C82C022AD6D0032A7FF442AEB5F8E9
:10D7B000B22C002A7FF49AAD13F07F0047D1624B60
:10D7C00062E7D5F8182A9342AED8B5F8C63C9A421B
:10D7D000AAD23346324631465B48C5F8106A48F053
:10D7E000C3FB594833463246314648F0ABFCFFF79D
:10D7F000F0BBDFF854A1A4E7534BC8E7544A03F049
:10D800007F032C2101FB0322103215E795F8CD3C54
:10D810009342D4D1D5F8E8394B485B6898474D49D5
:10D8200091F8783285F8CD3CD5F8E8391B68464840
:10D830009847042385F8C43C40E6002ABFD085F809
:10D84000CD2C0322D5F8E83985F8C82CEEE70199EC
:10D85000D5F8E42911F0800F3D4943D12C2000FB7D
:10D86000031101F5B871887850BB02F510630A788E
:10D8700003EB4213CA78D3F800C0023A60F3555C58
:10D88000012AC3F800C028D92F4BD5F8E829019305
:10D8900000204873926803F5337118469047019B46
:10D8A000F2E685F8C42C2C4AC5F8183A0021A2F5F6
:10D8B0003A70C5F8143A85F8CC1C48F055FB15E5CC
:10D8C00002F530630A7803EB42131A6822F400125F
:10D8D0001A60CA78023A012AD6D81A6842F08052F1
:10D8E0001A60D1E72C2303FB00111031BBE7C9B24A
:10D8F00005293FF6FFAEDFE801F0211C17120D08E5
:10D90000D5F8EC399B68984722E6D5F8EC391B6AC4
:10D9100098471DE6D5F8EC395B6A984718E6D5F8C4
:10D92000EC39DB69984713E6D5F8EC399B699847E1
:10D930000EE6D5F8EC395B69984709E6D5F8EC397D
:10D940001B69984704E600BF842200205025002070
:10D9500080220020884B00206C25002070B51B2001
:10D96000FCF730FD08B12923C3801C20FCF72AFDF9
:10D9700008B12923C380FBF751F92D482D4E2E4CB9
:10D9800047F01CFB4CF022F800220221432047F014
:10D99000E9FD49F0EDF8294901F580534FF0A04029
:10D9A0000122C1F8E00983F8A42383F8B123826B34
:10D9B00042F400128263224AC3F8A8234FF4817212
:10D9C000A3F8AC234FF401620025A3F8A62306F5C3
:10D9D0005C7106F5527283F8AF534DF09FFDD6F897
:10D9E0004433184AA2FB03239B090421013BE16253
:10D9F000A362636943F001036361236865F309234C
:10DA00002360236865F306132360236843F08003D3
:10DA10002360E36843F00103E3602A4602216920A2
:10DA200047F0A0FD236843F00103236070BD00BFF1
:10DA30000700340000000020004C0140A018002026
:10DA400040004001D34D6210BFF34F8F0549064B94
:10DA5000CA6802F4E0621343CB60BFF34F8F00BF8C
:10DA6000FDE700BF00ED00E00400FA0508B572B65E
:10DA7000FFF7EAFFF0B5AA4BB3F5C07F85B000F021
:10DA8000A78100F23381B3F5807F00F0A781B3F561
:10DA9000A07F00F0A181802B14BF05240624A14B98
:10DAA0001B8A03F00703A34240F09A819E4847F087
:10DAB00085FA9E499E4B0A689E4842F480720A602D
:10DAC000FF24CA2153225C6259625A62D0F874382A
:10DAD000DB0000F11481984A954B984FCA255324D6
:10DAE0000020FF215D625C62029002925D625C62D6
:10DAF000029E0432BA42306059625962F2D19049B2
:10DB00000020FEF7EFFC8F4B002103910393039B52
:10DB10001B680093009B012B00F02E81824847F088
:10DB20004DFA824A884B1169012060F302011161AC
:10DB3000196E02F5E43260F30101196613680343BC
:10DB4000136013689F07FCD59368804923F0030393
:10DB500093608B6813F00C0FC3F38102F9D10B684B
:10DB60007B4C23F0867323F480334FF41F000B604B
:10DB70008A604C60C1F8A020C8600B686D4A43F40D
:10DB800080330B60D2F800389E0307D44FF4405323
:10DB9000D2F800188D0301D4013BF9D1D2F8003836
:10DBA0009C03EFD56949634A0B6843F001030B609E
:10DBB000D2F800389807FBD5644B5A6842F48002CB
:10DBC0005A605A68482161F38E125A605968594A5E
:10DBD000012060F303015960596860F312415960F4
:10DBE000196841F080711960D2F800389901FBD5AD
:10DBF000564A936823F0F00393609368042161F31D
:10DC00004F339360936861F38C239360D2F8A43010
:10DC100043F03003C2F8A4309368022060F301039C
:10DC200093609368C3F38103022BFAD1D2F8A43036
:10DC300023F03003C2F8A430D2F8A4300B2161F3F2
:10DC40000F33C2F8A430D2F8A03023F40053C2F846
:10DC5000A030936813F00C0FC3F3810100F096809D
:10DC6000022900F0A1803B4A38493B488B683B4C75
:10DC70003B4DC3F303131844E36890F8AC04C2406F
:10DC80004FF6FF00034043F0052343F47A03E360BB
:10DC9000344B486FC3F87C022648334BA360D0F85E
:10DCA000343823F00043C0F834384B6F2F4843F02A
:10DCB00080734B67C5F8442347F080F9FAF780FF7B
:10DCC0002B4AD5F84433A2FB03239B09013BB3F154
:10DCD000807F09D24FF0E022F0205361002107231A
:10DCE00084F823009161136105B0F0BDB3F5E07FC6
:10DCF00070D0B3F5007F14BF05240024CFE61D4B80
:10DD0000002201920193019A03F11973126803F53D
:10DD10009E3303F2E1139A427FF4DDAEF3E600BFD7
:10DD2000C000000000C0FF1F1C0040000070004049
:10DD30000028004000300240542800406C28004079
:10DD4000316665425C280040003C024000380240D9
:10DD50000230030000127A00D8F5050800ED00E05B
:10DD600000000020884B0020000000081F00300049
:10DD7000D34D6210502800400320FEF7B3FB3F4B09
:10DD80001A6882F308885B689847FEE7D2F8A030EB
:10DD90005B047FF568AFD2F8A010394B394A11F413
:10DDA000805F08BF1A465FE7536853685168506840
:10DDB000354D334CC0F30240C3F388122B5C01F0A5
:10DDC0000F0104FB02F213FB01F3B2FBF3F24BE78A
:10DDD000022464E6012462E6032460E604245EE68D
:10DDE0002A4D2B4A2B4B6A606B606A646B64E9694D
:10DDF000AA6011F0020F14BF0026A526AB602B69A4
:10DE00009905FCD52B6943F020032B612B6943F066
:10DE100040032B614FF0004047F04CFB2B69032877
:10DE200023F020032B6117D0184D194A194BAA6013
:10DE3000AB602B699A05FCD52B69174A43F0100398
:10DE40002B614FF48010148247F034FB2B6923F0D0
:10DE500010032B61FFF70AFEA52EE5D12B690E4AB0
:10DE600043F010032B614FF48010168047F022FB23
:10DE70002B6923F010032B61D6E700BF0000FF1FC2
:10DE800000127A00006CDC02A0710608003C02401F
:10DE900023016745AB89EFCD00C0FF1F0149024850
:10DEA000FAF766BFEC1F00200000014002494FF066
:10DEB0008040FAF75DBF00BF1820002001490248EA
:10DEC000FAF756BF442000200004004001490248F0
:10DED000FAF74EBF702000200008004001490248B8
:10DEE000FAF746BF9C200020000C00400149024880
:10DEF000FAF73EBFC8200020001000400149024848
:10DF0000FAF736BFF420002000140040014902480F
:10DF1000FAF72EBF202100200004014001490248E9
:10DF2000FAF726BF4C2100200040014010B5064CF6
:10DF3000064804F24C71FAF71BFF04F6D8010448B6
:10DF4000BDE81040FAF714BFA018002000000140FF
:10DF50000044014001490248FAF70ABFA421002009
:10DF60000048014001490248FAF702BFD0210020D1
:10DF70000018004001490248FAF7FABEFC210020CF
:10DF8000001C004001490248FAF7F2BE2822002096
:10DF90000020004001490248FAF7EABE542200205E
:10DFA000004C01402DE9F0411348144D4FF4257207
:10DFB000002151F0D5F84FF00008A5F2BC47A5F5B7
:10DFC000847440F2FB2655F82810002354F83320BF
:10DFD00091420BD001330F2BF8D1002008F1070834
:10DFE0004CF0D0FFB045EED1BDE8F08107EBC303A4
:10DFF00093F8B803F2E700BFEC1F002094FA05087D
:10E00000EFF31183502282F31288026822F001029A
:10E01000DBB2026083F31188704700BF38B548F067
:10E02000A7FD1B20FCF7CEF908B12923C3801C20D3
:10E03000FCF7C8F908B12923C380204B93F8854227
:10E04000012C01D0012038BD1D4DC3F88852FAF7CC
:10E05000E5FD1C4846F0B2FF4BF0B8FC002202215F
:10E06000432047F07FFA184A02F580534FF0A04052
:10E0700083F8A44383F8B143C2F8E009816B134CE1
:10E0800041F400118163C3F8A8434FF48174A3F8ED
:10E09000AC4305F12002002405F148014FF401656D
:10E0A00083F8AF43A3F8A6534DF038FA2246214631
:10E0B0004FF0FF3047F056FA204638BD884B00201D
:10E0C0009803002007003400A01800204000400101
:10E0D00070B5002486B0CDE90144CDE903440DF1CB
:10E0E000040CC0E92944C0E92B44C0F8B4400546FB
:10E0F00000F1B80EBCE80F00AEE80F00CEF800400B
:10E1000095F8D130059444F23B36A5F8FC600BB984
:10E1100006B070BD1C09013C072C03F00F032BD87F
:10E120001A4E06EB4402B2F84C0140FA03F2D20751
:10E1300022D5012202FA03F3013B2644184051F094
:10E14000A3F896F85C21124B024403EBC204294663
:10E150002623104DE380204641F80C5F4BF0E0FC95
:10E160000D49A2880868B2FA82F24FF00043D3400A
:10E1700003430B6006B070BD2946064B41F80C3FC7
:10E18000002006B0BDE870404BF0CABCD8F50508C9
:10E19000D439002075A80008003C0140264A92F8B6
:10E1A0007C337BB3D2F88013884235D0012B29D041
:10E1B000D2F88813814233D0022B23D0D2F89013A7
:10E1C00088422FD0032B1DD0D2F8981388422BD031
:10E1D000042B17D0D2F8A013884227D0052B11D0DA
:10E1E000D2F8A813884223D0062B0BD0D2F8B01354
:10E1F00088421FD0072B05D0D2F8B813814208BF40
:10E2000007230AD002EBC30103F1010CC1F880031C
:10E2100082F87CC3184670470023DBB2184670476B
:10E220000123FAE70223F8E70323F6E70423F4E7E0
:10E230000523F2E70623F0E79829002010B4037FB6
:10E24000083300EB43035B88047F9BB214B98469F5
:10E25000022C4BD0FF2B046837D80382037F012B9D
:10E2600015D08369032B22D08369022B1FD0038A28
:10E270006068DBB242EA03431F4A194300EA020323
:10E28000194341F0007161605DF8044B7047836988
:10E29000022BE6D1038A6068DBB242EA0343164AE6
:10E2A0000B430240134343F080736360ECE741EAA1
:10E2B0000203028A616810480140D2B20B4343EA6C
:10E2C000024363605DF8044B7047FF230382038AB7
:10E2D0000948DBB242EA0342636811430340194331
:10E2E00041F0807161605DF8044B7047448A838A15
:10E2F00023449BB2AEE700BF009800FCB0F1FF3FA3
:10E3000000F093812DE9F04F032883B0044600F319
:10E310009B80BE4D542000FB0450D0F8DC61002EE1
:10E3200000F092800C9FC0F8E8710127C0F8F471EA
:10E3300080F8F871A0F8F031002380F8FA3180F805
:10E34000FA3140F67103B069000415D4542303FB7D
:10E35000045393F8FA31DBB2DBB1542303FB0453CB
:10E36000012283F8FA2193F8FA31DBB2002B50D165
:10E37000012003B0BDE8F08F013BE4D1542303FB3F
:10E380000453122083F8FA0193F8FA31DBB2002B20
:10E39000E3D170689E4F384040EA410040F490302D
:10E3A0007060542000FB04504FEA410A80F8FA31B3
:10E3B00040F67103B069870710D5542303FB04535B
:10E3C00093F8FA31DBB2B3B1542303FB04530222B6
:10E3D00083F8FA2193F8FA31DBB2C7E7013BE9D1C0
:10E3E000542303FB0453122083F8FA0193F8FA3103
:10E3F000DBB2002BE8D1B262542202FB045292F845
:10E40000FA0170B3032382F8FA3192F8FA31DBB2E1
:10E41000ACE7542303FB04530022D3F8DC1183F848
:10E42000FA2140F671038A6992060FD5542303FB43
:10E43000045595F8FA31774A2023CB61B2F88C3233
:10E4400001339BB2A2F88C32002092E7013BEAD163
:10E45000542303FB0453122283F8FA2193F8FA3170
:10E46000E9E782F8FA3140F67103B269500613D534
:10E47000542303FB045393F8FA815FFA88F8B8F148
:10E48000000F16D0542303FB0453042283F8FA210F
:10E4900093F8FA31DBB269E7013BE6D1542303FB81
:10E4A0000453122283F8FA2193F8FA815FFA88F86C
:10E4B000E5E7594B542704FB07F7FB182F44184690
:10E4C0004FF41052514601934FF02A09FFF7B6FE60
:10E4D00097F8F83109FB04F94B44143305EB430377
:10E4E000B3F8C6319BB2002B4CD004EB440BCBEB02
:10E4F000CB0B07F5FD76D7F8DC0186F8008040F6F7
:10E500007103826951075CD53378DBB20BB1052307
:10E51000337097F8F831426A5B44083305EB8303A4
:10E52000D3F8C401411CC3F8C411027097F8F83144
:10E530004B44143305EB4303B3F8C621013A92B2BE
:10E54000A3F8C621B7F8EC31013B9BB2A7F8EC3138
:10E55000B7F8EC319BB253B997F8F8214A4414321A
:10E5600005EB4202B2F8C62192B2002A3CD197F8DC
:10E57000F8314B44143305EB4303B3F8C6319BB277
:10E58000002BB8D1542303FB04530022D3F8DC1131
:10E5900083F8FA2140F671038A69900618D554234E
:10E5A00003FB045393F8FA31DBB2002B3FD0542322
:10E5B00003FB0453072283F8FA2193F8FA31DBB204
:10E5C000D4E6013B9DD1122333703378DBB29DE753
:10E5D000013BE1D1542303FB0453122283F8FA21B7
:10E5E00093F8FA31DBB2E0E7D7F8DC01337040F69C
:10E5F00071038269120611D53278D2B2002A33D162
:10E6000001985146FFF71AFEB1E700BF903A00208B
:10E61000009800FC884B00206C3C0020013BE8D1B6
:10E62000122333703278D2B2E8E7002070472022FC
:10E63000CA614A6863F309024A604A6863F30C32AC
:10E640004A604A6863F317424A604A6863F3186293
:10E650004A604A6863F38A22542303FB04534A60E6
:10E6600093F8FA31DBB281E6542303FB045306220C
:10E6700083F8FA2193F8FA31DBB277E638B583698B
:10E68000023B0446072B0CD8DFE803F048482F2F45
:10E690000C0C040403689A69D20672D51022DA6160
:10E6A000A37F38BD0568AA6912F0100253D0102369
:10E6B000EB612B6843F020032B60AB69980744BFE4
:10E6C0000023AB62AB69D90703D4AB6943F0010304
:10E6D000AB61237F083304EB43035B889BB2002BC1
:10E6E000DED01123A377A37F38BD03689A69D506CE
:10E6F00040F1BA80027F083200EB4202528892B2A7
:10E70000002ACBD19969890748BF9A629A69D207D2
:10E71000C4D49A6942F001029A61BFE703689A691A
:10E72000D50677D51022DA619A69900701D50022C3
:10E730009A629A69D20703D49A6942F001029A61F7
:10E74000237F083304EB43035B889BB2002BA7D0E5
:10E750001123A377A4E7AB6913F0800300F0EC80EA
:10E760002B6823F040032B60037F083300EB430347
:10E770005B889BB2002B40F01F810D238377837F42
:10E7800038BD9A6912F0080240F0968099698D06AA
:10E7900086D52021D961196821F0FE0119605968D8
:10E7A00062F309015960596862F30C315960596884
:10E7B00062F317415960596862F3186159605968EA
:10E7C00062F38A2159609969880748BF9A629A69F9
:10E7D000D10703D49A6942F001029A619A695207FB
:10E7E00015D5227F596A04EB82039A68501C986001
:10E7F0001170238A9BB253B1227F04EB4202538AE9
:10E80000013B9BB25382238A013B9BB223820123AB
:10E81000637745E79A69910751D5027F00EB820241
:10E820009168481C90600A789A62227F04EB420249
:10E83000538A013B9BB25382238A013B9BB22382C2
:10E84000237F083304EB43035B889BB2002B7FF4E8
:10E8500027AF237F002B7FF423AFA369022B7FF424
:10E860001FAF012323771BE79A69100724D49A6905
:10E87000950700F1B0809A6912F0040286D0227FD9
:10E88000083204EB4202528892B2002A3FF408AFE9
:10E89000227F596A04EB82039A68501C98601170B9
:10E8A000227F04EB4202538A013B9BB25382238AAC
:10E8B000013B9BB22382F3E60822DA61F0E69A6913
:10E8C00015066BD49A695007E2D49A6912F0400297
:10E8D00040F0A480996989067FF5E2AE2021D961D4
:10E8E000596862F309015960596862F30C31596043
:10E8F000596862F317415960596862F318615960A9
:10E90000596862F38A2159609A69D00644BF10227F
:10E91000DA619A69910744BF00229A629A69D20724
:10E9200003D49A6942F001029A611A68012122F027
:10E93000F6021A606177B3E6AA6992067FF5B0AE77
:10E940002022EA616A6863F309026A606A6863F315
:10E950000C326A606A6863F317426A606A6863F33C
:10E9600018626A606A6863F38A226A60AB69DB06D0
:10E9700044BF1023EB61AB69980744BF0023AB622F
:10E98000AB69D90703D4AB6943F00103AB612B68D2
:10E99000012223F0F6032B60627781E6028A92B2AD
:10E9A0003AB9017F083100EB4101498889B2002959
:10E9B0002ED10D23A37773E66968C1F30901FFF730
:10E9C0003DFC238E102B2B680CBF43F4804343F493
:10E9D00000432B6064E6227F083204EB4202528837
:10E9E00092B2002A3FF45CAE227F04EB820291686F
:10E9F000481C90600A789A62238A013B9BB223826A
:10EA0000227F04EB4202538A013B9BB2538247E6CA
:10EA10005968C1F30901FFF711FC41E6227F083272
:10EA200004EB4202528892B26AB9227F12B9A269FB
:10EA3000032A0BD05A6895013FF532AE5A6842F46A
:10EA400080425A602CE60E23A37729E60122227722
:10EA500059684FF41052C1F309012046FFF7EEFB4D
:10EA60001EE600BF004809E66C3C0020004805E6B1
:10EA7000C03C0020004801E6143D002000B5224BB8
:10EA8000224D85B0CA24532100225C625962019252
:10EA900001955C625962019903240C60FF2159625F
:10EAA000596272B61A4BD3E9A41351EA03041DD17B
:10EAB0001046154B1749CA25532400265D625C6237
:10EAC000029602915D625C6202990860FF21124821
:10EAD000596259625D625C62039603905D625C629A
:10EAE0000398026059625962FEF7C0FF0B4A126830
:10EAF0004EF6602404FB00F0521843F10003821824
:10EB000043EBE070D5E700BF002800405C280040E0
:10EB1000884B00206028004064280040A018002096
:10EB200008B500210320FDF7DDFC72B6FEF78CFF6F
:10EB3000154C08B5D4F8983294F89E02ABB914205D
:10EB4000FBF7F8F900BFD4F898325BB11A689B88DC
:10EB5000116994F89E220B4012B91BB1FFF7E0FF38
:10EB6000002BFBD0F9F72AFEECE719689A880B69AD
:10EB7000134020B1002BE2D10B691340FAE7002BC0
:10EB8000DDD00B691340FAE7884B0020164A174B7B
:10EB90009042D3F8443328BF1046B0EB930F14D201
:10EBA000B0EBD30F13D2B0EB131F12D2B0EB531F45
:10EBB00011D2B0EB931F10D2B0EBD31F0FD2B0EB3A
:10EBC000132F0ED24FF4807070470220704704203C
:10EBD0007047082070471020704720207047402061
:10EBE00070478020704700BF0051250200000020C0
:10EBF00011F001010ED1F0B590F82850C668012D32
:10EC000083B0044607D0B6F1807F01D90123037792
:10EC100003B0F0BD70470A4B476AD3F8A002FFF774
:10EC2000B5FFB6F1807FB880F2D9B7260A462577BE
:10EC30002B46384601A98DF8046044F043FEE7E70F
:10EC4000884B00202DE9F0410546406A94B01446F7
:10EC500000681F460E464CF0E5FF0B94264C0C97BF
:10EC600004F582630093254B019302230022029353
:10EC70000123CDE90922CDE90E22CDE910228DF83C
:10EC80000C308DF834308DF8483006922B7F8DF89B
:10EC9000202013921A4A049204F5816205921A1DEB
:10ECA000079223B3330E84F8093404F20A44330C78
:10ECB000DFF850802370330A6370A670D8F8A00282
:10ECC0006C6AFFF763FF6B7FA0809BB169462046AB
:10ECD00044F03EFE6C6A20684CF0A4FFD8F8A8020D
:10ECE000FFF754FFA080384614B0BDE8F08104F26D
:10ECF0000944DCE705A9EAE7000000202C4E0020CB
:10ED000059890008884B00202DE9F04FBA4BBB4FC2
:10ED100085B007F1A00A4FF001094FF0000BA3F5F1
:10ED20002776B8460BE00BF1010BBBF1040F09F19C
:10ED3000010908F128080AF1050A00F0F78098F89F
:10ED40000030022BEFD19AF903305A1C18BFDBB206
:10ED5000A94A08BF002303EB430002EB800014BF65
:10ED60009E464FF00D0E5FFA8BF20D2B5CD8A44936
:10ED7000002404E00134202C01F1030154D00F7869
:10ED8000002FF7D14D789542F4D19E49D6F8A8507E
:10ED900004EB44040C44416894F88E418460A94219
:10EDA000047000F03581D6F8CC50A94200F05781AC
:10EDB000D6F8F050A94200F05681D6F81451A94275
:10EDC00000F05981D6F83851A94200F05881D6F8A0
:10EDD0005C51A94200F05F81D6F88051A94200F051
:10EDE0005681D6F8A451A94200F06181D6F8C851E5
:10EDF000A94200F06C81D6F8EC51A94200F06B8179
:10EE0000D6F81052A94200F06A81D6F83452A942CD
:10EE100000F06981D6F85852A94200F07081D6F806
:10EE20007C52A94200F06F810133DBB2734500F1DF
:10EE30000C009AD9002300939AF90420531C18BFA0
:10EE4000D2B26D4B08BF002202EB420414BF9446BD
:10EE50004FF00D0C03EB84045FFA8BF10D2A5BD8A5
:10EE6000674B002004E00130202803F1030353D056
:10EE70001F78012FF7D15D788D42F4D1614B00EB03
:10EE800040001844636890F88E51D6F8A800A56039
:10EE9000834225704DD0D6F8CC00834200F0DC8050
:10EEA000D6F8F000984200F0D380D6F814018342DF
:10EEB00000F0DD80D6F83801834200F0E480D6F817
:10EEC0005C01834200F0EB80D6F88001834200F0C1
:10EED000EA80D6F8A401834200F0ED80D6F8C8019C
:10EEE000834200F0F080D6F8EC01834200F0E78026
:10EEF000D6F81002834200F0FE80D6F83402834236
:10EF000000F0F580D6F85802834200F00481D6F86C
:10EF10007C02834200F0FB800132D2B2624504F1F0
:10EF20000C049BD90023C8E90433FCE605B0BDE816
:10EF3000F08F4FF0000E774607EBC70306EB830315
:10EF4000781C93F9BC70002FE6D12F4A83F8BD904E
:10EF5000132183F8BC1002937346D418C8F81440E8
:10EF60000190CDF80CE0FBF7BDFF029B264AD3F8D9
:10EF7000C430196865F306011960DDE90030002B23
:10EF8000D0D061680D6867F300050D600399515892
:10EF9000227C022303FA02F242F00C024A60D8F803
:10EFA00010205568D5F800C067F3000CC5F800C004
:10EFB000157C1268AB4043F00C035360D8F818304E
:10EFC0001024C3E902471F82D8F804205F600C3286
:10EFD0001A60D8F81C304FF480711A601982C3E9A6
:10EFE0000177DF6009493B463A46FBF7A1FF012361
:10EFF00088F80C3097E600BF9C020020344E0020B9
:10F0000064F70508D8F50508A400002099AB0008AE
:10F01000BC46394601EBC10706EB8707013197F97A
:10F02000BC50002D7FF400AF3D4B00916344C8F805
:10F0300010300846142387F8BC3087F8BD90FBF7E2
:10F0400051FFD7F8C4301A6864F306021A60F3E679
:10F050004FF0480E02276FE74FF0240E6CE74FF099
:10F06000240C0121D6E74FF0480C0221D2E74FF0E3
:10F070006C0E032760E74FF06C0C0321CAE74FF0DA
:10F08000900C0421C6E74FF0900E042754E74FF090
:10F09000D80C0621BEE74FF0B40C0521BAE74FF0BB
:10F0A000B40E052748E74FF0D80E062744E74FF087
:10F0B000FC0C0721AEE74FF0FC0E07273CE74FF4AE
:10F0C000A27E092738E74FF4907E082734E74FF4F3
:10F0D000907C08219EE74FF4A27C09219AE74FF427
:10F0E000B47C0A2196E74FF4C67C0B2192E74FF4DB
:10F0F000C67E0B2720E74FF4B47E0A271CE74FF4A7
:10F10000D87C0C2186E74FF4EA7C0D2182E74FF48E
:10F11000EA7E0D2710E74FF4D87E0C270CE700BFDE
:10F12000A4000020704737B590F85F38032B0446E1
:10F130002FD100231F4D8DF807309DF8073094F82C
:10F1400060289A4201D803B030BD9DF8073005EB26
:10F15000C30393F864338BB181F0010383B19DF84D
:10F16000073005EBC303D3F86003FBF711FA9DF8F2
:10F1700007300133DBB28DF80730DEE70B46EDE7F1
:10F180009DF8073005EBC303D3F86003FBF7FAF9EA
:10F19000EDE7D0E910039B7903F00103994204D015
:10F1A00003B0BDE83040FBF7F3B903B0BDE8304031
:10F1B000FBF7E8B9884B002038B5044600790D46C6
:10F1C00050B1FBF7FFF808B10323C380E279294669
:10F1D000BDE83840FBF7D0BF38BD10B504462A2142
:10F1E000FFF7EAFF62792068013A02239340DB438C
:10F1F000036161790122BDE810404DF0EFBC10B50C
:10F2000004460921FFF7D8FF617920680022BDE894
:10F2100010404DF0E3BC38B510F8133CA0F6640480
:10F220001BBB94F850388BBBD4E909239A421CD0FD
:10F230005A1CA169A262CB5C21695B0043F4007394
:10F24000A4F854380A2384F85238012384F850383B
:10F2500094F85F388A4228BF0022012BA26201D0B5
:10F26000042B02D1606CFFF7CAFF94F84C38002BD6
:10F270006FD194F84D380133DBB2092B84F84D3847
:10F2800025D12046BDE83840F9F7D6BA94F952584E
:10F290006DB1B4F854184B08A4F8543801F00101CA
:10F2A0002046013DFFF73FFF84F85258DDE7D4E9DF
:10F2B00009239A4284F85058D7D194F85F38012B2B
:10F2C00001D0042BD1D1606CFFF787FFCDE70A2B6B
:10F2D0003FD194F84F382BB9B4F8563843F00103B6
:10F2E000A4F856382379D9070AD5B4F85608820508
:10F2F00001D4C3071AD4B4F85C380133A4F85C38DD
:10F30000012284F84C2894F84F280023012A84F81D
:10F310004D381ED184F84F386279636C02F00102D7
:10F3200059791868BDE838404CF0F4B9E36AC0F385
:10F33000470013B1216B9847E2E7E3696269D05453
:10F34000E369E2680133B3FBF2F102FB1133E361DD
:10F35000D6E738BD1A4B00B5A3F5687C03F1300E33
:10F36000DA794AB15A790CEB82010CEB4202D1F8FE
:10F37000E81389B2A2F800140C337345F0D100EB06
:10F3800040030CEB830393F8A72332B10438012820
:10F3900093F8A5330BD9052B02D900205DF804FBA7
:10F3A0000CEB430CBCF8002490B25DF804FB052B79
:10F3B000F3D80CEB8303D3F8E80380B2EEE700BF89
:10F3C000284F00200548D0F8383323B1DB6A13B149
:10F3D00000F54E7018470248704700BF982900207A
:10F3E0008006060838B51D4CD4F80C341B8843B988
:10F3F0001B4D002384F81B3485F83033C5F82C33BB
:10F4000038BDD4F81024002AF2DDD4F81414012AEF
:10F41000488806D00123124DA4F8180484F81A3441
:10F42000E7E78A880132121A9A42F3D10C4DD5F8D7
:10F43000383300221B69C5F8642305F54E709847E0
:10F44000D5F838339B68002BD3D005F54E7098471C
:10F450000028CED14AF0E2FECBE700BF884B002067
:10F46000982900200748D0F834331BB1064B93F895
:10F470001A340BB100207047D0F8383300F54E70C5
:10F480005B68184798290020884B002030B4174A41
:10F49000174B92F830C303F21C4505EB0C04C0E98E
:10F4A000004593F81B3492F83003834292F83003FE
:10F4B00014D8834206D300231A46184630BCC1E94B
:10F4C0000032704792F830031A1EC0F1800330BC3E
:10F4D0000CBF01200220C1E9003270471B1A002234
:10F4E000012030BCC1E90032704700BF98290020DC
:10F4F000884B00200E4B0F4A93F8301392F81B04F0
:10F5000093F83023904293F830230CD8904238BFC0
:10F5100093F83023D3F82C333ABFC2F1800280181D
:10F52000002018447047D3F82C33801A18447047D1
:10F5300098290020884B002038B5194D194CD5F872
:10F540000C24937B012B08D0D4F82C3303F2FF73E7
:10F550006FF30A03C4F82C3338BDD4F838335B6A30
:10F5600063B104F54E709847D4F838339B681BB1EB
:10F5700004F54E70984778B1D5F80C24D4F82C33A4
:10F580005288013B13445242134003F2FF736FF35E
:10F590000A03C4F82C3338BD4AF040FEECE700BF44
:10F5A000884B00209829002070B51E4C1E4D94F801
:10F5B000303394F8301384B005F21C4213440293A4
:10F5C00095F81B3403928B4220D894F83023934251
:10F5D00014D294F830131E46C1F18001F3B98C4661
:10F5E0000122CDE9001610B9BCF13F0F06D9002366
:10F5F000694602A84DF058FA95F81B3494F8300388
:10F60000C01AB0FA80F0400904B070BD94F830C35D
:10F61000A3EB0C0C614600260122E2E701EB030C90
:10F620000222DEE798290020884B00202DE9F043D4
:10F63000164685B0002936D0441E254D254F04EBD3
:10F6400001084FF0000901E0A0452CD095F81B04FB
:10F6500014F8013F411C2844C9B280F81C340B0641
:10F6600048BF002097F8303385F81B144ABF014685
:10F67000084685F81B94994297F8303336BFC3F19A
:10F680008003C01AC0183F28DED997F8303399425A
:10F69000DAD0114B93F89430002BD5D00020FFF72F
:10F6A00083FFA045D2D1694602A8FFF7EFFE20B143
:10F6B000DDE9003213443F2B02D805B0BDE8F083EA
:10F6C0000246334602A84DF0EFF905B0BDE8F083DD
:10F6D000884B0020982900200000002030B585B01C
:10F6E000694602A8FFF7D2FE58B9094C04F54E75D9
:10F6F000D4F8383328465B6898470028F8D005B01E
:10F7000030BD0246012302A84DF0CEF9EDE700BF5F
:10F710009829002070B5134D134C0023C5F83433DD
:10F7200049F0FEFDC4F81404FFF74CFED4F814347D
:10F73000C4F80C04A3B19A885B88D21A436802FB10
:10F740000333C5F83433F9F707FA95F8303394F8F2
:10F750001B249A42064601D0FFF7C0FFC5F82C6370
:10F7600070BD00BF98290020884B00202DE9F04192
:10F77000104ED6F83433154682189A420E4A88BF86
:10F780001D1A92F81B2496F830339A4204460F460D
:10F7900001D0FFF7A3FFD6F8382308480023C6F8A6
:10F7A00064332B46956A21463A46AC46BDE8F041A3
:10F7B000604700BF98290020884B0020D02C0020F3
:10F7C0008C461346014662461846CFE72DE9F04FB6
:10F7D00041F694628DB00021A5484FF0C1FCA54AC6
:10F7E0000023099309920999043209680A930A923D
:10F7F0000A9A126851EA020040F02B819E4B039353
:10F800004C2200219A489D4D4FF0AAFC00214C2229
:10F8100097484FF0A5FC039B954AD3F844341560F4
:10F8200001241471D3611746136253624CF028F817
:10F83000FFF770FF002108460DF098FFF9F78CF9EB
:10F84000B0F1000840F3A5818D4DDFF858E28D4EF0
:10F85000CDF808E0002407F14C0901942746A3469F
:10F8600005F29C4A04E00BF5006BD84540F3B080EC
:10F87000854B029A1B68C2F8D432F8F79FFF20220A
:10F8800051465846FFF772FF8049122250464FF00A
:10F89000A4FC0028E7D1BB4525D001997C4B01EBA6
:10F8A000410203EB820301934A1C184679490592F1
:10F8B000ABEB0703049301F0BBFB4946019B41F806
:10F8C0004C3B049B059AC9F80C70C9E90433D9F87C
:10F8D0001C300192C9E908336F4BC9F82830012365
:10F8E000C9F808308946039BD3F84434C9F81C3062
:10F8F0005F461222A918335D91F89C14994202F1D7
:10F9000001020BD00024202AF4D12037B8455146FB
:10F91000384653DBFFF72AFF0022EBE70134152CB2
:10F92000F1D1D0195D4F20223946FFF71FFF38462D
:10F9300000230A220BA90B9701F0ACFC07460B9899
:10F94000002301300A220BA90B9001F0A3FC0790C1
:10F950000B98002301300A220BA90B9001F09AFCAE
:10F9600006900B98002301300A220BA90B9001F09E
:10F9700091FC05900B980BA9013000230A220B90F3
:10F9800001F088FC04900B98002301300A221946EC
:10F9900001F080FC97B1DDE9063243EA4212049B94
:10F9A00005995B0143EAC123A7F2BC7143EA6003F6
:10F9B00042EA412243EA0243C9F81C30019B642B0E
:10F9C00000F0B5805F460BF5006BD8453FF750AFB0
:10F9D000019B642B00F0AB80BB451DD0019B2C4CE0
:10F9E0002C490C2202FB03445E1C3246204601F0E7
:10F9F0001FFBD9F81C20C9F80040ABEB0705C9E98B
:10FA00000822C9E90375244AC9F828200122C9F847
:10FA100014500196C9F80820019B002B03F1010145
:10FA200000F388804FEA4803B3F1805FC0F2B280F0
:10FA30000F4B9C6834B91A461B791BB11368002B15
:10FA400040F0DE80002108460DB0BDE8F04F0DF01B
:10FA50008DBE98184FF47A7200234DF079FF104B49
:10FA6000A3FB00231B0C40F2B27240F26D141DE0A8
:10FA700068660020602800400000002080DD060845
:10FA8000884B002044710608A01800202071060849
:10FA90004450002034710608C1F7000824500020AB
:10FAA00007452EC2982900205B1A013212F0030587
:10FAB00014BF21464FF4B7718B42F5DAA349002DEC
:10FAC00000F0988003910399D1F814148B42C0F28E
:10FAD0003A819F4D01245B1A55F8041F994204F1A5
:10FAE0000104F8DD013343EA4413A2F2BC7243EA95
:10FAF0004223984A039DB0FBF2F102FB11024FF43E
:10FB000061603C24B2FBF0F100FB11221C20C5F81F
:10FB10001804B2FBF4F004FB1022521042EA401227
:10FB200042EAC12242EA0343C5F8443468E664234A
:10FB3000019365214C268848DFF830A2874F06FBE9
:10FB400001F405193246002128464FF009FB3246E0
:10FB5000002128464FF004FB7F48814E40F804A066
:10FB600004F110034FF00109C5F808902F62AE624E
:10FB700040F803800344021DC3F804801834039B3B
:10FB80000199D3F844341351A018023143606B62D9
:10FB900048E72146704BDFF8D8914C2606FB01F46C
:10FBA0001D193246002128464FF0DAFA324600216C
:10FBB00028464FF0D5FA684B684E43F80490039AF4
:10FBC0002E62684ED2F8440404F1180104F11002C8
:10FBD0000127341FC8F10063BB404FF0020A85F8CB
:10FBE00005A0AF60A3502244536070503144486078
:10FBF00068621DE70C4603911D21C4F8181462E7E2
:10FC0000554900220023C1E910238C640A46CC63C5
:10FC100026462146D56C02F14C03B5B198689E6426
:10FC20004D1EA842C2E92366DE6300F085804D1CAC
:10FC3000A84273D113F8481C00293FF403AF1A649B
:10FC400043F8083C01461A46E4E7434A022629469F
:10FC500015E0D36B16635B0118BF03F6FF73C2E9AF
:10FC6000041114BF00EB13333346536318469063FB
:10FC700052F84C7FC31A1D44461C0134CFB113798E
:10FC8000701E002BE5D1136916635BB103F6FF7399
:10FC9000576900EB133353634FB107F6FF7700EB5F
:10FCA0001730E4E7576933465363002FF5D13046E8
:10FCB000DDE7DFF8C0E0CEF824432B4CCEF8FC4261
:10FCC00040240138CEF81853CEF808433F253E248F
:10FCD000CEE9C045CEF81403820F8300E0B140F2B4
:10FCE000FF141B1942F100025B0A43EAC25303F1FD
:10FCF0004002134403EBC000CEF81033C30DCEF81E
:10FD0000F432154BCEF80C23CEE9C7334302CEF8BC
:10FD1000F802CEF8F03295E60123E8E788427FF456
:10FD200091AE00293FF48EAE106CC56B0135C563F2
:10FD3000186493641A466DE700293FF483AE53F8C4
:10FD40000C2C0146EDE70124CCE600BF00000020AA
:10FD50001404002080510100686600200068214CD6
:10FD6000C1F700086C660020787106085C7106080F
:10FD70006C710608982900202DE9F043DFF82881EE
:10FD8000474D93B0FFF72EFB98F8303395F81B24BE
:10FD90009A4201D0FFF7A2FCD8F834730024C8F8C7
:10FDA0002C43002F6CD03F4E0AE098F8303395F882
:10FDB0001B249A4201D0FFF791FC2034A7421BD9A3
:10FDC00022463146684601F033F968464DF062F943
:10FDD000012201466846FFF729FCA3B2002BE4D1BB
:10FDE000D8F8D832002BE0D09A881B6859690A42AB
:10FDF00018BF12049A61D8E7FFF79EFB98F83033DA
:10FE000095F81B249A4201D0FFF768FC0023DFF825
:10FE10009490C8F82C331E461C4601E0A74229D90D
:10FE20002246494609A801F003F92122002168462B
:10FE30004FF096F9202269462046FFF797FC2022D2
:10FE4000054609A968464FF0C8F908B9202D00D029
:10FE50000136A3B22034002BE0D1D8F8D832002BE1
:10FE6000DCD01A689B8851690B4218BF1B04A7425B
:10FE70009361D5D8B6FA86F0400913B0BDE8F08397
:10FE8000FFF75AFB98F8303395F81B249A4201D0BB
:10FE9000FFF724FC0023C8F82C330120EDE700BF56
:10FEA000884B0020807106089829002000B501EBDE
:10FEB000020E714516D001390EF1FF3E41F2210CC0
:10FEC00011F8013F082280EA032003B2002B4FEA19
:10FED0004000B6BF8CEA430380B298B2013AF4D135
:10FEE0008E45EDD15DF804FB704700BFD0ED007A80
:10FEF000D0ED016A30EE677AE6EE877AB0EE670AF7
:10FF0000C0ED007A704700BFD0ED017AD0ED026AF3
:10FF100030EE677A90ED000AE6EE877A37EEC07A27
:10FF2000C0ED017AA6EE870A80ED000A704700BF97
:10FF300090ED017AD0ED036AD0ED027A30EE470AF7
:10FF4000A6EE807A90ED000A80ED017A37EE676ABE
:10FF5000E6EE867A37EEC07AC0ED027AA6EE870A20
:10FF600080ED000A704700BFD0ED056AD0ED017A40
:10FF700090ED066AD0ED025A90ED035AC0ED066A84
:10FF8000B0EE407A26EEA70AD0ED007A80ED057A31
:10FF9000A7EE870AD0ED077AA5EE860A90ED086AEB
:10FFA000D0ED045AC0ED087AA5EE670AA5EEC60AA0
:10FFB00080ED070A704700BFF0EE406AD0ED007A8E
:10FFC00090ED050A90ED067A90ED016AD0ED035AA6
:10FFD000A7EEA60AA6EE267AD0ED047A90ED026A84
:10FFE00067EEC07AA5EEC07AE6EE267A80ED057A55
:10FFF000C0ED067A704700BF2DE9F047DDF820A07C
:020000040801F1
:1000000055460F4615F8011B002B064614460CBF3B
:100010004FF020094FF0300939B3002A2BDD2B4671
:1000200000E09CB113F8012BA046013C002AF8D156
:10003000A8F1020854B1444649463046B847013C4D
:10004000FAD29AF8001008F1010459B13046B847C5
:100050002B4615F8011B0029F8D1A4EB0A04181946
:10006000BDE8F0872046BDE8F087002A02F1FF389E
:10007000E1DC0846F4E70024E8E700BF03685A1C07
:1000800002601970704700BF10B500F100440246CD
:10009000013C04E0B3EB0E0015D1A24214D012F8DB
:1000A000013BA3F14100192811F8010BA0F1410C0B
:1000B00098BF2033BCF1190F00F1200EEAD91B1AAA
:1000C00004D10028E9D110BD002010BD184610BD94
:1000D000884210B54FF001043ED301FB04F4B0FB9D
:1000E000F4FC8C45F9D2CCB122BB08E0A14203F864
:1000F00001EBB4FBF1F211D8B0FBF2FC1446BCF1F9
:10010000090F0CF1570E0CF1300204FB1C00EDDC62
:10011000A14203F8012BB4FBF1F2EDD900221A70D1
:1001200010BDA14203F801EBB4FBF1F2F6D8B0FB2D
:10013000F2FC1446BCF1090F0CF1370E0CF1300241
:1001400004FB1C00EDDCA14203F8012BB4FBF1F22F
:10015000EDD900221A7010BD8446002AEAD1CEE7FC
:10016000002870B503DA2D2301F8013B404209282D
:1001700086464FF0010307DD03EB83035B00B0FB12
:10018000F3F2092AF8D8E3B10F4CA4FB0320BEFB1D
:10019000F3F2092A02F1570602F130054FEAD000C6
:1001A00007DD092B01F8016B03FB12EE09D90346A9
:1001B000EBE7092B01F8015B03FB12EE01D90346C3
:1001C000E3E700230B7070BDCDCCCCCC0378202BA3
:1001D000024600F10100F9D0092BF7D02D2B28D0D1
:1001E0002B2B03BF5378B7EE000A0246B7EE000A86
:1001F000A3F13001C8B209289FED567A10D8F2EE6B
:10020000046A07EE901AF8EEE77A12F8013FE7EE7B
:10021000267AA3F13001C8B20928B0EE677AF0D986
:100220002E2B5ED003F0DF03452B07D020EE070A0C
:1002300070475378BFEE000A0246D9E710B45178F0
:100240002D2978D02B296AD0A1F13003092B02F196
:1002500001026BD80024002303EB830301EB43036B
:1002600012F8011FA1F130000928A3F13003F3D9DE
:10027000B3F59A7F1A4628BF4FF49A72072B66D9B6
:10028000DFED356A1346F7EE007A083B072B67EE81
:10029000A67AFAD802F00702DAB1F2EE046A012A6D
:1002A00067EEA67A15D0022A67EEA67A11D0032A45
:1002B00067EEA67A0DD0042A67EEA67A09D0052A41
:1002C00067EEA67A05D067EEA67A062A18BF67EE13
:1002D000A67A6CB387EE277A5DF8044B20EE070A06
:1002E00070475378A3F13001C8B2092802F1010226
:1002F00098D8F2EE046AF0EE665A07EE901AF8EE1D
:10030000E77A12F8013F87EEA66AA3F13001C8B27E
:10031000092866EEA56A37EE067AEED982E791786B
:10032000A1F13003092B02F1020293D9F7EE007A12
:1003300027EE277AD0E79178A1F13003092B02F15B
:10034000020288BFF7EE007AC4D8012483E7F7EEF3
:10035000007AA1E70000000020BCBE4CF8B5164DA5
:100360006B78BE2B25D1022229464FF6FF70FFF78E
:100370009DFD124FAC1C22884AB1A618BE4218D26D
:10038000052A16D92146FFF791FD3446F3E72146A9
:100390000222FFF78BFD0222A118FFF787FD06342A
:1003A000074B641B1C8041F60F53C31A5842584137
:1003B000F8BD0020FCE700BF0040000800800008F6
:1003C000A8A50020F0B5067906F0E003402B03D184
:1003D00045794FF0FF3406E0602B4FF00105F8D16E
:1003E000447905FA04F40023012006F00706AB4225
:1003F00000D1F0BD052E0FD8DFE806F00308101D70
:10040000242448B1C85CD75C78400FE020B1C856BE
:10041000D756C71B784278410133E8E70028FBD064
:1004200031F8130032F81370784080B220420CBFCC
:1004300001200020F0E70028EED031F9130032F956
:100440001370E6E70028E7D051F8230052F8237034
:10045000DAE7037903F01803102B1CD003D833B963
:10046000B0F80B007047182BFAD000207047104BE3
:10047000B0F80B0093F90030591C06BF0D4B1B79E7
:10048000DBB203EB430203EB820303EBC30300EB9A
:10049000430080B27047064BB0F80B0093F901306F
:1004A0005A1C06BF034B5B79DBB200EB4310F0E74D
:1004B0005C040020A8A50020032870B518D80D4BB7
:1004C000C60003EBC000C943057F427F01F0010174
:1004D00081EA0504A2420BD082693AB14D1B694200
:1004E00010689288694109018A40826133445C77CF
:1004F00070BD00BFA8A500200379062B0FD1C9B29B
:100500000E2998BF074BC26894BF5956002101239A
:100510008B40134214BF08464FF0FF307047481C11
:10052000704700BFA8710608092900D001B97047BB
:1005300001394A0002F00802930001F00301A3EB25
:100540009203C1EB0111C3EB0313C1EB01110022B4
:100550009B0089000260818043807047B5EEC00A2D
:10056000DFED347AF1EE10FACCBF30EE270A30EE30
:10057000670ADFED317A20EE270A30B5FDEEC07A4A
:1005800087B017EE904A054684EAE470002303A979
:10059000A0EBE470CDE90033029347F095F8002C0E
:1005A000B4BF2D23202303A88DF800304CF072FD3A
:1005B000012829D0022833D003281DD003A968467A
:1005C0004EF0D6FD68464CF065FDC41EE4B22246EE
:1005D000694628464EF06CFD00232B5528464CF00A
:1005E00059FD2E232B5401300DEB040128444EF00D
:1005F000ECFD284607B030BD302303A968468DF8CE
:1006000001304EF0B5FDDDE743F23002302303A99F
:100610006846ADF801208DF803304EF0A9FDD1E712
:1006200043F2300303A96846ADF801304EF0A0FD57
:10063000C8E700BF6F12033A00007A440CF010BD07
:1006400038B5054658B14C1E14F8011F284619B993
:10065000BDE838400CF018BD0CF002FDF4E738BDE1
:1006600070B50546B0F8090044F0CAFB064B93F894
:10067000386004462846FFF7ECFE16B1E3681844DC
:1006800070BDA368FBE700BFA8A5002038B50546EC
:100690000C46FFF7E5FF2A7902F0070302F0E002BB
:1006A000602A29D1052B0CD8DFE803F0030B0F0BD0
:1006B0001B1B6A7901239340DBB2027814B1134308
:1006C000037038BD22EA0303FAE76A7901239340F5
:1006D0009BB2028814B113430380F2E722EA0303BA
:1006E000FAE76B7901229A40036814B1134303605F
:1006F000E7E723EA0203FAE7052BE2D8DFE803F095
:100700000303050507070470DBE70480D9E70460ED
:10071000D7E708B520214EF03AFD0346184623B12D
:100720000278202A03F10103F8D008BD08B5CB07F1
:1007300001D4FDF79BF908BD2DE9F341124D134F8C
:10074000002305F8393F044600EB8106B44203D18B
:100750000F4802B0BDE8F081394628464EF008FD4A
:10076000214668464EF031FD4FF0000820216846D2
:100770004EF00DFD28B9694628464EF0F9FC0434C8
:10078000E4E780F80080F1E7A8A5002079E10608F9
:10079000E1A500202DE9FF47914604468A461E4602
:1007A000FFF7AAFE421CBDF83070DDF83480054624
:1007B0001FD0B9F1FF3F1FD0CDE90009144A2368CB
:1007C00031463846C0474A4620795FFA8AF1FAF73F
:1007D000DBFB024600B10288D3B20393C2F30323CA
:1007E000120BCDE90052029323680A4A314638467B
:1007F000C04704B0BDE8F0877B06FAD40C902368AC
:10080000054A31463846C44604B0BDE8F047604763
:100810006CE0060879E006089EE006082DE9F04342
:10082000154685B06A1C8946BDF830600D9F194693
:1008300028D04FEA101800F00F0408F14008CDE965
:100840000045174A43463046B847C0B1EBB20D2BBE
:10085000D9F8000099F8051011D82A46FAF7E8FBF4
:1008600068B1038802780392C3F303221B0BCDE91E
:100870000043029243460B4A00213046B84705B078
:10088000BDE8F0837306FAD40309074A00F00F00AD
:100890000C9040333046BC4605B0BDE8F04360479D
:1008A000ADE00608BFE00608E9E006082DE9F043E0
:1008B00087B04FEA1018DDF8389015461F4608F14A
:1008C000400800F00F0421B30DF004F9C379164A73
:1008D000CDE900430646434629463846C847A8B1F5
:1008E0003068FAF7F5FBB3791049727913F0020F0B
:1008F0000F4B18BF0B46F1790094CDE90331CDE9D8
:10090000010243460B4A00213846C84707B0BDE8FC
:10091000F083094A0E94434629463846CC4607B030
:10092000BDE8F043604700BFFDE0060863E206084B
:100930002DED06080FE1060831E1060848400823BE
:1009400041B240000029C0B2B8BF5040013BF7D1CE
:10095000704700BF30B505688D42044618D901F1D3
:10096000FF3E681E00231EF801CF082183EA0C0316
:100970004FFA83FC5B00BCF1000FDBB2B8BF534001
:100980000139F5D17045EED16A1C22602B7030BD63
:1009900000236A1C22602B7030BD00BF10B52DED06
:1009A000028B08EE101AB8EE488ADFED7E7ADFED92
:1009B0007E0A28EE008A044628EE278AB0EE480A0E
:1009C0004DF048FE9FED797AB4EEC70AF1EE10FAC9
:1009D000F0EE407A40F3BD809FED736ADFED746AFC
:1009E000B0EE677AB4EEE67AF1EE10FA77EEC67AF8
:1009F000F6DC9FED707AF4EEC77AF1EE10FA40F370
:100A0000C5809FED6A7A77EE677A27EEA76ADFEDF9
:100A10006A5ADFED6A6A9FED6A7A9FED660ADFED3A
:100A2000620AE6EE256A67EE865AA6EE267A38EE68
:100A3000000AE5EE877AB0EE678A4DF00BFEDFED37
:100A40005B7AB4EEE70AF1EE10FA5BDDDFED566A91
:100A50009FED577AF0EE407AF4EEC77AF1EE10FA95
:100A600030EE660AF6DCDFED537AB4EEE70AF1EE1B
:100A700010FA62DDDFED4D7A37EEC00AF7EE007A4C
:100A8000DFED504ADFED4C5A9FED4C7AC4ED097A08
:100A9000B0EE675AA8EE245A0023A36160EE006A04
:100AA00087EE856A63612362E361A6EEA57A9FED16
:100AB000445AA6EE875A20EE264AF0EE675AA4EE74
:100AC000050AE8EE645ABDEC028BB6EE007AF8EE49
:100AD000006A77EEC07A26EE077A66EE266A27EE7F
:100AE000277A66EE806A67EE867A25EE866A84ED5E
:100AF000007AC4ED017A84ED027AC4ED036A84EDD4
:100B0000046A10BDDFED307AB4EEE70AF1EE10FAB8
:100B1000A9D5DFED256A9FED2D7AF0EE407AF4EE4F
:100B2000C77AF1EE10FA30EE260AF6D4DFED217A1C
:100B3000B4EEE70AF1EE10FA9CDCDFED257AB4EEB4
:100B4000E70AF1EE10FA44BFDFED1F7A37EEC00A74
:100B500094E79FED1D7AB4EEC70AF1EE10FA7FF527
:100B600048AF9FED116ADFED196AB0EE677AB4EE17
:100B7000E67AF1EE10FA77EE867AF6D49FED0D7AEA
:100B8000F4EEC77AF1EE10FA3FF73BAF9FED107A23
:100B9000F4EEC77AF1EE10FA44BF9FED0B7A77EED0
:100BA000677A32E727D4D236DB0FC940DB0F4940E2
:100BB000E4CB1641DB0FC93F92E741B99730083CBF
:100BC00015A82ABEF304353FDB0F49C0E4CB16C19C
:100BD000DB0FC9BF08B5DFED2D0A4DF03BFDDFEDA2
:100BE0002C7AB4EEE70AF1EE10FA28DDDFED276A81
:100BF0009FED287AF0EE407AF4EEC77AF1EE10FA23
:100C000030EE660AF6DCDFED247AB4EEE70AF1EEA8
:100C100010FA2FDDDFED1E7A37EEC00A20EE007AE3
:100C20009FED1E6ADFED1E6ADFED1E7AE7EE066AB3
:100C300020EE076AE6EE877AA6EE270A08BDDFED0A
:100C40001A7AB4EEE70AF1EE10FADCD5DFED0F6A9E
:100C50009FED167AF0EE407AF4EEC77AF1EE10FAD4
:100C600030EE260AF6D4DFED0C7AB4EEE70AF1EEA8
:100C700010FACFDCDFED0E7AB4EEE70AF1EE10FAEF
:100C800044BFDFED097A37EEC00AC7E7DB0FC94082
:100C9000DB0F4940E4CB1641DB0FC93F92E741B976
:100CA0009730083C15A82ABEDB0F49C0E4CB16C11B
:100CB000DB0FC9BFB0EEC07AF0EEE06AF4EEC76AAF
:100CC000F1EE10FAB4BFF0EE475AF0EE665AF5EEC8
:100CD000405AF1EE10FAF0EE407A44D0F4EEC76AD2
:100CE000F1EE10FA8CBFB0EE475AB0EE665A85EEC0
:100CF000256A9FED1E2A9FED1E3A9FED1E4ADFEDED
:100D00001E4ADFED1E2ADFED1E3A9FED1E5AA6EEAB
:100D1000423AE6EE223AA6EE034AF7EE005AE6EE33
:100D2000044AE6EE235AA6EE245A85EE250AF4EE8E
:100D3000C76AF1EE10FA48BF9FED137AF5EEC00ACC
:100D400048BF37EE400AF1EE10FA48BF9FED0F7A28
:100D5000F5EEC07A48BF37EE400AF1EE10FA48BF10
:100D6000B1EE400A70479FED070AE0E739094E3DB2
:100D7000E3B59E3E88FA163E45FE7F3F99FB243F31
:100D800069A2163EA7DFA834DB0FC93FDB0F49403D
:100D90002DE9F04F144689B088462178013203923C
:100DA000002900F01681002507461E46A94609E0E5
:100DB0003846C047039C01352178631C0393002902
:100DC00000F08F802529F3D16078A31C3028CDE96D
:100DD000033923D0A0F13003DBB2092B4FF0000A16
:100DE00026D96C282AD078287FD8572878D9A0F11E
:100DF0005803202B79D8DFE803F0BD78787878782D
:100E0000787878787882AF78787878787878787821
:100E1000AA787878789E788A7878BD00A078E31CE4
:100E20000393A0F13003DBB2092B4FF0010AD8D8AD
:100E300004AA03A948F088FA6C28D4D1039C22782C
:100E40000134782A0394B7D8572A40F28E80A2F151
:100E50005803202BB0D801A151F823F0930F0108BB
:100E6000B90D0108B90D0108B90D0108B90D010846
:100E7000B90D0108B90D0108B90D0108B90D010836
:100E8000B90D0108B90D0108010F0108AF0F0108E4
:100E9000B90D0108B90D0108B90D0108B90D010816
:100EA000B90D0108B90D0108B90D0108B90D010806
:100EB000B90D0108510F0108B90D0108B90D01085C
:100EC000B90D0108B90D0108390F0108B90D010864
:100ED000BF0F0108B90D0108B90D0108930F0108F2
:100EE00028B9284609B0BDE8F08F039C64E725289F
:100EF000FBD1039C25213846C04701355CE7039CA4
:100F000056F8041B3846C9B2C047013554E70DF105
:100F1000140B56F8040B039C5B4600220A21FFF7D2
:100F2000D7F8049ACDF800B0534641463846FFF74B
:100F300063F8054440E7039C56F8043B0093049A89
:100F4000002341463846FFF757F8054434E7039C31
:100F500056F8043B1D602FE70DF1140B56F8040BF7
:100F6000039C5946FFF7FCF8DBE7002AB9D0252A95
:100F7000C0D021E7A0F15802B2FA82F20DF1140BB1
:100F800056F8040B52095B461021FFF7A1F8039CA9
:100F9000C7E7A2F158020DF1140BB2FA82F256F82B
:100FA000040B52095B461021FFF792F8B9E70DF1E7
:100FB000140B56F8040B5946FFF7D2F8B1E70DF1C0
:100FC000140B56F8040B5B4600220A21FFF780F849
:100FD000A7E70D4685E7F8B5104C0746E06D0D46CE
:100FE0001646A0B10E49FFF72BFBE06D3946FFF71F
:100FF00027FB0C49E06DFFF723FB0B49E06D3346FF
:101000002A46FFF7C5FE0949E06DFFF719FB94F882
:10101000603013B1012384F86130F8BDA8A5002029
:1010200043E106081BF906083D06010850E10608E1
:101030000EB400B584B005AB019053F8042B0649FB
:10104000039301A8FFF7A4FE019B00221A7004B0CD
:101050005DF804EB03B070477D000108F7B5114E51
:1010600007463046002300F8623F0C460E4B0F49FE
:10107000002F18BF194615464EF07AF80C4F04EBB6
:1010800045056236AC4202D10A4803B0F0BD39468C
:1010900034F8022B6846FFF7CBFF694630464EF026
:1010A00067F8EFE7A8A5002054E106085DE106080F
:1010B00066E106080AA60020F7B50C4E0C4F002387
:1010C00006F8933F044600EB4105AC4202D10948C3
:1010D00003B0F0BD394634F8022B6846FFF7A8FF8D
:1010E000694630464EF044F8EFE700BFA8A500205F
:1010F00010E206083BA60020F8B5084F4E1E054634
:1011000001F11F0416F8012F28463946FFF790FF1A
:10111000A64205F10205F5D1F8BD00BF6BE1060856
:101120000246531C084605D1034B1A681B790A6016
:101130000B71704701497BE7A8E0060811E2060839
:1011400010B5013114460CF0C5FC28B9054B1A68DE
:101150001B792260237110BDC27903492046BDE886
:10116000104065E7A8E006080AE1060803685A1C73
:10117000026019700368090A5A1C026019707047EE
:1011800010B402681346511C016013F8021B03607F
:10119000D31C5478036093781B0443EA0423141D82
:1011A0000460D0785DF8044B0B4343EA006070475D
:1011B000A0F13003092B07D920F02000413819286D
:1011C0008CBF00200120704701207047303809286B
:1011D0008CBF002001207047413819288CBF0020A7
:1011E00001207047613819288CBF0020012070470A
:1011F000202805D0093804288CBF00200120704722
:1012000001207047A0F14103192B98BF203070478F
:10121000A0F16103192B98BF2038704702B310B5B5
:101220008446841803E0981A15D1A44514D01CF8FC
:10123000013BA3F14100192811F8010BA0F1410E67
:1012400098BF2033BEF1190F00F12002EBD91B1A11
:1012500004D10028E9D110BD002010BD184610BDF2
:101260001046704770B5044608460D464BF012FF15
:10127000064602E014F8013F43B1324629462046B3
:10128000FFF7CCFF0028F5D1204670BD1C46204654
:1012900070BD00BF2DE9F043064686469EF800C0AB
:1012A000BCF1200F7446ACF109050EF1010EF5D02A
:1012B000042DF3D9BCF12B0F64D0BCF12D0F26D136
:1012C0000127102A94F801C004F1010423D04FF043
:1012D000FF35B5FBF2F502FB05FE6FEA0E0E5FFA75
:1012E0008EFE9046002014F801CBBCF1390F4CF073
:1012F0002009ACF1300C29D85FFA8CFC944528DA2F
:10130000A84226461ED81BD000FB08C0EBE7102AD7
:101310004FF00007DBD1BCF1300F0AD16078A0F1AB
:101320004105192D98BF2030661C78280CBF023467
:1013300034466FF070454FF00F0E4FF01008D1E7B4
:10134000F445E1D94FF0FF301F40CCE7B9F1600F11
:101350000AD801B10E6067B923B16FF0004398421B
:1013600028BF1846BDE8F083A9F157095FFA89FC48
:10137000C4E723B1B0F1004F28BF4FF00040404216
:10138000BDE8F08300279CE773B50E46104905467B
:10139000FEF77AFE18B93070012002B070BD2C78CB
:1013A000602C8CBF613C413C082C0FD801350123D7
:1013B0000A2201A92846FFF76DFF019BAB4205D029
:1013C0000F2803D8013440EA0410E4E70020E4E7E2
:1013D000A8E0060801230A2200215BE770B50D464C
:1013E0001446FFF796F90646A0B1FFF7F3FF40F663
:1013F00034039842A8BF1846B0F5617FB8BF4FF4D8
:101400006170A0F561731922B3FBF2F32B7023789E
:10141000013323703046FFF77CF90646A0B1FFF791
:10142000D9FF40F634039842A8BF1846B0F5617F53
:10143000B8BF4FF46170A0F561731922B3FBF2F3EA
:101440006B70237801332370304670BD2DE9F04175
:1014500016461F460446394630464FF47A7200233A
:101460004CF076FA3C4D3D4B054483FB0560284427
:10147000E917C1EB601183FB01030B44384EC81719
:10148000C0EB631086FB003CC317364EC3EBAC03C6
:1014900086FB03764FEAE37ECEEBE61EC1EB011638
:1014A000A5EB860CC0EB0015A1EB8501617103EB88
:1014B0004301A0EBC10040F2B55101FB1E33B3F56F
:1014C000896F84F806C020714FEA8E0633DA40F245
:1014D000DA218B4237DCB3F5B77FB4BF4FF0000E93
:1014E0004FF0010E204F0EEB4E0107EBC101754688
:1014F000C88A4FEA4E0808EB0E0C07EBCC0C0CF137
:10150000160C0B2101E03CF8020D984210DD013968
:10151000F9D1F044012137F83800A170013306F504
:10152000FA6E1B1A7544E37022812580BDE8F081B4
:101530000131C9B2F1E703250B4F40F29650AE4698
:101540004FF00608D7E70225074F40F22940AE4684
:101550004FF00408CFE700BF80BC92C78988888815
:10156000ABAAAA2A73B06D16BC0606080C4B10B5C0
:10157000D3E9004354EA030209D1014640F20113C2
:101580000020C1F8023088710880088110BD054A2A
:101590001268121943F10003FFF758FF012010BD34
:1015A000184E0020A01800202DE9F0410446944276
:1015B0001546084609D2B4FBF2F6154B05FB164456
:1015C0001B5D00F8013BBDE8F081B4FBF2F69642EA
:1015D000B6FBF2F70CD20E4B05FB176705FB164462
:1015E000DA5D00F8012B1B5D00F8013BBDE8F081DE
:1015F000BA42B7FBF2F807D9054B05FB187813F888
:10160000082000F8012BE7E74046FFF7CDFFF3E79E
:10161000B871060830B5694CB4F8E834B4F8EE2473
:10162000B4F8F014B4F8F204B3F57A7F88BF4FF43D
:101630007A7383B088BFA4F8E834B4F8EA34B3F519
:101640007A7F84BF4FF47A73A4F8EA34B4F8EC34A8
:10165000B3F57A7F84BF4FF47A73A4F8EC34B2F513
:101660007A7F84BF0022A4F8EE24B1F57A7F4CD9AA
:101670004FF47A718842A4F8F01466D89A4224BFD5
:101680000023A4F8EC34884224BF0023A4F8F034EB
:10169000B4F80035B4F8FE249A4284BF0023A4F8BD
:1016A000FE34B4F80835EBB1454DAA78062A3ED988
:1016B000297900296FD19FED437A94F8AC2807EE81
:1016C000903A06EE902AF8EEE77AB8EEE66AAB7941
:1016D000C6EE276A0BB137EE077AB4EEE67AF1EE82
:1016E00010FA3ADC6279032A1DD8374B03EB421318
:1016F0002279C4F8B438032A0ED8344BEA2102FB0D
:101700000133C4F8B83803B030BDB0F57A7F84BF78
:101710000020A4F8F204B1E72C4BC4F8B83800223A
:10172000227103B030BD0022274B6271E0E72849E7
:1017300001EB820191ED187A29790029BDD0531F60
:10174000032BCFD9002ACDD02AE000219A42A4F859
:10175000F2149DD3A4F8EC149AE767EE877ABCEEF6
:10176000E77A8DED017A9DF8043007EE103AB8EE75
:10177000C77AF4EEC77AF1EE10FAC4BF0133DBB2D8
:10178000D3B1102BA8BF1023DBB2934238BF13464E
:1017900084F8AC38A6E7053A032AA3D99FED097A65
:1017A000B7EE000A80EE070A4CF086FF2B888342D2
:1017B00028BF03462B8095E70123E5E7A8A5002075
:1017C000303E00206F12033864A60020E4A60020FB
:1017D000BC0606082DE9F04F9B4E83B096F8BC3846
:1017E000A3F11702022A00AF00F28F82974B7B60B1
:1017F00096F8CC383B60964BDFF86CA203F16C098D
:10180000984600241FE098F90420142A00F07882FA
:1018100058464DF039FD1BF4003F21D0012800F05F
:101820006F82082800F36C8215B11BEA0A0F06D1FB
:10183000396858464AF032FA002800F0618208F10F
:101840000C08C14512D0D8F800B01BF00105DAD061
:1018500058464DF019FD01341BF4003FE4B2DDD1D0
:101860000128DEDC08F10C08C145ECD1013C022C5A
:1018700000F246820023022086F868390EF0E4FF69
:1018800096F87039D6F86C59022B00F0CD820028FA
:1018900000F019836F4B96F8CDA903F56A794FF4E0
:1018A0007A7E4FF0000C4FF0640B33F8082CB2F541
:1018B0007A7FB3F8462088BF23F808ECB2F57A7F28
:1018C00033F8062C88BFA3F846E0B2F57A7F33F8E8
:1018D000042C88BF23F806EC33F8061CB2F57A7F97
:1018E00084BF002223F804CC9142B3F85A10B3F815
:1018F0005C2098BF23F806CC914293F86B2088BFF8
:10190000A3F85AC0013A632A93F86C2088BF83F881
:101910006BB00132D2B2092A88BF83F86CC003F1E0
:101920006501002213F8320011F8014F01328442A0
:1019300038BF81F800C0032AF4D1BAF1010F18BFF3
:1019400083F886C0EA339945AFD1DFF8209199F842
:101950000230042B00F0958243B9B9F80030B3F59A
:10196000F07F84BF4FF4F073A9F80030FFF752FE08
:10197000394896F8E019FEF7D7FD96F8FF191030B0
:10198000FEF7D2FDB6F80E2AB6F80C3A1343B6F8B5
:10199000102A13431BB213B10123A6F8123A2F4B9E
:1019A0002B40002B00F0A582E90700F14D826A046C
:1019B00000F1BD812B0740F12582294AD6F8C039B4
:1019C00015401340C6F86C59C6F8C03915F40043E9
:1019D00000F0E081002386F8D33886F8E338E80485
:1019E00040F1E28196F81F3ADFF878A0022B04BF9D
:1019F000012386F81F3A0AF17804534602E00633C1
:101A00009C420CD01A780A2AF9D19978DA78914256
:101A100002D35A79002AF2D00A2023F00BFF0023C8
:101A20004FF4806086F868390EF00EFF002800F051
:101A30003D820C4DAB469BF8051021B39BF800008E
:101A4000F8B1534617E000BFA8A50020BC06060861
:101A5000A0AE0020EEA6002098AF00200960000292
:101A6000FE9FFFFDCCAF0020BC020200303E0020F4
:101A700006339C4207D01A788A42F9D15A79002A53
:101A8000F6D023F0D7FE0BF1060B5C45D3D199F8C5
:101A900002A0BAF1080F00F0BA8196F8CD3996F895
:101AA000E524A3F10103B3FA83F35B0986F89C3ABA
:101AB00096F8CE39A3F10103B3FA83F3032A4FEA70
:101AC000531388BF002286F8A23AD6F8C03988BFDF
:101AD00086F8E524BD4AC3F3C03186F89F1A03EAAD
:101AE0000201D6F86C39C6F8C0191A40F37CC6F862
:101AF0006C29002B00F0B481B6F8B83A002B40F006
:101B0000A581D6F8BC3AB3F5000F24BF0023C6F870
:101B1000BC3AD6F8C43A23F4007323F002031BB195
:101B200040F20223C6F8C43A96F8C03A96F8C88A3A
:101B3000013B042B88BF0123AAF1050A88BF86F860
:101B4000C03ABAF1030F40F21B81B8F1000F1CD06C
:101B500000233B60DFF8A0A206E0ABF1060BABEB85
:101B6000090BD84540F2E580D3461AF8010F00284A
:101B7000F3D00BF0D7FF0028EFD081798B07ECD59D
:101B80003A680123002A40F0D98099F8063013B151
:101B9000002389F80630B6F8263C03F00F02042A29
:101BA00003D8C3F30313022B03D94FF42063A6F821
:101BB000263CB6F8283C03F00F02042A03D8C3F3EE
:101BC0000313022B03D940F60123A6F8283C96F80C
:101BD000951C96F8A12C96F8943C914205D90022C8
:101BE00086F8952C53B1A6F8982C96F8A02C9A421A
:101BF00004D2002386F8943CA6F8983C96F88A3DD7
:101C000096F8962CDFF8F4C19A4284BF002386F838
:101C1000963C0CF1800B6346796813F8032D02EBB8
:101C200042020A4492F85CA192F85D9192F85EE15A
:101C300013F8010F9979DA785045A8BF5046494505
:101C4000A8BF49467245A8BF72466345187099718E
:101C5000DA70EDD103F1200CDC45DCD1D6F8F028A8
:101C6000002A00F00581002001212B782B2B07D1C1
:101C70006B78043301FA03F313421CBF9A4301202B
:101C80000635AC42F1D108B1C6F8F028504C6D468B
:101C900004F10808234601E043455DD013F8012F05
:101CA000072AF9D9002304F8013F0133082BFAD1A0
:101CB000B6F8C629B6F8C4399A42AD4602D3454BA8
:101CC000C6F8C439444B454CFF2286F8BC2D03F1BD
:101CD0006C0013F9082C142A05D053F80C1C34EAB4
:101CE000010100F0CB800C339842F2D13C4B5A7981
:101CF000022A01D100225A710C37BD46BDE8F08F8F
:101D00003849394843F092F8B4E5384A7A6002EB32
:101D1000C30393F87C20002A3FF46AADD3F88030E7
:101D2000002B7FF465AD172386F8BC3860E5304A98
:101D300044E63A680023002A3FF427AF99F81120BF
:101D4000002A7FF428AF99F80520012A3FF41DAF3F
:101D5000002B7FF41AAF1EE788B0E9462022FF214E
:101D600048464DF0FDF91A4A03E0424549F8233050
:101D70009ED012F8013F59F823100131F5D091E7B8
:101D8000002389F80430B8F1000F00F0A780012388
:101D90003B60DFE696F8D328002A3FF420AEE80443
:101DA00086F8E3383FF51EAE29067FF51BAE96F8A0
:101DB000BC28182A04D80F4BD340DA073FF512AEDF
:101DC000DFF83CA00AF1780429E600BF9CD445184E
:101DD000423E0020AE014A01ACAE002001000200EC
:101DE000084E0020A0AE002044020708BC060608EA
:101DF000F6DFFFFD00410001373E002069A600200C
:101E0000CCAF0020AC047FF5E1AD3E4AD6E599F8B1
:101E10000630002B3FF441AE99F81130012B04BF7E
:101E2000022389F8113038E600283FF433AD90F9E9
:101E300004404FF0FF0901E080F8089020460EF0C2
:101E4000F3FC0028F8D125E52F4AB7E596F8B40A47
:101E50000BF068FE00287FF454AEA6F8B80A50E6EE
:101E60002A4B1A430B43C6F86C29C6F8C03943E61F
:101E70002B2023F0DFFCD6F8F028F4E686F8BC2D02
:101E800034E7D6F8C03923F48053C6F8C039B9F81E
:101E9000203025F48055B3F57A7FC6F86C59BFF42D
:101EA00065AD4FF47A73A9F820305FE5D6F86C3948
:101EB00023F00063C6F86C39D6F8C03923F000630C
:101EC000C6F8C039B5E5D6F8C03925F0800523F04D
:101ED0008003C6F86C59C6F8C039DBE499F81130B4
:101EE000002B7FF458AE99F80530012B7FF453AEE8
:101EF0004BE6D6F8C03943F0080345F00805C6F8AC
:101F0000C0395AE5F6BFFFFDF79FFFFD000405004D
:101F10002DE9F04F714F724ED7F8CC3DDFF8D891D4
:101F200003F2DC534E4583B0C7F8CC3D80F0D3803C
:101F3000012301936B4BDFF8C4B106F11C0503F1DB
:101F40000208684B5988002900F0B08008EB0102B4
:101F50005A4580F0AB80444608E0118814460A4494
:101F6000002900F0A3805A4580F0A080052940F2A6
:101F70009D8035F81C3C6188C3F30B039942ECD17A
:101F800063799B07E9D155F8141C238894F804A0C1
:101F90000093304642F04AFF35F81C1CBAEB113F63
:101FA00000F08A800023019335F8181C55F8140CB2
:101FB00055F8044CC1F30B0146F0B4FD1C364E45F8
:101FC000206005F11C05BCD3D7F86C39464CC7F826
:101FD000C039FFF7FFFB3B797979444DEA2203FBD7
:101FE0000242A4F1800303EB4113C7F8B828C7F8F5
:101FF000B4381FF053FF4FF0FF33D7F8B8086B60C9
:102000002DF06EF823F05EFC04F6E80304F516618B
:1020100002E00633994259D01A78002AF9D19C7807
:10202000D878844202D358790028F2D097F81C3A25
:102030002A72B7F8202A642103EB830301FB02F222
:1020400003EB83039B00642A2949B8BF6422642BF5
:10205000B8BF6423C7F8C43DC7F8C82DC7F8E02D42
:102060000023A1F56D7287F8E43D87F8E63DC7F8D7
:10207000102E00230022C1E90423C1E906232EF01B
:1020800023F9B7F8180E97F81A1E26F037F838F02B
:102090001BFE16F0B5F9174A01981268C7F8CC2D47
:1020A000012387F8E53D03B0BDE8F08F55F8141C17
:1020B000304642F0BBFE75E7009BA11D9A1F3046DB
:1020C00042F0EAFE00287FF46FAF6BE73A7D003AFA
:1020D00018BF0122AAE70123019375E7A8A50020F4
:1020E0009C01070800400008E4A600205C040020D2
:1020F00068B30020A0180020D0090708008000085D
:1021000038B50122184D84180328034685F81C2E83
:10211000E4B217D9FF2824D0144A002341F2024127
:1021200000E034B10233402B22F8021B04F1FF34EB
:10213000F7D11D44FF2385F8203EBDE838400E202E
:102140000EF098BCEA2205F59E7003FB02002B718D
:10215000C5F8B8082CF0C4FF2AF06AF82AF04CF948
:10216000DAE70023E5E700BFA8A50020C8B30020F8
:10217000054BD3F8642E012142F4001283F8611E4E
:10218000C3F8642E704700BFA8A500202DE9F843CE
:102190000468C4F30A0906460F4604F17848B9F109
:1021A000000F16D0B8F5002F3B6834D2314D2A69A4
:1021B00042F001022A614FF48010236043F07AF963
:1021C0002B6923F001032B6103282BD06FF0020051
:1021D0002CE0B8F5002F16D2264D2B6943F00203F0
:1021E0002B616C612B6943F040032B614FF0004081
:1021F00043F060F92B6969F341032B610328D1D0C7
:102200004FF0FF3012E004F1774303F57803B3F5A4
:10221000002F0DD30B6804F1774202F57802B2F576
:10222000002F18D33368043333600020BDE8F883EF
:10223000104D2B6D43F002032B656C652B6D43F045
:1022400040032B654FF0004043F05EF92B6D69F3BE
:1022500041032B65D2E7074D2A6D42F001022A6542
:102260004FF48010236043F04FF92B6D23F00103EE
:102270002B65A9E7003C02402DE9F0435C4F3B7819
:10228000B12B8BB062D1FEF769F880F00104E4B2A3
:10229000584B594DB3F86B31DFF87081ADF804300D
:1022A00004F00104454553D3002C00F09F80534BAC
:1022B0005349544A0597DB1B0693534B4E4D00265A
:1022C0000996CDE9076659605A6059645A6401223B
:1022D0008DF825203422DA6001A9022205A88DF8A4
:1022E000246049F0D5FF022201A94FF6FF70FDF7E7
:1022F000DDFD0446454538D3022202A905A8002584
:10230000ADF8085049F0C4FF022202A92046FDF7AB
:10231000CDFD40BAC043ADF80C00022205A803A9C8
:1023200049F0B6FF0898002849D1374B1A6942F0A6
:1023300080021A611A6D42F080021A659DF924002C
:10234000B0FA80F040090BB0BDE8F08301249FE7AC
:10235000A988AB69A8681E68C1F30B0146F0E2FBCF
:102360001C35864218BF01249CE7AF888DF81160A8
:10237000C7F30B07BB1DADF80C302B88C3F30B0262
:10238000ADF80E201B0B062203A905A88DF810300E
:1023900049F07EFF062203A92046FDF787FDD5F808
:1023A000089004463A46494605A849F071FF204680
:1023B0003A464946FDF77AFD1C3504469AE707ABD5
:1023C000C0F10402294618444CF0CAFE9DF92400CD
:1023D00018B907A905A8FFF7D9FE002308939DF8AF
:1023E00025308DF82400002BA8D09EE70120AAE715
:1023F00000400008BC0606089C0107080080000891
:1024000023016745AB89EFCD003C0240D0090708A6
:1024100070B5194D194EFFF7DDF9D5F8CC3D012205
:1024200003F2DC53C5F8CC3D85F8682E0324FFF792
:1024300023FF58B13378B12B08D1FDF78FFF013C52
:102440000BD060B9FFF718FF0028F3D1013CEED1A3
:10245000052048F0A1FB47F00BFD0028F8D0084A02
:102460001168C5F8CC1D0122002385F8E52D85F8FB
:10247000683E85F8693E70BDA8A5002000400008B0
:10248000A018002010B50A4C012384F81C3EE37408
:10249000FFF7BEFFFFF73CFD41F20242FF23A4F825
:1024A000202E84F8223EBDE810400E200EF0E2BA45
:1024B000A8A5002090F89230DFED6B6A6B4A07EE1A
:1024C000903A90F8963005EE103A90F8943004EE79
:1024D000903A90F8953005EE903A90F89830F8EEF2
:1024E000E77AB8EEC55A04EE103A67EEA67A25EE02
:1024F000265AF8EEE44AF8EEE55AB8EEC44A25EE5C
:10250000275A64EEA64A65EEA65A24EE264AF0B58E
:10251000B7EE007A90F8917064EE854A65EEA75A9E
:1025200024EE274A00F16F06014602F11805002447
:10253000B0EE476AB0EE473A137807EE903AF8EEFD
:10254000E77A67EE857A67EE867AFDEEE77A17EE30
:10255000903AFA2BA8BFFA2323EAE3730B7253785D
:1025600007EE903AF8EEE77A67EEA47A67EE867A9D
:10257000FDEEE77A17EE903AFA2BA8BFFA2323EA8A
:10258000E3734B72937803EE903AF8EEE33A63EE1E
:10259000A57A67EE877AFDEEE77A17EE903AFA2B86
:1025A000A8BFFA2323EAE3738B72938807EE903A6D
:1025B000F8EEE77A67EE847A67EE867AFDEEE77AE0
:1025C00017EE903AB3F57A7FA8BF4FF47A7323EAF7
:1025D000E3738B812B68D5ED007A002BF8EEE77A58
:1025E0003FDD90F8973002EE903AF8EEE22AB0EE36
:1025F000436AA2EEE66A63EE863A83EEA76AA2EE2B
:10260000A66A013465EEA77A67EE877A67EE867A66
:10261000FDEEE77A17EE903AFA2BA8BFFA2323EAE9
:10262000E373BC4206F8013F00DDF0BD012C13D17D
:1026300090F8933007EE103A90F89B3006EE103A7F
:10264000B8EEC77AB8EEC66A27EE267A26EE266A74
:102650000435083208316FE7B7EE007AB0EE476A0A
:10266000F6E7B7EE006ACCE70AD7233CA00B0608D2
:1026700090F899306BB3B0F864308BB190F89A2031
:1026800002EB82036421C3EB0313B3FBF1F3A0F865
:102690006430962312FB03F3B3FBF1F3A0F866302A
:1026A00043884BB190F89A3003EB8303C3EB0313D9
:1026B0006422B3FBF2F34380B0F850304BB190F892
:1026C0009A30962213FB02F36422B3FBF2F3A0F8D4
:1026D0005030704790F821304BB3438B83B190F862
:1026E0002230FA2213FB02F203EB8303B3F57A7F65
:1026F000A8BF4FF47A7364218383B2FBF1F2428363
:10270000838843B190F82230FA2213FB02F364224B
:10271000B3FBF2F38380C3884BB190F8223003EB14
:102720008303B3F57A7FA8BF4FF47A73C3807047F1
:1027300070B50B4C002504F56A7694F8913013B10E
:102740002046FFF7B7FE2046FFF792FF01353046DF
:10275000FFF7C0FF042D04F1EA04EED170BD00BF05
:10276000E4A6002010B5064C4FF48072002104F559
:10277000D5604CF0F5FC0023C4F8A83710BD00BFAD
:10278000A0B60020034BD3F8AC0708B10AF07CBC1C
:10279000704700BFA0B6002008B50B4605490246A9
:1027A000D1F8AC0728B10449FEF7F2FABDE80840B9
:1027B000E8E708BDA0B600203D060108024B01462F
:1027C000D3F8AC07FDF73CBFA0B600200048F5E702
:1027D0002BED06080CB4C30607B500D561B9049803
:1027E00005A90191FFF7D8FFFFF7F0FF012003B023
:1027F0005DF804EB02B070470020F8E708B5FFF77A
:10280000DDFFBDE80840E1E710B504460348FFF7E7
:10281000D5FF2046BDE81040F0E700BF76E106088E
:1028200010B508460749FDF72FFC002815BF012405
:10283000002405480548FFF7E7FF2046BDE81040A3
:1028400009F070BE7BE1060884E10608ABE10608EA
:10285000034B0146D3F8AC0708B10AF001BC70473E
:10286000A0B600200CB407B510F020000BD079B949
:102870002320FFF7EDFF049805A90191FFF78CFFD6
:10288000FFF7A4FF012003B05DF804EB02B070472E
:102890000020F8E70FB407B504A951F8040B019123
:1028A000FFF77AFF03B05DF804EB04B07047194BF3
:1028B0001B682DE9F0415BB31748184FDFF86480BF
:1028C000FFF79CFFFFF75EFFFCF78CFD0025FCF790
:1028D000C9FD044640B113200EF0CCF8FFF776FF97
:1028E000BDE8F0410E4889E73B78012BF3D0404624
:1028F000FFF7D0FF792D05F1010602D1FFF766FF42
:102900002646FFF73FFF6420F7F714FB3546DEE766
:10291000BDE8F081CC2C0020C7E10608A24F0020C2
:10292000E1E106084DFB060838B50B4D05EBC00587
:102930000C4695F908050AF0E5FF01460748FFF740
:10294000A9FF95F80E352BB1611C0548BDE838404C
:10295000C9B29FE738BD00BFBC060608D8F8060814
:1029600010E206080FB407B504A951F8040B019151
:10297000FFF712FFFFF72AFF03B05DF804EB04B086
:1029800070472DE9F041037903F0E002402A4AD074
:1029900009D82ABB03F00703052B1CD8DFE803F096
:1029A000161B161B090F602A44D0802A3ED0BDE8B2
:1029B000F081D0F805102148BDE8F041D2E7D0F809
:1029C000052051421E48BDE8F041CBE7B0F8072092
:1029D000B0F80510F6E7B0F90720B0F90510F1E7F7
:1029E0004679184D184805EBC605FFF7E7FE95F840
:1029F0001C7600240123A74202D8BDE8F041E5E699
:102A0000D5F8186656F824204FEA84084AB113B95D
:102A10000E48FFF7D3FE56F808100D48FFF73AFFAF
:102A200000230134E7E741790A48C5E78279417913
:102A30000948C8E7BDE8F041084893E7E7E1060820
:102A4000FDE10608BC06060814E2060868E406086C
:102A5000D8F8060825E2060836E206084DE2060820
:102A60002DE9F04385B0FCF7ADFC0269838901884C
:102A70000292826801924288009242681B4EDFF8FF
:102A80008080DFF880901A4F04461A48FFF76AFFEB
:102A9000002515B91848FFF7B1FED8F800309D425F
:102AA00013DA3378052B96BF09EB83030022D3F8A2
:102AB000D027B38800937388294638460135FFF73D
:102AC00051FF062D06F10606E3D146F029FC4288A7
:102AD000838864689B1A03FB0444FCF70BFD0246E1
:102AE0000648214605B0BDE8F0433BE750BE002054
:102AF000CFE2060865E20608C3E20608DEE2060841
:102B0000984F0020BC0606080249034801F5FD6104
:102B10000EC927E700F0FF1FFBE2060870B5134C53
:102B2000134D144E002294F8073503F0010302B14F
:102B300070BD002BFCD001212846FFF713FF752044
:102B40002DF05EFE01463046FFF70CFF1A202DF0F7
:102B500057FE01460848FFF705FF1B202DF050FEE9
:102B600001460648FFF7FEFE0122DCE7A8A500208B
:102B70000FE306081BE306082EE3060841E30608F8
:102B80002DE9F04FBE4BBF4C1A68BF49BF4BC04840
:102B9000B2FBF3F291B0FFF77DFEB4F8D427BD4D40
:102BA000BD4EDFF89893DFF898A3DFF878B34FF4C1
:102BB0007A73B2FBF3F103FB11220A20B4F9D63782
:102BC00092B2B2FBF0F2B548FFF7CCFEB44AB54979
:102BD000B548FFF75FFEFFF7F9FDE97CB34AB44B58
:102BE000B44806EB8101D31AD1F8E8172A88FFF719
:102BF000B9FEFFF7EBFDB048FFF7E0FD94F8D817FA
:102C0000AE48FFF747FEAE48FFF7D8FDAD4B94F84E
:102C1000D9171A88AC4892B2FFF73CFEFFF7D6FDF1
:102C2000AA49AB48FFF736FE4FF00008474695F833
:102C3000033503F00103B8F1000F00F0E980002F25
:102C400040F01B81A348FFF7D9FDDFF8F882D4F8E4
:102C5000E097DFF8F4A2012708F1180B0123BB402D
:102C600013EA090F14D01AF8072058F827305BF838
:102C7000271053F822209848FFF70CFE012F05D1AA
:102C800094F8011811B19548FFF704FEFFF79EFD77
:102C90000137062FE2D19248FFF790FDD5F8C039F1
:102CA0001B0640F1848194F86C38032B8CBF8D484F
:102CB0008D48FFF783FD95F87039022B40F046816F
:102CC0008A48FFF77BFD94F86C38042B00F266818C
:102CD0008748FFF773FD94F87C38002B00F065817E
:102CE00006EBC303D3F8C4188248FFF7D3FDFFF700
:102CF0006DFD94F8EB35D4F8EC757F4806EB830353
:102D0000D3F8F818FFF7C6FD27B13A7A797A7B48ED
:102D1000FFF7C0FDFFF75AFDFCF754FB016921B135
:102D200082687748120DFFF71DFEFFF74FFD754BC8
:102D3000754819684FF47A73B1FBF3F1FFF7AAFDF8
:102D400005A8FEF713FC38B105A908A849F064FEF0
:102D50006E4808A9FFF79EFDFFF738FDD4F80889F3
:102D6000B8F1000F00F0278107EE908ADFED686A66
:102D7000B8EEE77AC6EE877AFDEEE77A17EE903A7C
:102D8000644F17F8F80C30B1634A039392ED090AC7
:102D90004BF092FC039BD4F888485CB107EE904A54
:102DA000DFED5B6AF8EEE77A86EEA77AFDEEC77A8A
:102DB00017EE904A37F8F61C6429A8BF6421CDE9C4
:102DC000000442465548FFF7CDFD37F8F42C54482F
:102DD0006423B2FBF3F103FB112217F8E33C06EB8B
:102DE000830692B2D6F80C39009317F8E43C4D4EA6
:102DF000FFF7B8FD4C48FFF7E1FCD5F8644E01251C
:102E0000002C40F0DA80FFF7E1FC11B0BDE8F08F54
:102E1000002B3FF414AF17B14846FFF7CFFC012158
:102E20005046FFF737FD94F8DC3706EB830358462E
:102E3000D3F8F017FFF72EFD95F88638DA0702D59C
:102E40003A48FFF727FD95F8D035032B09D03848CD
:102E5000FFF720FD95F8D035012B02D13548FFF75B
:102E600019FDD5F854355B7B0127BB42B8467FF688
:102E7000DEAE3148FFF70EFDD9E6FFF7A7FCE4E62A
:102E800044030020A0B600205CE3060840420F0087
:102E900066E30608A8A50020BC06060878E3060835
:102EA000F0FF0220000800009AE3060800800008F6
:102EB00000400008ACE30608C3E30608D5E30608B3
:102EC000DDE30608144E0020DFE30608F3E30608FE
:102ED000F8E3060817E4060846F506081CE40608A9
:102EE00020E4060826E4060832E4060842E4060860
:102EF0005EFC060886E40608A2E40608ABE40608C1
:102F0000B5E40608A0180020D0E40608EAE40608A4
:102F10000024744998C700205C040020FDE40608E2
:102F200043E5060892E4060868E50608C6F80608C0
:102F300002E406080AE406080FE4060868E4060846
:102F4000FDE306080C0F06087804002002200DF0AF
:102F50009BFC074608B92048B3E690F9040044F00A
:102F60009BFB804637F09AFE06EB80004146D0F886
:102F700080281A48FFF78EFC95F87339012B04D18D
:102F80001748FFF71BFC17489BE6BB79164806EB72
:102F90008303D3F88018FFF77DFCF4E795F87239C6
:102FA0000BB9124895E6124893E612499CE612487E
:102FB000FFF704FC9BE64346E2E694FAA4F0B0FA7D
:102FC00080F005FA00F024EA00040DF0A7FB0146AA
:102FD0003046FFF75FFC13E748E4060852E40608B2
:102FE00062E4060867E406089BEF06086BE406083F
:102FF0007BE4060854E3060896E406082DE9F04F42
:10300000DFF8708198F8073099B0002B00F09480B9
:103010004F48504EDFF860B1DFF86091DFF860A1F3
:10302000FFF7ECFB00252F460BA9E8B215F064FC76
:103030009DF83430002B53D0139C54B107EE904AC6
:103040009FED450AF8EE677A80EE270A4BF034FBD5
:1030500004460B9A29465846FFF71CFC109A002A92
:103060006CD002FB04F04FF47A73B0FBF3F30993D6
:10307000DDF848C0BCF1000F62D00CFB04F142F255
:103080001073B1FBF3F198F80730082D18BF7F18C3
:10309000002B57D017980790159806901698059012
:1030A0000A2311984FF47A7EB0FBFEFE0998CDF802
:1030B00010E0B1FBF3FE03FB1E11CDE902E109991B
:1030C000B1FBF3F103FB1100CDE90010BCFBF3F3FE
:1030D00021465046FFF746FC0023C6E90D33B36294
:1030E00001351E2D06F140069ED198F8073003B336
:1030F0001A4C1B4854E938124FF47A73D208B1FBCA
:10310000F3F354F8D81CFFF72DFC0A22154897FB5F
:10311000F2F102FB1172FFF725FC134B1B78432BD6
:1031200004D154E935211148FFF71CFC002344F871
:10313000D83C19B0BDE8F08F0D486AE7099297E7CF
:103140006146A0E721464846FFF70CFCC4E700BFF4
:103150007EE5060820BF00208096184B98C7002007
:1031600025E6060845E60608A035002069E60608BB
:10317000DCE50608A8A50020E6E5060874F80608C0
:10318000F5E5060870B5224C2248FFF717FB14F846
:10319000F83C002B37D0204B93ED090A4BF08CFA0A
:1031A00001461E48FFF7DEFB1D4D1E48FFF706FBDC
:1031B0001D4B95F8E5081D4A00280CBF104618461F
:1031C000FFF71CFB95F8E5380BB334F83A1C1848A8
:1031D000184E194DFFF75EFB14F83C0C00280CBF8D
:1031E00030462846FFF70AFB34F8381C1348FFF72F
:1031F00051FB14F83B0C00280CBF30462846BDE8B4
:103200007040FFF7FBBA0E48FFF7F8FACCE770BD45
:1032100098C70020A3E606085C040020BDE6060867
:10322000A8A50020CCE6060862E206089900070877
:10323000DDE606089CE6060893E6060804E70608AD
:10324000C2E606080EB403B503AA52F8041B0192A5
:10325000FDF7C1FE064BD3F8AC3723B9054B064941
:10326000D86DFDF7EDF902B05DF804EB03B07047DF
:10327000A0B60020A8A500202BED06082DE9F047F8
:1032800098460B7903F0E005402D81460F4616461F
:1032900032D1644DDFF8A881DFF8B091002416E048
:1032A0003B7903F00703013B042B04D8DFE803F06C
:1032B00014171A1D2100315D5A48FFF7EBFA7B798C
:1032C000013BA34202DD4846FFF778FA01347B79DF
:1032D000A342E5DCBDE8F08731572846EDE736F834
:1032E0001410FAE736F91410F7E756F824104046A0
:1032F000E3E756F82410F0E703F00703052B57D84F
:10330000DFE803F0031F27292C3E3478602D55D0C9
:103310002CD8002D75D1B7F80550B7F80760414893
:103320002146FFF7B7FAAC4239DBB44237DCB8F1DB
:10333000000FCFD0324629463B48BDE8F047FFF7A3
:10334000A9BA96F90040602D38D00FD8002D58D179
:1033500051E03488DAE7B6F90040F4E7D6F800A087
:10336000202D54464DD034D9602D27D0802DB1D199
:1033700032782E4B2E48002A14BF3146194635E0CC
:10338000202D34683DD0EFD821462648FFF782FA39
:10339000D7F80510A14202DB4B42A34221DDFFF723
:1033A00015FA3A68234923464846BDE8F04749E7FD
:1033B000202D25D01ED9602DD8D100247B7944FA48
:1033C00003F3DB07BDE8F0474CBF1B481B48FFF782
:1033D00061BA51461A48FFF75DFAD7F805108A45D9
:1033E000DDD8B8F1000F3FF475AF1648BDE8F047DF
:1033F000FFF750BA0024B7F90550B7F907608EE718
:1034000000247A79104B03EBC20393F81C26A242E6
:10341000C5DDD3F8183653F82400BDE8F047FFF7B0
:10342000CDB900BF11E2060872E006082EFC0608BE
:10343000D8F806082AE7060862E206089900070895
:10344000FAE1060824E70608BC060608DDE30608DC
:1034500070B50546084616460C46FDF701F9334699
:10346000024621462846BDE8704007E70EB403B582
:1034700003AA52F8041B0192FDF7ADFD044B054968
:10348000D86DFDF7DDF802B05DF804EB03B07047CE
:10349000A8A500202BED06080049E7E744E7060849
:1034A00038B50C46054615492046FCF7EDFD30B908
:1034B000FFF73EF91248BDE83840FFF79FB91149C0
:1034C0002046FCF7E1FDA0B90F4B83F8CD0183F84E
:1034D000D50183F8B70283F8BF0283F8A10383F80C
:1034E000A90383F88B0483F8930483F80505074840
:1034F000E1E72846BDE83840CEE700BF53E70608BD
:1035000059E7060874E70608A8A500207CE7060826
:103510000049ABE798E70608F8B5064608460C46AA
:10352000FDF758FF2021054620464BF030FE0446AB
:1035300018B93046BDE8F840EAE7124F124E3B7822
:1035400032789A4204F1010401D0FCF7C7F80F4B1E
:1035500020461D6049F09EFD012201462046FCF7F1
:1035600065F83B7832789A4201D0FCF7B7F82046EC
:1035700049F090FD2A460146BDE8F8400448FFF7AF
:10358000F1B900BFC82C0020A34F0020C42C00209C
:10359000AFE706082DE9F041064688B008460D461B
:1035A000FDF718FF2021044628464BF0F0FD20B916
:1035B000304608B0BDE8F041AAE7FDF70BFF224610
:1035C000054601460F48FFF7CDF985B1202D2A4663
:1035D000694628BF20222046FCF7C8F8E846064680
:1035E0000027B74208DBAD1B3444002EEDD1FFF7B6
:1035F000EDF808B0BDE8F08118F8010BFFF728F9E5
:103600000137EEE7C5E706082DE9FF4707460846FC
:103610000D4649F03FFD082845D105F1FF3801AEC0
:10362000073531464246B14612F8010FFDF7F0FD6D
:10363000AA4201F8010BF7D10023DFF87CA08DF836
:103640000C30A84517D11B4948462CF08FFD19486E
:103650001949082310F8012B11F8014B10326A4464
:10366000013B02F80C4CF5D114488DF80C3001A93F
:10367000FFF778F914E018F8010FFDF7C9FD06F817
:10368000010B0446014650464BF081FD28B121460E
:1036900030464BF07CFD0028D3D03846FFF7FCFEC7
:1036A00004B0BDE8F0870028D1D0384604B0BDE8AA
:1036B000F0472DE76CAE0020C0800608DDE7060865
:1036C00007B5009313460A460249FFF7CFFE03B041
:1036D0005DF804FBE4E7060810B504460748FFF769
:1036E0008DF8FCF749FB20B1BDE810400448FFF716
:1036F00085B820460349BDE81040B7E6FDE7060857
:1037000007E806080FE806082DE9F041144BD3F846
:10371000E43288B00446F3B11A6804A9D56A1846A1
:103720006A46A847064688B1DFF8408004AC6D467B
:10373000002735F8022B34F8021B40460137FFF70B
:1037400011F9BE42F5DC08B0BDE8F081054920461C
:10375000FFF78CFEF7E7044908B0BDE8F04185E6C5
:10376000A0B6002030E8060848E8060816E8060873
:1037700070B5054608460C4649F08CFC024668B117
:10378000102804D1084821464BF027FD30B12846C7
:10379000054B064A0649BDE8704067E6BDE8704043
:1037A00001490448FFF7DEB84FE8060860E806085C
:1037B0006BE8060895E8060870B5054608460C460D
:1037C00049F068FC024668B1042804D10848214643
:1037D0004BF003FD30B12846054B064A0649BDE8CB
:1037E000704043E6BDE8704001490448FFF7BAB8AD
:1037F000A3E80608A8E806086BE80608B8E8060883
:103800002DE9F04307469BB008460C4649F042FCC0
:1038100020220646002101A84BF0A2FC2EB3402E28
:1038200007D03B494023324638461BB0BDE8F04341
:103830001CE601AD04F140084FF0000902222146C8
:1038400068464BF0DCFC0023102209A968468DF87D
:103850000290FDF71FFD099B0DF10202934223D157
:103860000234A04505F8010BE8D109AC4122002142
:1038700020464BF075FC274D002E3CD015F82C6CE3
:10388000D6B12022A5F12B0101A84BF0EDFC98B197
:10389000A5F12B012046FDF72FFC1F4A1F492346A7
:1038A0003846FFF7E3FD04E01A781D493846FFF774
:1038B000DDFD1BB0BDE8F0831A4B93F83830D3B967
:1038C000CEB9194E01AB1A4603CAA24230607160EC
:1038D000134606F10806F6D101232046124905F8E1
:1038E0000B3CFDF709FC1148FEF78EFF10482146FE
:1038F000FFF738F8DDE715F80B3C1BB915F82C3C41
:10390000002BF3D008492046FDF7F6FBEEE700BF99
:10391000CBE8060898C7002009E906086BE8060806
:10392000EDE80608A8A500206DC7002013E90608E9
:1039300022E906082DE9F74F834608460C4649F070
:10394000A9FBDFF818810646D8F86C7928B1024641
:1039500033492046FDF762FC80B93946314843F0CF
:103960001BFE3149314821EA070143F015FE304979
:10397000304803B0BDE8F04F43F00EBE23782D2B46
:103980002D4B03BF013406F1FF364FF0010A4FF013
:10399000000A4FF000094FF0FF3553F8041B51B1F6
:1039A000324620460193FDF739FC019B00280ABFEF
:1039B0004D460021012109F1010989B9B9F11D0F15
:1039C000EBD11E492246584603B0BDE8F04F4DE505
:1039D0003B43C8F86C391A491A4B12E01A4913E0F4
:1039E000114A0123AB401A40002AF7D007EA03022C
:1039F000BAF1000FECD027EA0303C8F86C39134979
:103A0000134B002A18BF1946124B134803EB8503CA
:103A1000D3F8202903B0BDE8F04FFEF7A3BF00BFE5
:103A2000E1E506085AE906089CD4451864E9060849
:103A3000632BBAE770E90608DC0F06087EE9060882
:103A400052E906084BE906082FE906083BE9060893
:103A500042E90608BC060608D0EF0608A8A5002023
:103A60002DE9F74F019008460E461746984649F053
:103A700011FB0446E8B93F483F4DFEF70BFF2046D7
:103A80000CF064FE3B68184206D020460CF070FE35
:103A900001462846FEF7FEFE0134172CEFD13B68A5
:103AA00013B93648FEF78AFE03B0BDE8F04FFEF7C3
:103AB0008DBE024632493046FDF7B0FB0546A8B937
:103AC0003048FEF77BFE2C462F4D20460CF03EFE84
:103AD00010EA080F06D020460CF04AFE01462846A0
:103AE000FEF7D8FE0134182CEFD1DDE733782D2B0B
:103AF00003BF013604F1FF34012500254FF0000912
:103B000048F4000B48460CF033FE2246824601463C
:103B10003046FDF783FB00BB48460CF017FE1BEA5E
:103B2000000F1AD08DB1B9F1170F1CBF3B6840EAE6
:103B300003081648C7F80080FEF740FE12485146B9
:103B400003B0BDE8F04FFEF70DBFB9F1170F1CBF72
:103B50003D6885433D600E48EEE709F10109B9F182
:103B6000180FCFD10B490198324603B0BDE8F04F92
:103B70007CE400BF8FE9060891E4060899E906088D
:103B8000E1E50608A0E9060892E4060842E906080D
:103B900052E906087EE90608014A40F202235FE77F
:103BA0006CB00020014B024A5AE700BFFFFF7F00C4
:103BB00064B0002010B5044601202CF047FB20B96A
:103BC00020460449BDE8104050E4BDE810400248DA
:103BD000FEF7C8BEABE90608BAE90608064B10B501
:103BE000044653F8080C36F0D1FF20B920460349AB
:103BF000BDE810403AE410BD98C70020C5E90608AA
:103C000070B5054608461646FDF7E4FB0D4B041E4D
:103C100093F8C82A0EDB944205DA0B482146FEF7DA
:103C2000A1FE204670BD2EB1FF2C03D10748FEF740
:103C300099FEF6E70649013A2846FFF717FC4FF0D0
:103C4000FF34EEE7A8A50020DBE90608ECE906084A
:103C5000FFE906082DE9F04F074691B08148824DF3
:103C60000E46FEF77FFE814945F804DC00232B70E9
:103C70000622012391F8C81A304640246C7009F0DE
:103C8000BDF90A20F6F756F92B780C2BDAB240F280
:103C9000E4809DF80C60FE2E2CD0FF2E15BF0F2463
:103CA000152400250125944240F0D780611EC9B239
:103CB00068463CF0FBFB04F140030DEB030414F8F1
:103CC000413C834240F0C4806A1E012A9DF80D30B9
:103CD00012D903F01F0761375C096548FEF76EFDD6
:103CE000022D39D0013C042C34D8DFE804F00B2D30
:103CF0002F3331000225D6E79DF80E709DF80F4056
:103D00001E46EAE75B48DFF8C491DFF8C4A1DFF89C
:103D1000C4B1FEF773FD5848FEF750FD6C464FF0F6
:103D2000000814F8011B484608F10108FEF7B2FD2F
:103D3000B8F10C0F16D00AFB08F3B3F1553FF0D8D9
:103D40005846FEF73BFDECE74C48DCE74C48DAE729
:103D50004C48D8E74C48D6E700238DF83F300DF1AA
:103D60001F00D0E7FEF732FD022D3AD06422B6FBE9
:103D7000F2F102FB11623B464448D2B2C9B2FEF7EF
:103D8000F1FD85F001035B42DBB2012B59D8404ABB
:103D9000404B9DF810104048404E00290CBF114682
:103DA0001946FEF7DFFD9DF811103D4B3D480029F7
:103DB0000CBF31461946FEF7D5FD022D41D19DF8C5
:103DC00012403948FEF7FAFC8CB1FF2C1FD00A23B1
:103DD000B4FBF3F103FB11423448D2B2FEF7C2FD4B
:103DE00008E033483A463146FEF7BCFDCFE730469F
:103DF000FEF704FD9DF813402E48FEF7DFFC44B1AA
:103E0000FF2C21D02C482146FEF7ACFD04E02B48C6
:103E1000EEE72248FEF7F2FC204E214FDFF89C80AF
:103E20000DF11305002415F8013F7BB1FF2B14BFE2
:103E30003A464246214622480134FEF793FD042CBF
:103E4000F1D111B0BDE8F08F1C48E3E73246F1E74D
:103E50001C493846FFF70AFBF3E71B48FEF7CEFC88
:103E6000EFE700BF45EA060898C70020A8A5002094
:103E700056EA060861EA060887EA060868EA0608BC
:103E800070EA060878EA060854E3060899EA060884
:103E90002EEA060825EA0608D0EA060835EA0608EA
:103EA0001CFA0608E7EA0608EEEA060802EB06082E
:103EB000B5EA06080AEB060811E2060839EA060820
:103EC0001AEB060825EB060835EB06086BE1060839
:103ED000ABAAAAAA2EFC06082DE9F843DFF8A890A1
:103EE00007460C46204649F0D5F8064660B91E4BF9
:103EF0001E4893F8BC281E4B03EB8203D3F890199D
:103F0000BDE8F843FEF72EBD024649462046FDF7C0
:103F100085F960B1DFF86480002558F8041BB1B959
:103F2000224638461349BDE8F843FFF79FBA1248C6
:103F3000124C134DFEF742FC54F8041B19B12846ED
:103F4000FEF7A8FCF8E7BDE8F843FEF73FBC3246B1
:103F50002046FDF763F901350028DED1024B094CFC
:103F600083F8BC58BEE700BFA8A500203EEB0608BA
:103F7000BC0606087EE90608A0E9060850100608F7
:103F800092E406082DED0608E1E5060838B50D4671
:103F900004461A4905222846FDF740F968B9184B2E
:103FA00093F8602022B9012183F8601083F8612022
:103FB000BDE838401348FEF721BC134903222846C8
:103FC000FDF72CF9A0B90E4D95F8603063B195F866
:103FD00061304BB10D492046FFF748FA002385F8C0
:103FE000603085F8613038BD0948FEF707FCF5E719
:103FF00020460849BDE83840FFF738BA7AF9060884
:10400000A8A5002048EB0608C5FA06085EEB0608DE
:1040100095EB0608A9EB060870B5184C94F86030CB
:1040200005467BB194F8613063B11549FFF71EFA7C
:1040300028461449FFF71AFA002084F8600084F833
:10404000610070BD104B13F80B2CA2B113F82C2C8F
:104050008AB9A3F12B021D1DA3F10B06106851684C
:104060002C4603C40832B2422546F7D1012283F818
:104070003F200AF0FDFA0120E3E700BFA8A50020D9
:104080005EEB0608B8EB060898C7002008B50346A3
:1040900010460AB9002008BDDB0601D50029FAD078
:1040A000FEF7B2FBF6E7F8B50D4E96F83830054648
:1040B00093B9F8BD25B12388C3F30B039D4204D007
:1040C000D4E90201A2884AF0F3FF1C34BC42F1D3C8
:1040D000002386F83830ECE7024C034FF6E700BFC8
:1040E000A8A500209C010708D00907082DE9F04F7A
:1040F000164685B0CDE901011A4600213046FFF78A
:10410000C5FF314C009006F010034FF00009A246A5
:104110000393FEF737FB2379029A03F018039342C7
:1041200003D0002A44D1182B42D14FF00D0B0BFBCA
:1041300009A3B3F8090040F063FE80462046FCF76F
:1041400088F9D8E902210746024401442046FCF7D9
:1041500039F980F00101009A0546C9B23046FFF7EF
:1041600095FF039B009003B115BB0BFB09FBB30646
:104170005AF80BB00ED56DB914485946FEF78AFBB4
:10418000D8F8082001982B463A442146FFF776F8E4
:10419000FEF71CFB0E485946FEF77CFBD8F80C20B6
:1041A000019800233A442146FFF768F8FEF70EFB1A
:1041B00009F1010940F25623994504F10D04A8D1F3
:1041C00005B0BDE8F08F00BF1C1E0608D6EB060840
:1041D000D7EB060820B10078B0FA80F040097047AC
:1041E000012070472DE9F74F81460846FFF7F2FF9F
:1041F0000E46054670B1002401A9204643F064FA3A
:10420000013401464846FFF7EDFF122CF4D103B00C
:10421000BDE8F08F0846FDF7DDF8C4B2112C71D867
:10422000701C3D4D3D4EFCF774FA05EB44086700E9
:1042300098F840A08346B8B9AAF102014B424B411D
:104240003D4495F84020B25C002B54D095F84130A5
:10425000192040F2EE2100FB03133148214603B040
:10426000BDE8F04FFEF77EBB017830464AF08FFF85
:1042700078B1032C94BF002201222A4902EB4202AA
:10428000831B0A4452FA83F393F804AABAF1030F8A
:1042900005D1484603B0BDE8F04FFFF7FDB85846DA
:1042A000FCF737FAF0B1BAF1020FF2D1FDF792F84C
:1042B00040F6CA0380B29842A8BF184640F2EE23E7
:1042C0009842B8BF1846A0F2EE201923B0FBF3F0D5
:1042D00088F84100AAF1020253425341EA1982F8D8
:1042E00040A0ADE7BAF1020FF4D1484603B0BDE8F3
:1042F000F04FFFF70DB90C48214603B0BDE8F04F71
:10430000FEF730BB094911232A46484603B0BDE8F1
:10431000F04FFFF7D5B900BF98C70020D08206083C
:10432000E1EB0608BC060608F1EB0608FEEB060802
:104330002DE9F04F0346A1B00846FFF74BFF0546B5
:1043400028B1184621B0BDE8F04FFFF7E1B8DFF81B
:10435000C4920B90FF238DF8283059F8083CADF833
:104360003000CDE9050093F838200D908DF8382005
:104370000F90ADF840001193099107464FF0FF38B8
:10438000934909A84AF0A2FE044618BB914F014682
:104390000AAC0B0190481A57002310F9016BB24286
:1043A00040F0D28010464E1C43F076F9314602466A
:1043B0003846FEF7D7FA022E4FF00101E9D19DF9F8
:1043C00038A09DF92830534540F0C5808348FEF75A
:1043D000C9FA4DE02378002BD2D0032FD4BF00269A
:1043E0000126062F00F2A980DFE807F0044750916C
:1043F00004475000042F10D079492046FCF732FFC3
:1044000058B14FF480600CF03FFA002800F0B581FD
:1044100090F90400012306930AE072492046FBF755
:1044200033FE70B959F8083C93F93800042F22D0B4
:10443000119B119320AB03EB061606F8580C0137BD
:104440009EE7204643F018F80028EFDA01230A22FD
:1044500012A92046FCF71EFF40B2002803DB129B86
:104460001B78002BE2D060482246711CFEF77AFAD6
:1044700021B0BDE8F08F0023DBE72046FCF7AAFF60
:1044800020AB03EB061646F8540CD8E757492046F4
:10449000FCF7E8FE5649B0F1000A204618BF4FF07D
:1044A000010AFCF7DFFE08B14AF0020A3301DFF827
:1044B00068C1079320AB03EB0616BCE80F0006F8B3
:1044C00050AC12AE0FC6BCE80F000FC6BCE80F0020
:1044D0000FC69CE8030086E8030000260DF1480A99
:1044E000B346DAF8001020464AF0A8FE10B19AF858
:1044F00004301E430BF1010BBBF1070F0AF1080A50
:10450000EFD1079B80336B4403F84F6C97E7394931
:104510002046FBF7B9FDA0B137492046FBF7B4FDB3
:1045200000288CD02046FCF755FF0328804686D90A
:1045300001463248FEF716FA9AE73148224608212A
:1045400094E7012305937AE70133092B7FF425AF24
:104550002C4801318AE70B9B1BB9AAF11402554282
:10456000554100235F1CE368002B62D194F900B031
:1045700058460CF059F9D4F8049018B10668002E8A
:1045800040F08B80B9F1000F237A14BF4E464FF4F0
:104590006146666023B91C48FEF7E4F903232372E1
:1045A000627A2AB1194807923946FEF7DBF9079A71
:1045B0000292237ACDE9006300231A461946584631
:1045C0000CF09CF9E06048BB11483946B2E700BFE7
:1045D00079E1060888EC0608470A0608A5EC0608F3
:1045E00021EC06082CEC060830EC06084BEC06081B
:1045F00049FA06084EEC06089BE9060854EC060842
:104600006CEC060893EC0608BEEC0608D9EC06082C
:10461000F4EC060898C70020C81006085849594A03
:104620005948B9F1000F18BF0A4633463946FEF71C
:1046300031F9022F04F110044FF0010392D1119EC1
:104640000D9F4DB15148FEF7D9F833681B6A1BB175
:104650004F493A4630469847059B002B50D04D496C
:10466000474BBAF1140F18BF19464B48FEF77AF9B9
:10467000BAF1140F09D1059B002B43D03368DB69D5
:104680001BB14649002230469847069B002B43D178
:1046900000223146384642F007FFE660B9F1000FCC
:1046A0002CD04946304603F091FA3D4AB3683D4864
:1046B0003946FEF757F994F80890B9F1000F0CD07D
:1046C0003279914509D038484B463946FEF74AF9C8
:1046D000336849469B6930469847637A23B17279BB
:1046E00032483946FEF73EF9F36A002BA1D0304834
:1046F0003946FEF737F90023F3629AE7204AD5E7F7
:104700001F49B2E7B8F1000FBFDB3368DB69002B4C
:10471000BBD028494246B6E709F0AEF80520F5F7C8
:1047200009FCDFF89490DFF894A000254FF0030B0C
:104730009AF8C83AAB42ABD919F8014FC4B1204638
:1047400009F0F0F9804698B12046F5F73BFEEBB250
:10475000044610B180F806B0C37120460921F5F770
:10476000E7FD98F80630DB07204603D5F5F70AFF8A
:104770000135DDE7F5F70CFFFAE74FF0FF3049E6CA
:104780002DED060806EC060810ED0608C6ED060835
:10479000CD7B010814EC0608EFED06082D07010893
:1047A0000FEC06082EED060853ED060876ED060818
:1047B000ADED0608B9040108373E0020A8A5002089
:1047C0002DE9F74F05460846FFF704FD0B46044662
:1047D00018B9334A92F864702FB9284603B0BDE87F
:1047E000F04FFEF759BE2F49DFF8C090DFF8C080C8
:1047F000DFF8C0A001AA18464AF095FC264610B979
:1048000009F046F808E056B9012201462846FFF7AC
:10481000F7F9421C04461AD103B0BDE8F08FFCF74B
:10482000D9FD2F28834634D80FB109F025F8BBF104
:10483000060F13D098F8C81A01235FFA8BF2E0B282
:1048400008F0DCFB59465046FEF78CF80027154966
:1048500001AA002001364AF066FCD0E7D8F8C0393A
:104860001B0112D5FF2C0ED0E1B22846FFF7F2F95A
:10487000E8E72846FFF7EEF9013798F8C83AF9B2A9
:104880008B42F6D8DEE70027F7E70748FDF7B6FFCB
:10489000D8E72F2249462846FEF7E8FDD7E700BFB4
:1048A00098C7002079E10608ABE9060823EE060860
:1048B000A8A5002012EE06082DE9F7430746084692
:1048C000FFF788FC0B46044628B1384603B0BDE824
:1048D000F043FEF71DBE2F49DFF8B89001AA184635
:1048E0004AF021FC26460546A04665B92A4B3246C9
:1048F00053F8080CA1B248F07EF968BB2749384646
:10490000FEF7B4FD28E0B8F1000F06D0B8F1010FB2
:1049100025D03846FEF7FCFD1EE0284648F0BAFBDD
:104920001F49064602462846FCF778FC50B31D494D
:1049300032462846FCF772FC30B31B493246284603
:10494000FCF76CFC10B3194932462846FCF766FCAC
:10495000F0B13846FEF7A0FD03B0BDE8F083B31E0A
:104960005A425A4129463846FFF74AF9421C044642
:10497000F2D001AA494600204AF0D5FB08F101080F
:104980000546B2E74646F4E70126F2E70226F0E7DD
:104990000426EEE779E1060898C700204FEE0608E6
:1049A00043EE060846EE060849EE06084CEE0608F9
:1049B0002DE9F74380460846FFF70CFC0B460546F9
:1049C00028B14046FEF7A4FD03B0BDE8F0832F49AF
:1049D000DFF8B89001AA18464AF0A5FB2F46044616
:1049E0002E467CB9022DECD1A7F57A73B3F57A7F08
:1049F00021D927494FF4FA634FF47A724046FEF703
:104A00005FFEE1E74DB1012D10D001AA494600201B
:104A10004AF089FB01350446E3E70122214640467E
:104A2000FFF7EEF8431C0646EFD1CDE72046FCF732
:104A3000D1FC0746E9E7174BD3F89C36B8B25B6860
:104A40009847FF2EBCEEC00A0DD1134BF8EE407A0A
:104A500093F8C82A114BA24213DC10EE101A10482A
:104A6000FDF780FFB0E70F4B0F48F8EE407A03EBFD
:104A7000860310EE102A3146C3ED1A7AFDF772FF55
:104A8000A2E7E3EC017A0134E5E700BF79E106082B
:104A90005DEF0608A0B60020A8A5002000C80020F1
:104AA0007AEE060898C700206DEE0608F8B50746AE
:104AB0000846FFF78FFBC8B11F4B9E6A0136304690
:104AC0000BF056FE34460546F0B90134182CA8BF49
:104AD000002420460BF04CFE0546A8B9B442F4D1A0
:104AE00038461649BDE8F840FEF7C0BC0846FCF75A
:104AF00071FC04460BF03CFE054628B921461048DF
:104B0000BDE8F840FDF72EBF0B4B9C620BF078FF21
:104B10000C482A462146FDF725FF172C09D80A4BD9
:104B20000C2202FB043393F8440ABDE8F8400BF072
:104B3000A1BF0020F9E700BF5C04002089EE060851
:104B40009DEE0608B3EE0608BC06060838B5124D01
:104B500004460846FFF73EFB60B1104B104893F93E
:104B600000104B1C0ABF0F4BC9B21979BDE8384081
:104B7000FDF7F8BE0846FCF72DFC032804D8C0B2A8
:104B8000FDF7BEFA2946E4E720460749BDE838406C
:104B90000322FEF76BBC00BF2DED06085C0400206D
:104BA000CCEE0608A8A50020DCEE060838B5124DAC
:104BB00004460846FFF70EFB60B1104B104893F90E
:104BC00001104B1C0ABF0F4BC9B25979BDE83840E0
:104BD000FDF7C8BE0846FCF7FDFB032804D8C0B2A9
:104BE00012F002F92946E4E720460749BDE83840BB
:104BF0000322FEF73BBC00BF2DED06085C0400203D
:104C0000C8EE0608A8A50020D7EE06082DE9F74F44
:104C1000444BDFF828911A7989F800205A7993F8E3
:104C200038300091054689F801200BB907F098FC4F
:104C300040F020F900263C4CB0460D233A4A00993A
:104C4000734352F803A05046FCF70CFB002841D0F8
:104C5000B8F1000F01DDFDF7B9FD34485146FDF70D
:104C600019FE002221462846FEF7F2FBFDF7AEFDB5
:104C7000237903F01803082B46D0102B49D0204687
:104C8000FDF77FFE284B0D2202FB0633B3F8090027
:104C900040F0B6F88346D8B12046FBF7DAFBDBE9F3
:104CA00002210746024401442046FBF78BFB78B9FA
:104CB000019051461E48FDF7EDFDDBF80810019A02
:104CC00028461346CA192146FEF7D8FAFDF77EFD9D
:104CD00008F10108013640F256239E4204F10D040A
:104CE000ABD10020FFF7DFF9FF2389F8003089F806
:104CF0000130B8F1000F11D1009A0E49284603B0D7
:104D0000BDE8F04FFEF7B2BB0B492846FFF71EFF88
:104D1000B5E709492846FFF749FFB0E703B0BDE80A
:104D2000F08F00BFA8A500201C1E0608DBEB0608BC
:104D3000F7EE06087EE906082DED06085C04002063
:104D40002DE9F74F804608460F4648F0A3F9044680
:104D500020B1012825D13B782A2B22D1A948AA4E7F
:104D6000AA4FFDF74BFD0025B1464FF00D0A04F0A8
:104D700001040AFB05F3384659F80310FDF78AFDD4
:104D8000314622464046FEF763FB0135FDF71EFD26
:104D900040F256239D4206F10D06EAD103B0BDE86C
:104DA000F08F3D2138464AF0F2F9002800F02381C7
:104DB00003469A4613F8012D202AFAD0AAEB070AD7
:104DC0000130054610F8013B202BFAD0DFF838B24D
:104DD0005FFA8AFA4FF000090D2303FB09F35246EC
:104DE0005BF80310009138460BEB0304FCF716FA4E
:104DF000064670BB0099084648F04CF9824528D118
:104E0000277907F0E001402900F0898012D871B3BA
:104E100066797F4A02EBC606002796F81C260092A8
:104E2000BA463B46009ABA4202D9BAF1000F62D0A4
:104E30002BB12DE06029ECD0802900F0A480404601
:104E40007449FEF713FB204603B0BDE8F04FFDF7B1
:104E500098BD09F1010940F256239945BCD16E492C
:104E60003A46404603B0BDE8F04FFEF7FFBA07F000
:104E70000703042B1CD10B460A222846FCF70AFA2A
:104E8000D4F8053083420146D9D32046FBF7FEFB18
:104E90000D2303FB09F961485BF80910FDF7FAFCE3
:104EA00000222146404603B0BDE8F04FFEF7D0BADD
:104EB000052B0DD101230A222846FCF7EBF9D4F883
:104EC000053083420146BADB5B428342B7DCDCE754
:104ED0002846FCF77FFA17F0050F0BBFB4F8052042
:104EE000B4F90520B4F80730B4F907309042014610
:104EF000A5DB9842EAE7D6F8181651F8270060B10A
:104F000029460193FBF7C0F8019B30B9394620468A
:104F10004FF0010AFBF7BAFB5346013782E763798A
:104F2000009307F00707013F009BB342B0DDAA469C
:104F300015F8013B202BFAD02046FBF791FB0546E4
:104F4000042F04D8DFE807F0030E0E141D005046AE
:104F5000FCF740FAA8552C2150464AF018F90136C2
:104F6000451CE1E75046FCF735FA25F81600F2E754
:104F700000230A2200215046FCF78CF945F8260050
:104F8000E9E70123F5E7284648F084F8E37994F847
:104F900005A0A779DB0706460AD52046FBF760FB8C
:104FA0000378014623B1324628464AF016F9E0B9A3
:104FB000DEB1B74219D32046FBF752FB3A46002137
:104FC0004AF0CEF8B2453FF663AF1549324628465F
:104FD0004AF003F900283FF45BAF2046FBF740FBA3
:104FE000324629464AF064F852E70E493A464046AE
:104FF000FEF73CFA23E73946404603B0BDE8F04FE0
:1050000004E600BF07EF06081C1E0608DBEB0608D7
:10501000BC06060855EF06087EE906084AEF0608B2
:105020002EFC06081AEF06082DE9F04F914687B0CE
:105030000C461A4600218046FFF728F84D460646E2
:105040000027B9F1000F66D02946062220464AF013
:105050000BF90028324614BF0121002140460CBF45
:105060004FF0010A4FF0000AFFF710F806462878C3
:1050700013F0AAF98346F8B1687913F0A5F9AB7873
:10508000EA789BF805E095F801B04FF461714FF0B4
:10509000190C1CFB03131CFB0212297900B1407987
:1050A000CDE90410CDE90232CDE900EB1B4A3B46C5
:1050B00051464046FDF7D6FB207813F085F983462C
:1050C000F8B1607913F080F9A378E2789BF805E0F5
:1050D00094F801B04FF461714FF0190C1CFB0313ED
:1050E0001CFB0212217900B14079CDE90410CDE911
:1050F0000232CDE900EB094A3B4651464046FDF7F6
:1051000069FB0137142F04F1060405F1060598D157
:1051100007B0BDE8F08FCA46CEE700BF63EF0608D0
:105120002DE9F041054686B00846FFF753F80F46D3
:10513000064638B100235C491A46012006B0BDE896
:10514000F04171E70846FCF745F91328044600F3DF
:10515000A18006254543781C8DF81760FBF7D9FA26
:10516000524E074660B1FCF735F9C0B211F020FE8F
:1051700030B17319027983F8242A01238DF817308E
:105180003846FBF7C6FA074668B1FCF723F90D2845
:1051900009D8062303FB046383F8250A9DF817301A
:1051A00001338DF81730DFF80081A91C0DF11702CB
:1051B00041443846FCF712F9FBF7ABFA074668B1F1
:1051C000FCF708F9012809D89DF81730062202FBE0
:1051D0000462013382F8280A8DF817303846FBF74D
:1051E00098FA80B1FCF7F6F8C0B211F0E1FD50B1C9
:1051F0009DF817300179062202FB0462013382F820
:10520000291A8DF817309DF81720042A4FF006034D
:105210002FD103FB04630022A3F8282A062505FBEF
:10522000046520F04FFB95F8240A13F0CDF895F8AB
:10523000271A95F8267A19234FF46172804695F85B
:10524000290A13FB012613FB072713F0BDF8437946
:1052500098F80520039395F8283A0097CDE9016363
:10526000134895F8253A2146FDF77CFB06B0BDE8CA
:10527000F081052A05D103FB0463002283F8292A63
:10528000CCE7062ACAD008EB0502002348F805300F
:105290009380C3E7074913233246284606B0BDE88A
:1052A000F041FEF70DBA00BFCCAF0020A8A500204A
:1052B00063EF06087CEF06082DE9F04F904689B0B1
:1052C0001A460C4600218146FEF7E0FE3B4EDFF811
:1052D000F0B008F16C0307464546079394F90400C3
:1052E0000BF0A2FA00285DD0B8F1000F63D0294678
:1052F0000C22204649F0B8FF00283A4614BF01218D
:10530000002148460CBF4FF0010A4FF0000AFEF79B
:10531000BDFE074695F9040042F0BEF9EA7906EBB6
:1053200082020346D2F8802804922A7A06EB82028F
:105330005146D2F880280392AA7906EB82024846A9
:10534000D2F8802802926A7906EB8202D2F880288D
:1053500001922A6800925A46FDF784FA94F90400F3
:1053600042F09AF9E27906EB82020346D2F88028ED
:105370000492227A06EB82025146D2F880280392E8
:10538000A27906EB82024846D2F88028029262791E
:1053900006EB8202D2F880280192226800925A46D7
:1053A000FDF718FA079B0C35AB4204F10C0495D1BC
:1053B00009B0BDE8F08FC246D0E700BFBC060608C2
:1053C00082EF06082DE9F04780468CB00846FEF7CC
:1053D00001FF054638B1002359491A4601200CB097
:1053E000BDE8F04768E7CDE909000B90079107A8F1
:1053F000544949F06BFE064642F03EF8431C044611
:105400000ED12B460A2208A93046FBF743FF089B22
:105410001B782BB9C4B2132C96BF333444B264B298
:1054200020460BF0B3F9054628B94046FEF734F89C
:105430000CB0BDE8F08743498DF8284007A849F033
:1054400045FEB0B300230A221946FBF723FF0226CC
:105450000990DFF8F090DFF8F4A00027494607A88C
:1054600049F034FEF8B1FBF7B5FF374A002352F894
:10547000041B88421FD1DBB20AEB8302D2F88028DA
:10548000904210D1022F20D0032F23D05A1E012F7B
:10549000D2B215D00B2A03D88DF829300136F6B2D6
:1054A0000137042FDAD1052E1AD84046FEF730F81E
:1054B000BEE70126CDE70133102BD8D10023DBE76F
:1054C000052AEDD88DF82A30E8E7092BE8D88DF8C1
:1054D0002C30E3E79A1E0D2AE2D88DF82B30DDE759
:1054E00009AB03CB286018686960A860204642F0C9
:1054F000D3F8164A9DF82B1002EB81010346D1F830
:10550000801804919DF82C1002EB8101D1F88018CD
:1055100003919DF82A1002EB8101D1F880180291C5
:105520009DF8291002EB81020021D2F88028019217
:10553000099A00920846064AFDF74CF978E700BF41
:10554000A0AE002079E106083C0F0608BC0606085C
:1055500082EF06082DE9F04F90468BB00C461A46B4
:1055600000210746FEF792FD4546099000264FF0C0
:10557000190A4FF46179B8F1000F4BD029460A227D
:10558000204649F071FE0028099A14BF012100212C
:1055900038460CBF4FF0010B4FF0000BFEF776FDC5
:1055A0002A890692EA8805922A790492EA78039277
:1055B000AA7809901AFB029202926A781AFB029268
:1055C00001922A7800923346134A59463846FDF72D
:1055D00049F922890692E288059222790492E278BA
:1055E0000392A2781AFB0292029262781AFB02924C
:1055F000019214F80A2B00923346074A594638465E
:105600000136FDF7E7F81E2E05F10A05B3D10BB000
:10561000BDE8F08FC346DCE79FEF06082DE9F043B5
:1056200080468BB00846FEF7D5FD0F46044638B1DC
:1056300000235E491A4601200BB0BDE8F04389E71C
:105640000846FBF7C7FE1D28054600F3A5800A267D
:105650004643781C8DF82740FBF75BF810B1012317
:105660008DF82730FBF755F8514C074668B1FBF72A
:10567000B1FE0D2809D80A2303FB054383F88800EF
:105680009DF8273001338DF82730DFF82091711C09
:105690000DF1270249443846FBF7A0FEFBF739F825
:1056A000074668B1FBF796FE232809D89DF82730F6
:1056B0000A2202FB0542013382F88B008DF8273065
:1056C0003846FBF726F8074668B1FBF783FE0D283E
:1056D00009D89DF827300A2202FB0542013382F8DF
:1056E0008C008DF827309DF82730062B0CD009EB65
:1056F00006020023404649F80630536013810BB080
:10570000BDE8F043FDF704BF0A2606FB054600236B
:105710003846A6F88E30A6F89030FAF7FAFF07461A
:1057200018B1FBF757FEA6F88E003846FAF7F1FFDE
:1057300030B1FBF74FFE0A2303FB0543A3F89000AB
:105740001C4B4FF0FF325A600A2303FB05424FF413
:105750006170B2F890300693B2F88E30059392F8EB
:105760008C30049392F88B30039392F88A101923AB
:1057700013FB0101029192F8891013FB01030193BD
:1057800092F88830009300210B4A2B460846FDF71B
:1057900021F80BB0BDE8F08308491D23224640469E
:1057A0000BB0BDE8F043FDF78BBF00BF20C8002061
:1057B00098C700205C0400209FEF06087CEF0608D5
:1057C0002DE9F04F2DED088BDFF828A195B080462C
:1057D00091461E460C461546002794ED008AB5EE0C
:1057E000408AF1EE10FA7DD0D4ED019A94ED029A40
:1057F000D4ED038AB9F1000F49D0D5ED00BA95ED8B
:1058000001BAD5ED02AA95ED03AAB4EE6B8AF1EECA
:1058100010FA6CD1F4EE4B9AF1EE10FA67D1B4EEB7
:105820006A9AF1EE10FA62D1F4EE4A8AF1EE10FAB9
:105830000CBF0121002132468B46404681F0010118
:10584000FEF724FCB0EE6B0A064611A8FAF786FEB6
:10585000B0EE4B0A07900EA8FAF780FEB0EE6A0A87
:1058600006900BA8FAF77AFEB0EE4A0A059008A84F
:10587000FAF774FE0599069A079B0390029101922C
:10588000009352463B4659464046FCF7EBFFB0EECC
:10589000480A11A8FAF762FEB0EE690A83460EA81C
:1058A000FAF75CFEB0EE490A06900BA8FAF756FE2E
:1058B000B0EE680A059008A8FAF750FE069B059A14
:1058C0000390CDE900B302923B4652460021404688
:1058D0000137FCF77FFF082F04F1100405F11005D4
:1058E0007FF47BAF15B0BDEC088BBDE8F08F0021D5
:1058F000A1E700BFC2EF06082DE9F14FDFF8ACB118
:1059000006460C462046FEF765FC074638B10023E4
:105910005E491A46012001B0BDE8F04F50E75C49EE
:1059200005222046FBF77AFCA0B95A4B0022C3F8A7
:10593000E421C3F8F421C3F80422C3F81422C3F805
:105940002422C3F83422C3F84422C3F8542201B0FD
:10595000BDE8F08F042259462046FBF75FFC054660
:105960002046002D45D1FAF7D4FE07460028EED098
:1059700047F090FBDFF838A15FFA80F85AF8049BF3
:10598000B9F1000F07D144492246304601B0BDE8C5
:10599000F04FFDF76BBD424649463846FBF73EFCEB
:1059A000013584460028E9D1384A034617460021CC
:1059B0000133082B42F8101BFAD1384B03EBC50515
:1059C000D5F880E0BEF1000F05D13548354C494689
:1059D000FCF7C8FF96E795F87C50AC45F5DA0EEB7E
:1059E0000C130FCB07EB0C1484E80F000CF1010C27
:1059F000F3E7FBF7EFFC072805463DD82046FAF70A
:105A000088FE074658B3FAF7E1FB224B03EB051378
:105A100083ED790A01243846FAF77BFE074638B150
:105A2000FAF7D4FB1B4B03EB051383ED7A0A013421
:105A30003846FAF76EFE074638B1FAF7C7FB154B42
:105A400003EB051383ED7B0A01343846FAF761FE58
:105A500038B9304601B0BDE8F04FFDF759BD0446F6
:105A6000D9E7FAF7B3FB0B4B032C03EB051383EDDC
:105A70007C0A3FF44CAFECE70B4907233A4630462B
:105A800001B0BDE8F04FFDF71BBE00BF84B8002099
:105A90004EEC0608A0B600207EE90608BC06060803
:105AA000DBEF06082DED06087CEF0608D6EF0608AA
:105AB000501006082DE9F74F92460C461A46002171
:105AC0008146FEF7E3FADFF870B0804656460025BF
:105AD000BAF1000F2ED031460422204649F0C4FB13
:105AE0000028424614BF0121002148460CBF01276F
:105AF0000027FEF7CBFA738801933AF8253000931C
:105B000080462B465A4639464846FCF7ABFE63882A
:105B1000019334F8043B00935A462B4639464846D5
:105B20000135FCF757FE042D06F10406D0D103B071
:105B3000BDE8F08F5746EAE7E5EF06082DE9F341A7
:105B400005460846FEF746FB0C46074638B10023DB
:105B500033491A46012002B0BDE8F041AAE73149B5
:105B60002046FAF791FA70B92D4B04224FF47A705F
:105B70004FF4FA61013A1880598003F10403F9D116
:105B800002B0BDE8F0812046FBF724FC032806465E
:105B900041D82046FAF7BDFD074698B1FBF71AFC3D
:105BA0004FF0010804463846FAF7B3FD20B1FBF781
:105BB00011FCB8F1000F09D1284602B0BDE8F04150
:105BC000FDF7A6BC40F2EE248046ECE7A4F2EE22FC
:105BD00040F2DC539A4203D8A0F2EE229A420AD94C
:105BE000114940F6CA0340F2EE22284602B0BDE851
:105BF000F041FDF765BD0D4B0D4A03EB8603002117
:105C0000A3F8B441A3F8B601CDE9004033460846F5
:105C1000FCF7E0FDB4E7074903233A46E5E700BF98
:105C20004CC900204EEC0608F6EF060898C7002085
:105C3000E5EF0608FEEB06082DE9F04F89468FB028
:105C4000174600211A460646FEF720FADFF874A030
:105C5000054600240DF1240B59F82480CDF8088066
:105C6000594602A841F0C2FC57B357F824300393B9
:105C700098452A4614BF0121002130460CBF4FF041
:105C800001084FF00008FEF701FA04A9054603A831
:105C900041F0ACFC04A900912346524641463046EF
:105CA000FCF7E0FD2346CDF800B0524641463046B1
:105CB0000134FCF78FFD402CCED10FB0BDE8F08F42
:105CC000B846EFE704F00608F0B5074689B0084685
:105CD000FEF780FA0E46054638B1002319491A46E8
:105CE000012009B0BDE8F040A6E70846FBF772FBCB
:105CF0003F2804461DD83046FAF70BFD01462046E2
:105D000035F02CF978B10F4803AE314600EB840032
:105D100041F06CFC0C4A0096234629462846FCF7C5
:105D200059FD09B0F0BD384609B0BDE8F040FDF7B7
:105D3000B3BB06493F232A46384609B0BDE8F040C8
:105D4000FDF7BEBC5CC9002004F006087CEF060825
:105D50002DE9F04F924685B00C461A460021814647
:105D6000FEF794F9DFF874B0804655460026BAF184
:105D7000000F31D029460422204649F075FA002848
:105D8000424614BF0121002148460CBF01270027CD
:105D9000FEF77CF9EB780293AB7801932B880093A4
:105DA000804633465A4639464846FCF75BFDE37861
:105DB0000293A378019334F8043B00935A46334688
:105DC000394648460136FCF705FD102E05F104055D
:105DD000CDD105B0BDE8F08F5746E8E70EF00608D4
:105DE000F0B5074685B00846FEF7F4F90E460546BD
:105DF00038B100231C491A46012005B0BDE8F04027
:105E0000A6E70846FBF7E6FA0F28044623DC3046EF
:105E1000FAF77FFC0146204635F086F9A8B1134B0E
:105E200004F1400203EB8203294693F8C721029252
:105E300093F8C6210192B3F8C43100930C4A23466B
:105E40002846FCF7C7FC05B0F0BD384605B0BDE8F4
:105E5000F040FDF721BB07490F232A46384605B01D
:105E6000BDE8F040FDF72CBC5CCA002098C70020BC
:105E70000EF006087CEF06082DE9F04F85B01446B9
:105E800002911A4600210546FEF700F94FF000087E
:105E90000646062303FB08F707F5A0774FF0000935
:105EA000029B13F807B0002C00F08280E35D03939F
:105EB0009B45324614BF0121002128460CBF4FF0FC
:105EC000010A4FF0000AFEF7E1F8039B3A4ACDE9D8
:105ED00000930646434651462846FCF7C3FCCDE9ED
:105EE000009B354A43465146284609F10109FCF713
:105EF00071FCB9F1060F07F10107D1D108F10108D2
:105F0000B8F1060FC5D14FF4B277029BA7F5B2796D
:105F100013F807A0002C4DD014F807B0DA4532462C
:105F200014BF0121002128460CBF4FF001084FF09B
:105F30000008FEF7ABF8CDE9009B06461E4A062393
:105F400041462846FCF78EFC0623CDE9009A1A4A02
:105F500041462846FCF73EFC013740F26F139F4252
:105F6000D3D1029B93F86F71B4B194F86F81474518
:105F7000324614BF0121002128460CBF0124002411
:105F8000FEF784F8002300930B4ACDF80480072322
:105F900021462846FCF766FC00230093064A019739
:105FA000072321462846FCF715FC05B0BDE8F08F15
:105FB000A24694E7A046C7E720F00608F0B50546DC
:105FC00085B00846FEF706F90B46044638B10023B3
:105FD0001B491A46012005B0BDE8F0404CE71949BD
:105FE000184F6A46184649F09EF801AE88B1032C56
:105FF00004D12846FDF78CFA05B0F0BDFBF7EAF9AD
:106000006A4646F8040B39460020013449F08BF803
:10601000ECE7032CEDD1DDE90146039F31463A461A
:10602000E0B235F0BDF818B92846FDF735FAE3E7D8
:1060300005483B4632462146FCF794FCDCE700BFAE
:106040005CC9002079E1060820F006082DE9F04F30
:10605000924689B00C461A4600210746FEF716F80C
:10606000002607905546B3464FF019094FF4617862
:10607000BAF1000F28D029460622204649F0F4F84C
:106080000028079A14BF0121002138460CBF4FF0A9
:10609000010B4FF0000BFDF7F9FF6A79079019FB30
:1060A000028205922A7919FB02820492EA7803920D
:1060B000AA7802926A7801922A7800923346124AAC
:1060C00059463846FCF7CEFB627919FB02820592ED
:1060D000227919FB02820492E2780392A27802925A
:1060E0006278019214F8062B00923346064A59460C
:1060F00038460136FCF76EFB0A2E05F10605B7D1CE
:1061000009B0BDE8F08F00BF34F006082DE9F04F6C
:10611000074689B00846FEF75DF88B46044638B15D
:10612000002354491A46012009B0BDE8F04F8DE71D
:10613000514B084693F8A0AC93F8A19C93F88A8D34
:10614000FBF748F90928054600F38B8006264643ED
:106150000BF101008DF81F40FAF7DBFA474C83463C
:1061600048B1FBF737F90D2805D8A31983F8FC02CD
:1061700001238DF81F305846FAF7CBFA834668B1F1
:10618000FBF728F9504509D8062303FB054383F89C
:10619000FD029DF81F3001338DF81F305846FAF785
:1061A000B8FA824668B1FBF715F9484509D80623C5
:1061B00003FB054383F8FE029DF81F3001338DF881
:1061C0001F305046FAF7A5FA814668B1FBF702F98D
:1061D000804509D3062303FB054383F8FF029DF89E
:1061E0001F3001338DF81F30DFF88880311D0DF12D
:1061F0001F0241444846FBF7F1F89DF81F30062B7B
:106200000BD008EB06020023384648F8063093808E
:1062100009B0BDE8F04FFDF77BB903FB05424FF431
:10622000617092F80113192313FB0101059192F893
:10623000001313FB0103049392F8FF32039392F8C7
:10624000FE32029392F8FD32019392F8FC320093F1
:1062500000210B4A2B460846FCF7BCFA09B0BDE802
:10626000F08F084909232246384609B0BDE8F04FAF
:10627000FDF726BA9CB90020A8A50020A0B60020F2
:1062800034F006087CEF06082DE9F04F0F468BB07E
:10629000144600211A460646FDF7F8FE0546002C76
:1062A00000F0DD8022783B789A4218BF0121024637
:1062B00008BF002130460CBF4FF001084FF0000826
:1062C000FDF7E4FE23789E4A054641463046FCF73A
:1062D000C9FA3B789A4A41463046FCF77BFA002CD3
:1062E00000F0BF8062787B789A4218BF01212A466D
:1062F00008BF002130460CBF4FF001084FF00008E6
:10630000FDF7C4FE63788F4A054641463046FCF7E8
:10631000A9FA7B788B4A41463046FCF75BFA07F1D5
:10632000C9030593A31C0693822307F1020A04F113
:10633000CA0B07934FF000093B784B4500F393805D
:10634000002C00F0F68097F8EA3094F8EA209A42A0
:1063500018BF01212A4608BF002130460CBF4FF06C
:1063600001084FF00008FDF791FE94F8EA30764AF4
:10637000054641463046FCF775FA97F8EA30724A0E
:1063800041463046FCF726FA002C00F0D48004F198
:10639000EA0307F1EA0204F1FA014FF0010833F8C9
:1063A00002CF32F8020F844518BF4FF0000899421F
:1063B000F5D188F001012A46C9B23046FDF766FEE4
:1063C0000821054604F1EC00FAF776FE5F4A034621
:1063D00041463046FCF746FA97F8EA1007F1EC0020
:1063E000FAF76AFE594A034641463046FCF7F2F98D
:1063F000002C00F0A2804FF0FC094FF0010807EBE1
:10640000090104EB0900F9F73FFE09F1040900282E
:1064100018BF4FF00008B9F58E7FF0D188F0010168
:106420002A46C9B23046FDF731FE082104F1FC00CE
:10643000FAF782F9464A034641463046FCF712FA1B
:1064400097F8EA1007F1FC00FAF776F9404A03469C
:10645000414630460BB0BDE8F04FFCF7BBB9A04653
:1064600037E7A04655E7079BFB180993002C5ED041
:10647000079B0998E31819460893F9F705FE059B51
:106480005A789BF800309A42069A06BFB0FA80F814
:106490004FEA58184FF00008AAF10203023A0AF135
:1064A0000E0133F802CF32F8020F844518BF4FF0C7
:1064B00000088B42F5D188F001012A46C9B2304666
:1064C000FDF7E4FD6278069905469BF81800FAF797
:1064D000C5FD02909BF800300193089B00931D4A74
:1064E00009F1010341463046FCF7BCF9059B7A7877
:1064F000587E5146FAF7B2FD059A029012F8013F14
:10650000019309F10109099B05920093114A4B4639
:1065100041463046FCF75EF9069B10330693079B15
:1065200009330AF1100A0BF1010B079304E7A046A7
:10653000DCE7A04621E7A0464EE7A04680E700BF83
:106540004DF006085FF006088DF00608A5F0060875
:10655000BCF0060874F006082DE9F04F8FB0044631
:1065600002AA0846B14948F0DEFD054640B9034697
:106570000246AF494120FFF787FE0FB0BDE8F08F1C
:10658000AC49F9F781FD064628BBA84902AA48F0A4
:10659000CAFDFAF71FFF0828054606D9A6490823B1
:1065A00032462046FDF78CF8E7E7A44C94F8A03C6F
:1065B00083420CDC84F8A05CDFE73146384633F0D8
:1065C0003BFD013694F8A03CB342F6DCF2E7064608
:1065D00004F54A67F6E79A492846F9F755FD064655
:1065E000E0B9924902AA48F09EFDFAF7F3FE0828A6
:1065F000054603D9934908233246D2E78F4C94F8D5
:10660000A13C834202DC84F8A15CB6E7304629460F
:10661000013640F009FF082EF8D1F4E78A492846F0
:10662000F9F732FD064600BB804902AA48F07BFD1F
:106630000028A2D0FAF7CEFE0828054603D98349E0
:1066400008233246ADE77D4C94F88A3D834209DD4C
:10665000014604F54A6033F033FD294604F54A60EB
:1066600033F03CFD84F88A5D87E779492846F9F7DD
:106670000BFD064618BB714BDFF8B09193F88A7D8D
:1066800006AD01461022284648F06AFDA846BE42E3
:1066900002AA80F20A814946002048F044FD10B960
:1066A0006C493A460AE1FAF795FE013628F8020BE2
:1066B000EDE795E80F00684C84E80F005DE7674957
:1066C0002846F9F7E1FC0646C0BB5C4BDFF85C915D
:1066D00093F88A7D06ADBE4202AA80F2F380494655
:1066E000002048F020FD014610B95D493A46E5E03A
:1066F0000322284648F083FDAA464FF000082846AA
:1067000046F0C8FC404502D801360435E3E79AF864
:106710000000FAF77DFD08F101080AF8010BEEE729
:10672000504DB6000446B4423FF427AF06AB1919EA
:106730002819032233F06AFC0434F4E74A49284656
:10674000F9F7A2FC0746002840F0AC80DFF8EC80A7
:10675000364998F8A06C02AA48F0E5FC00283FF4FE
:106760000CAFFAF737FE451E01D4AE4203DC3F49B9
:106770003346012215E72D4902AA002048F0D3FC38
:10678000014600283FF4F9AE0026082203A88DF840
:10679000146048F034FD0DF10C0903A846F07AFCB2
:1067A000B0421BD8214902AA002048F0BCFC0028B6
:1067B0003FF4E3AE037898F8A1AC01930026B1460C
:1067C00056451A4902AA4FF0000080F2858048F031
:1067D000AAFC834650B9264952466FE099F800005A
:1067E000FAF716FD013609F8010BD6E7A6B99BF8B2
:1067F0000030303B092B0FD91E49F9F745FC38B161
:106800001D495846F9F740FC70B11C495A4655E0FD
:106810004FF001094FF0FF365846FAF7DBFD00282C
:1068200030DA17495A4649E0B146F3E779E10608FC
:1068300048B20020D3F00608D9F00608A8A5002029
:10684000E4F00608EDF00608FBF0060807F106087C
:1068500019F1060808F2060834B3002043F10608CF
:1068600028F2060844B300206DF1060872F106080C
:1068700048F2060855E106087EF1060885F106088B
:10688000BAF106080EAB03EB4603013623F8200CE1
:1068900096E72049524611E033F8022B24F8022FE4
:1068A000013730E01C492A4608E01C49002048F026
:1068B0003AFC00283FF4FDAE19493A462046FCF761
:1068C000D5FD5AE61549002048F02DFC00283FF47C
:1068D00027AF14493A46F1E748F025FC0028D8D103
:1068E000114C05EBC50082302044082203A933F087
:1068F0008DFB0198FAF78CFC08EB050304EB0514FB
:1069000083F86A0D06ABBE42C6DC454485F8829D1D
:1069100033E600BFCFF10608F2F1060879E1060878
:1069200025F106084FF1060848B200202DE9F04F86
:1069300089B00F4690460021139A03930646FDF74F
:10694000A5FB87EA08086FEA0803DFF8849006933E
:1069500004460025284609F0F9FE129B184230D063
:10696000069BDFF870B0034014BF4FF0010A4FF0F0
:10697000000A049310EA07030CBF4A465A46284609
:106980000593079209F0F4FE039B079A0090804656
:1069900051463046FBF766FF049BB3FA83F122466B
:1069A00049093046FDF772FB059A039BCDF800803C
:1069B0000446002A0CBF5A464A4651463046FBF769
:1069C00009FF0135172DC5D109B0BDE8F08F00BF13
:1069D0006DF20608D0EF060870B5044608460E466C
:1069E00046F058FB3146054602462046FAF716FCAB
:1069F00068B9635D1846FAF7FBFB00B933B9013596
:106A00002C44204601340378202BFAD070BD00209E
:106A1000FCE708B504460948FBF7D0FEFBF7B2FED9
:106A2000074B53F8080C09F051FF06F0C1FE012C8A
:106A300001D143F01DFAF7F719F800BF74F2060808
:106A400098C7002010B5044608460B46FDF7C2FB68
:106A500028B9094903221846FAF7E0FB28B9074884
:106A6000FBF7D2FE0120FFF7D4FF20460449BDE822
:106A70001040FCF7FBBC00BF80F2060884F2060859
:106A8000A9EB06082DE9F74F064601AA08462F494B
:106A9000DFF8C880DFF8C890DFF8B0A048F043FB0B
:106AA0004FF0000B04465D4601271CBBBBF1000FF5
:106AB00028D1274C002D44D026482946FBF752FF09
:106AC00094F838300BB905F04BFD3EF0D3F90023B4
:106AD00084F86130FBF72CFE15B12846FDF7E3FA88
:106AE0009FB13046FDF798FA78B1FBF791FC002092
:106AF000FFF78FFFBBF1000F0AD02046FAF76AFCC0
:106B000085B2C5B93046FCF7C7FC03B0BDE8F08FCD
:106B100041462046FAF7A6FB80B949462046FAF7D7
:106B2000A1FB0028EED05F4601AA5146002048F0A4
:106B3000FAFA0446B9E74FF0000BF5E74FF0010B06
:106B4000F2E70548FBF760FEBFE700BF79E1060802
:106B5000A8A50020AFF20608D2F20608A6F20608A1
:106B6000B1F9060810B50C46FDF756FA78B1084B96
:106B70000122DA74FBF74CFC0648FBF745FE064998
:106B80002046F9F781FA10B10020FFF742FF10BD4F
:106B9000A8A50020E8F206087BE10608F0B5032965
:106BA00085B005460C46164614D80B4F3970FBF7D6
:106BB0000DFE0A492846FDF7C9FF0949224601A8EA
:106BC000FAF736FA01AB324608212846FDF78EFA6D
:106BD000FF233B7005B0F0BD5C0400202DED0608DE
:106BE000CCEE0608F0B5032985B005460C461646DE
:106BF00014D80B4F7970FBF7E9FD0A492846FDF7D9
:106C0000D5FF094922466846FAF712FA6B46324622
:106C100010212846FDF76AFAFF237B7005B0F0BD0E
:106C20005C0400202DED0608C8EE060810B586B0FD
:106C30000E4B04930E4B03930E4B02930E4B01939A
:106C40000E4B0F4A0F49009304460F4B0F48FBF7BA
:106C500021FEFBF7BBFD3CB10D4A0E490E4806B0C4
:106C6000BDE81040FBF77EBE06B010BD25F3060858
:106C70002AF3060835F306083EF306084AF3060829
:106C80005CE30608EFF20608B3A50020FAF2060856
:106C90004FE80608A3E8060854F306080120C5E7F4
:106CA0002DE9F04F0A4689B000210546FDF7EEF9BF
:106CB000394C059094F9000006F024FE8146608866
:106CC0003EF09EF8354BD0F808B093F8387017B105
:106CD0005F46D0F80CB0A379012B38BF012306938F
:106CE00000262279637906FB02331BF80380002F0C
:106CF0003BD0FB5C059A0793434514BF012100215B
:106D000028460CBF4FF0010A4FF0000AFDF7BEF90C
:106D1000079B0590013653B303F00F021B09403364
:106D2000CDE9006302924B461D4A51462846FBF7C7
:106D300099FDB8F1000F24D008F00F034FEA18189E
:106D4000029308F14003CDE90063154A4B465146D2
:106D50002846FBF73FFD069BB342C2DC114B0834CB
:106D6000A342A7D109B0BDE8F08F3B46C2E7002F90
:106D7000DFD00D4A00964B4651462846FBF772FD80
:106D8000D7E76B06E7D4084A00964B46514628469B
:106D9000FBF720FDDFE700BFC40B0608A8A5002015
:106DA00081F30608D40C060897F306082DE9F04F86
:106DB0000A468DB000218346FDF768F9704CDFF874
:106DC000CC91039004F1800A0025A37A99F83860E9
:106DD000AB4200F3938010345445F5D140F21620B5
:106DE0003EF00EF8D0E902450DF1180A002E4FF0E2
:106DF00015024FF00001504604BF2546344648F0C6
:106E0000AFF900272E78002E3ED0697805913046E4
:106E100006F060FE95F90290049009F101025342D8
:106E20005341002C00F0A98005990022A05CB042DB
:106E300040F09F80224492F90280C14540F0978043
:106E400052788A4208BF012301220AF8072003F082
:106E5000010383F00101039A05935846FDF716F9E3
:106E6000059B039044B1474A0499CDE900B23046EE
:106E70004246F9F7D3FC059B434A0499CDE900B299
:106E800030464A46F9F7CAFC0137152F05F10305CC
:106E9000B8D184B3DFF8EC80DFF8EC90564604F10B
:106EA0003F0716F801ABBAF1000F21D12078F8B1F5
:106EB00094F9023001331BD0617806F00BFE039A7F
:106EC000054601215846FDF7E1F894F902200390A8
:106ED000534620782946CDE900B8F9F79FFC207881
:106EE0005346CDE900B94FF0FF322946F9F796FC39
:106EF0000334BC42D5D10DB0BDE8F08FE0883DF041
:106F00007FFFD0E90231627A207A002E08BF19464D
:106F100005FB002208BF33468F562BB39E56039ABB
:106F20000493B74214BF0121002158460CBF4FF013
:106F300001084FF00008FDF7A9F8049B039043B146
:106F4000104B3246CDE900B3294643462046F9F7B7
:106F500021FC0D4B2946CDE900B33A464346204675
:106F6000F9F718FC013530E74FF0FF36D7E700237B
:106F70006AE703323F2A7FF459AF4FF0FF3868E7E2
:106F80008804002065280108D5270108A8A500204D
:106F90002DE9F04F80468BB008460D4646F07AF852
:106FA000024600283AD0A9492846FAF737F904469C
:106FB000A0BBFBF70BFCA648A64DA74EA74FDFF8DA
:106FC000E082FBF71BFC142040F042FA0721B4FBDF
:106FD000F1F1C1EBC102A21A304601320131FBF7D7
:106FE00059FC95F8199095F91800B9F1000F0ED0D9
:106FF00006F088FC4A4601464046FBF7B3FC0134E4
:107000000E2C05F12405E1D10BB0BDE8F08F06F0A0
:1070100079FC01463846FBF7A5FCF0E72846904985
:1070200005AA48F080F8054620B901464120FFF73F
:10703000BDFEE9E78B49F9F727F820B98A494046B0
:10704000FCF714FAE0E7894E082700243168284647
:10705000F9F71AF8002808BF3446013F06F1100678
:10706000F4D154B982492846F9F70EF828B181497C
:107070002A464046FCF7FAF9C6E7002078498DF821
:10708000130005AA48F04FF80646002C4ED0002801
:107090004AD0FAF79FF9031E43DB2279062A3BD137
:1070A000E168012202FA03F008423AD07248DBB2EA
:1070B00040FA03F1C90734D59A40013A104048F02C
:1070C000E3F80546E0883DF09BFE6C49D0E90223D9
:1070D00091F83810002918BF1A46217A637A05FB07
:1070E0000133D118002712F90390029103975C49EC
:1070F00005AA002048F017F8834600283FD16049D0
:1071000001239CB3029A204692F90020CDE9003178
:107110002946F9F73FFB77E75D1E13B1A37A9D423D
:10712000D0DB58493246A4E7574EFAE768B10DF173
:107130001301FAF729F928B19DF813502846F3F7FF
:1071400041F920B95149324693E74F4EFAE72846B4
:10715000F3F752FF8146284606F0A8FC0390284624
:1071600006F0E0FC254607460294C0E7CDE9003171
:107170009DF813004A463946F9F750FB44E7394970
:10718000F8F782FF064600282FD1ACB1404FEDB290
:10719000207972B22946F3F7F7FE00283FF434AFA6
:1071A0000288037800933146C2F303233846120B5A
:1071B000FBF7D8FB0136EBE738687979344C72B2CB
:1071C000F3F736FF00283FF41FAF028803780093DF
:1071D0003146C2F303232046120B0136FBF7C2FBF4
:1071E0000E2E38687979EAD10EE72A495846F8F721
:1071F0004BFF002877D05846FAF7ECF8824642B2A7
:107200009CB12079E9B2F3F7BFFE00284ED12946A0
:107210002046F9F771F926681F49CDF800B00346FA
:1072200032464046FCF722F9EEE65FFA8AF60D2E6A
:107230003868797936D99DF813301849CDF800B0FF
:107240001A09403203F00F03EBE700BFABF3060867
:10725000B0F30608A4000020C6F3060892E406086E
:1072600079E10608E1E50608D8F30608880400205D
:1072700009F70608ECF30608FE7F1000A8A5002019
:10728000D5270108FBF306082DED06080BF40608C8
:107290001DF406089BE906083FF4060862F4060898
:1072A00037F50608F3F7C4FE0028C4D006AE314611
:1072B0005046F9F735FF08A94846F9F731FFCA45A6
:1072C00020D04FFA8AF38CB1029A294613702046D7
:1072D000F9F712F9276800960246154808AB3946B7
:1072E000FBF740FB90E64FF0FF3ADFE7039A1148C7
:1072F00093709DF813200096110908AB02F00F025D
:107300004031EDE75CB129462046F9F7F5F82668EB
:107310000246094808AB3146FBF724FB74E69DF8AA
:1073200013200648110908AB02F00F024031F3E7C1
:107330008AF40608ADF40608D5F40608F0F4060849
:107340002DE9F04F07468BB040F216200C463DF079
:1073500057FD2246054600213846FCF797FE434B71
:10736000D5E9024593F83830002B08BF254606467C
:107370004FF015024FF0000104A808BF1C4647F06B
:10738000EFFE05F13F03039395F80090B9F1000F6C
:1073900031D095F801A0002C65D022460023117849
:1073A000494558D128336B4492F80180012203F8F3
:1073B000182CD045324614BF0121002138460CBF9D
:1073C0004FF0010B4FF0000BFCF760FE064654B186
:1073D000B8F1000F07D0264B00935A463B46414672
:1073E0004846F9F763FA234B00935A463B46514609
:1073F0004846F9F75BFA039B03359D42C4D13CB381
:10740000DFF86C90DFF86CA0651C0DF110084034BB
:1074100018F8013BCBB915F8013CB3B116B13046B1
:10742000FBF7F2F9297815F8010CCDF800903B46EE
:107430000022F9F73BFA002215F8010CCDF800A064
:107440003B461146F9F732FA00260335A542DFD153
:107450000BB0BDE8F08F0133152B02F103029ED172
:107460004FF00008A5E7A046A3E700BFA8A50020AD
:1074700065280108D52701082DE9F04F07468DB092
:1074800008460D4645F006FE044628B9014601208F
:107490000DB0BDE8F04F53E70246A6492846F9F77C
:1074A000BDFE30B9A44938460DB0BDE8F04FFBF73A
:1074B000DDBFA24922462846F9F7B0FE002857D181
:1074C000FBF784F99E48DFF8B882DFF88892DFF88E
:1074D000B4A2FBF793F917203FF0BAFF0F2518F974
:1074E000016B002E38D097483146FBF7D3F90124C1
:1074F0000023A1B23046039306F04EFB074606F088
:10750000D7FB90F90020039B8346D2B10BB9FBF760
:107510005DF9BB799BF801109BF90000039103F022
:107520000203002B0CBF4F465746C1B106F0EAF9E3
:107530000399009103463A4683482146FBF712FA25
:1075400001230134052CD4D113B98048FBF756F937
:10755000013D15F0FF05C2D10DB0BDE8F08F06F07A
:10756000D1F93A46034621467948FBF7FBF9E7E7AC
:10757000002478498DF81B4007AA284647F0D3FD20
:1075800018B93846FBF788FFE6E70DF11B01F9F75C
:10759000FBFE81460028F4D09DF81B502846F2F7E8
:1075A00011FF20B96C493846FBF760FFD4E7DFF8DC
:1075B000D88123464FF0FF3403EB430218F8022032
:1075C00095420BD0002C02DA002A08BF1C4601337A
:1075D000152BF1D1002C16DA6049E4E71C465D4911
:1075E00007AA002047F09FFD0646002800F094807F
:1075F0005049F8F749FD20BB594FDFF88881DFF883
:107600008C91044614E04FF00009E8E7306896F8E2
:1076100007A0F3F75DFDB179737911F0020F0CBF8C
:10762000394641460246009148465146FBF79AF9D1
:1076300001342146284606F04DFA06460028E5D1D9
:107640008AE7484902223046F9F7E8FD4FEA151A61
:107650000AF1400A05F00F0B002845D10390B01C39
:10766000F9F7B8FE039902460491284601310592C4
:10767000039106F02FFADDE90313059A38B93A4968
:1076800000965B4652463846FBF7F0FE64E7C07949
:107690009042E9D11F466300B9F1000F31D01A19A9
:1076A00042445678013E7A1C234414BF29460021E7
:1076B00008EB030208F803107B1C53700AACFF238D
:1076C0009370394622462846F9F73AFD08AA314612
:1076D0002846F9F735FDB74216D1244808AB5A467B
:1076E0005146FBF73FF937E721493046F8F7CCFC24
:1076F00020B1204900965B465246C4E74FF0FF3761
:10770000C9E74FF0FF36CEE71B48009408AB5A4656
:107710005146FBF727F91FE704EB4404174B00938E
:10772000A044024698F8011001232846F9F7BEF854
:1077300012E700BFE1E50608D8F30608ABF3060838
:107740000CF5060825F506082CF506084DF5060883
:107750003EF5060879E1060853F506086AF50608BD
:107760002DED060893F5060896F50608E8F50608D7
:107770009BE90608C2F5060806F60608D5270108A3
:10778000A871060863E20608A83D00207EF50608F9
:107790002DE9F04F89B0074605AA08469C4947F0F5
:1077A000C2FC054630B901464120FFF779FA09B01D
:1077B000BDE8F08F9749F8F767FC044600283CD1F4
:1077C0009548964D964EDFF89882FBF717F81420EF
:1077D0003FF03EFE95F9060006F094F82968AA8865
:1077E00001F13F4101F57E01B2FA82F2890A0346B6
:1077F0004131C2F11F023046FBF74CF8E97911B173
:107800004046FBF747F80134FAF7E0FF502C05F14A
:107810000805DFD17E4905AA002047F084FC814994
:10782000F8F732FC0028C2D138467A49FFF724FE27
:1078300078493846FFF7ACFBB9E7DFF8FC91002444
:1078400019F9340006F05EF8804601462846F8F73C
:107850001BFC40B10134222CF2D173492A46384630
:10786000FBF704FEA3E76A4905AA47F05CFC06465D
:1078700090B3F9F7AFFD05466C4B03EBC4034FEA39
:10788000C40A93F80E354BBB002D29DC09EB0A0323
:10789000588893F8049093F805A03DF0B1FAEBB244
:1078A000D0F808B0009303FB09AA002E00F09A80DC
:1078B0003378002B00F0968006A93046F9F764FD76
:1078C000002800F08C809DF8185005BB0BF80A507A
:1078D0005748FAF793FF6AE70546CDE7002D05DD27
:1078E000012B1A4638BF0122954208DD012B514970
:1078F00038BF012301223846FBF7E2FE57E744492F
:1079000005AA002047F00FFC013D0646BEE72846C9
:10791000F2F758FD814600285DD02B0940330293D1
:107920000BF80A5005F00F03434F03934FF0000884
:10793000BB79012B38BF012301930026788897F883
:1079400004B097F805A03DF05BFA06FB0BA3826834
:10795000D15CA94222D1444504D10099B1421DD045
:107960000021D154DDE9021234485FFA86FB5FFA48
:1079700088FAFAF78FFF59465046FAF7D5FF444583
:1079800009D12F48FAF786FF50465946FAF7CCFF3F
:107990002C48FAF77FFF2C48FAF730FF019B01369D
:1079A000B342CBDC08F10108B8F1220F07F1080758
:1079B000BED1D9F80010B9F80420244801F13F41A4
:1079C00001F57E01B2FA82F2890AC2F11F02413149
:1079D000FAF7C8FFEBE63846FBF75EFDE7E61C4921
:1079E00032463CE71BF80A30013573B11A091949D0
:1079F00003F00F03403206A8F9F71AFB06AB16484E
:107A00002A464146FAF7AEFFD1E6144BF7E700BF2E
:107A100079E10608ABF306082CF60608D4390020F5
:107A20006AF6060875F6060879F60608BC06060822
:107A300095F606087CEF0608C40B0608A7F60608AC
:107A4000DEE10608CBF606084DFB0608D5F606086B
:107A5000F1F6060890F306080DF70608A8E00608F8
:107A600010E20608224BB0F5FA6F1A680346A8BF69
:107A70004FF4FA63B3F57A7FB8BF4FF47A73D20448
:107A800016D540F2DC52904215D007EE903A40F203
:107A9000DB529042F8EE677A1FD8DFED166A9FED51
:107AA000167A9FED160A77EEE67AA7EE870A7047F8
:107AB000B0F57A7F02D89FED120A704707EE903A30
:107AC000DFED106A9FED107A9FED100AF8EE677AED
:107AD00077EEE67AA7EE870A7047DFED0D6A9FED35
:107AE0000D7A9FED0D0A77EEE67AA7EE870A7047CA
:107AF00068AF002000007A44D62000C000E0824435
:107B00000000000000407A4466100040000040423F
:107B100000A0BB44D62000400000834410B40023E2
:107B2000094C0A490A4AC0F802404FF4EB7C5DF860
:107B3000044BA0F806C003700381C0F80A10C0F817
:107B40000E204382704700BF4A01B400C2010E01FB
:107B500096004400704700BF704700BF0020704788
:107B600001207047704700BF704700BF704700BFDB
:107B7000704700BF9FED010A704700BF0000000082
:107B800000207047064B1B78834206D9054B00EB5B
:107B9000400003EBC003586970470020704700BFE6
:107BA000291F00202C1F0020034B00EB400003EB9B
:107BB000C003587C704700BF2C1F0020024B187870
:107BC000003818BF01207047291F002003681B6977
:107BD00003B11847704700BF70B5094C236873B1F3
:107BE0000546002606E099681A681E7321609047D2
:107BF000236823B15A68AA1A002A1846F3DA70BD1E
:107C00002008012008B5254B1B68DB040AD5B5EE1A
:107C1000400AF1EE10FA12D19FED210A46F04CFD18
:107C200080B208BDDFED1F7AB4EEE70AF1EE10FA7C
:107C30001CDA9FED1D0A46F03FFD80B208BDDFED66
:107C4000197AB4EEE70AF1EE10FAE5D49FED177A4F
:107C5000B4EEC70AF1EE10FA14D870EE677A9FED11
:107C6000147A9FED140AA7EE870AE4E770EE677AAC
:107C70009FED117A9FED110AA7EE870A46F01CFDD1
:107C800080B208BDDFED0E7A9FED0E7A70EE677A56
:107C90009FED0D0AA7EE870ACDE700BF68AF002071
:107CA0000080BB440000404200007A4400E082446F
:107CB00066BEFFBE0060BB4438DFFF3E00407A4432
:107CC0000000834466BEFF3E00A0BB44F8B5CB4B2A
:107CD0001B6813F004052DED048B40F0DD809FED53
:107CE000C88AC84C13F0200305D094F8803013F0F4
:107CF000020340F09F8094F8C120DFEDC38A94F81E
:107D0000C01012F0010240F0AC80002940F08D80DC
:107D1000D4ED317A9FEDBD7ADFEDBD6A67EE877AEB
:107D200094ED337AE8EE267A38EE477AC4ED317A6C
:107D300084ED327A63B194F8D420D4F88430C4F856
:107D4000D03001218A4284F8C21018BFC4F8C8306C
:107D5000B04B1E780D2E0BD1D4ED217A9FEDAE7A6B
:107D6000AE4B67EE877AFDEEE77A17EE902A9A809F
:107D70009FEDA37AB0EE489A0025D4ED397AD4ED80
:107D80003A6A94ED388A37EE677AE6EE877A37EE0C
:107D9000C87AC4ED397AA6EE878A84ED388A84EDF4
:107DA000378A0DB184ED328A94ED3B7AD4ED3D7A79
:107DB000DFED9B5AD4ED3E6A94ED3C0A84ED3B8A9C
:107DC00038EE477AB0EE676A97EE256AE6EE867A75
:107DD00037EEC07AC4ED3D7AA6EE870A84ED3C0A00
:107DE00084ED3F0A46F068FC02B282EAE273A3EB3C
:107DF000E2739BB2092B40F2DC80002AACBF0A3848
:107E00000A3005B20D2EA4F8005100F0BD80242EDA
:107E100000F0D180382E05D1B0EE480A46F04CFC77
:107E20007E4B9880BDEC048BF8BD84F8C22084F8AA
:107E3000C0206DE7D4ED247AB4F89430F8EEE77AF8
:107E4000C4ED217A002B40F08280DFED6F8A94F838
:107E5000C12094F8C01012F001024FF001033FF46A
:107E600054AF002962D0D4ED339A6A4A94F8C270B4
:107E7000167838EE699AA3B117BB002D00F0A880E0
:107E800094ED210A70EE487A012377EEA97A84F8FE
:107E9000C230C4ED347A17E05A4C012594ED1D8AA6
:107EA00020E70D2E65D0DFED568AA7B9002D4AD008
:107EB00094F8D430002B44D1B0EE497A01255CE728
:107EC00094ED210AD4ED347A30EE670A0D2E84ED5C
:107ED000370A00F08A8094F8D4307BBB94ED377A6F
:107EE000002DEBD094F8D53077EE487A06EE903A34
:107EF00077EEA97AF8EEE66AF0EEE77A67EEA67A10
:107F0000DFED486AF4EEE67AF1EE10FAC4BF68EEEF
:107F1000A66AC6EEA78AF7EE007A77EEE87A67EEF1
:107F2000897AE8EE877AB0EE677A26E7D4ED319A5F
:107F30000122C4ED339A84F8C02096E7022B02D0C8
:107F40000DB1012BB8D094ED377A012515E707EE76
:107F5000903ADFED336A9FED347AF8EEE77AC6EEB9
:107F6000A78AF4EEC78AF1EE10FA88BFF0EE478ACE
:107F70006DE7DFED2E7A94ED370A20EE270A46F002
:107F80009BFB264B98808EE7DFED257A9FED270A35
:107F9000224C68EEA77A29EE000AFDEEE77A17EE8A
:107FA000903A238046F088FBBDEC048B6080E5802E
:107FB000F8BD002526E7DFED1D7A94ED320A20EEAC
:107FC000270A46F079FBBDEC048B144B5880F8BDB2
:107FD0000D2EB8D1DFED157A94ED370A20EE270A81
:107FE00046F06AFB0D4B9880ADE7DFED107A20EE8E
:107FF000270A46F061FB094B98806CE780BE0020A1
:1080000000000000200801209A99993ECDCC4C3FF9
:10801000CDCC4C3EA03500200AD7233CA43500200F
:108020000000C84200401C466666663FCDCCCC3D91
:108030002DE9F04F6B4B1B7887B0002B00F0CB8005
:10804000694D6A48A968FAF78DFC69686848FAF7CB
:1080500089FC684B6848D3E90031C91A674B1A6834
:10806000B1FBF2F2FAF77EFCFAF7B0FB6448FAF7DC
:10807000C5FB6448FAF7C2FB4FF00008624B1B785F
:108080005FFA88F4A34222D8FAF7A0FB5F4D604E56
:10809000002455F8041F30460134FAF7FBFB162C78
:1080A000F7D1FAF793FB5B4D594E01242B466968D3
:1080B0001B683046C91A0134FAF7ECFB162C05F19F
:1080C0000405F3D107B0BDE8F04FFAF77FBB524B80
:1080D000142603EB840306FB045693ED410AB6F81D
:1080E0000E9046F0E9FA96F81EA01AF0010F0CBFA8
:1080F0002D2252221AF0020F0CBF2D2354231AF006
:10810000040F0CBF4FF02D0C4FF0560C1AF0080F57
:108110000CBF4FF02D0E4FF0430E81B21AF0800FBE
:108120004FF03C0BB1FBFBF105914FF064010CBF2C
:108130004FF02D0A4FF0530A80B201FB09F1671C82
:10814000CDE902A10490CDE900CE34483946FAF7D2
:10815000A1FBB37FDB073AD55C23314A6343D118D7
:10816000D05891ED010A70B1DFED2E7AB8EE400AD9
:1081700020EE270A07EE900AF8EE677A80EE270ACB
:1081800046F09AFA00B2642290FBF2F102FB11026F
:108190002548FAF77FFB142101FB075701FB045424
:1081A000F988628A0491218B0391E18A0291A18B63
:1081B0000191A18A009102F0030319214B431B484E
:1081C000218A9208FAF7CEFB08F1010856E7184811
:1081D000FAF7F4FADFE7174807B0BDE8F04FFAF70F
:1081E0000DBB00BFAC180020943800204FF70608E4
:1081F0005FF70608C839002076F70608A81800209F
:10820000A3F70608FFF7060870B000203C390020ED
:10821000AFF8060840390020200801205BF8060866
:10822000B435002000401C4678F806088DF8060892
:1082300084F80608B3F806082DE9F84F00261F4D0C
:10824000DFF88090DFF880A007460C46B046204655
:10825000FBF7C0FFD5F800B048B921465846F9F7FA
:1082600001F820B968682146F8F7FCFF80B158464C
:10827000FAF7A4FA696811B15046FAF70BFBA9683E
:1082800011B14846FAF706FBFAF7A0FA4FF00108D9
:108290000136382E05F11005D9D12046FBF79AFF9B
:1082A00048B9B8F1000F06D1224638460449BDE866
:1082B000F84FFBF7DBB8BDE8F88F00BF7C3C060841
:1082C000DBF80608D5F80608CFF80608F8B5384CEC
:1082D0002368002B57D00A2801D00D2851D1354DE5
:1082E00095F824310BB1FAF771FA334E2321304659
:1082F00046F04DFF08B1801B20602368002273B94F
:1083000002B12360FAF72EFA95F82431F3B1BDE8F3
:10831000F8402A48FAF752BA01220B46EFE7591EF5
:10832000705C2028F8D092B90022254C224FF254DC
:108330003926013E0DD13146224B9C4212D2E368D0
:108340002068984795F82531002BDBD1F8BD2360D4
:10835000EAE721683846FEF73FFB01460028EBD1EB
:108360001034E6E795F8243123B117491748FAF796
:1083700069FFC7E71648FAF721FA0F48FAF73EFAFD
:10838000C0E7FF2BE2D8A0F120025E2ADED80BB9AD
:108390002028DBD05A1C2260074AD054054B93F8A2
:1083A0002431002BD2D0BDE8F840FAF751BA00BF13
:1083B00048BE00202008012048BD002076E10608C4
:1083C0007C3C0608FC3F0608EFF806080BF9060897
:1083D00011F9060870B5254C2378012B00D070BD2B
:1083E000234B1B68002BFAD0224D2B6828465B6874
:1083F00098470028F3D0204B204E1A683388928883
:108400009A421FD31E49096800224968EA622A6815
:1084100003FB01F12846D36898472B689B6813B18A
:1084200028469847F8B1174A338852680133338099
:10843000002AD4D0116893884A69134218BF1B04DC
:108440008B6170BD0F4A104B52681B780021217060
:10845000002AC4D091881268C3F340031B0101FABB
:1084600003F3936170BD41F0D9FEDCE7A24F002019
:10847000CC2C0020D02C00209C4F0020A04F0020AE
:10848000944F0020702C00207C2C00202DE9F84F08
:108490002DED028BB04CB14B94F8C12094F82651CD
:1084A0001F88D20780465DD5AD4E94ED4E8A012DD2
:1084B00000F09080022D49D0ADB9B4F82C319F4224
:1084C000A84B00F2B6801A68F37DD4F83C1103EB98
:1084D000830303EB8303521AB2EB830FC0F22681AE
:1084E000012584F82651F37B33B1B38923B19E4B28
:1084F0001B78002B40F0918094F82721AA4238BFC6
:108500002A46337A632B07D8022D94F8301100F0F5
:10851000DD80002940F0EE80944B9FED957A1A7033
:10852000D4E95230C4F84C311B1A07FB03F307EEB1
:10853000903AF8EEE77AB17BA7EE878A84ED4E8A0F
:1085400000293BD1BDEC028BBDE8F88FB4F82A318D
:10855000BB42C8D2834B01251B6884F82651C4F85E
:108560003C31C0E7EA1E012A45D918897C4EC0F388
:108570000B0046F089FE092897DDB6F80690B9454C
:1085800002D83388BB4290D2B7EB490F8DDC03236E
:10859000DFED787A744A84F8263184F82731002395
:1085A000B0EE678AC4ED4E7A1370A4F82831A4F8AF
:1085B0002A31A4F82C31A4F82E312CE0012A00F045
:1085C000A380022ABED1BDEC028B0720BDE8F84F84
:1085D00008F050BAB4F82E31BB422FD2B4F828318B
:1085E000BB42604B38BF00251B6838BF84F826515A
:1085F000C4F83C3177E75A4EB6F80690B94502D830
:108600003288BA422CD2B7EB490F29DC032D40F057
:108610009A8094ED4E8A032565E711F0B7FB002898
:1086200079D102239D422A4684F8273138BF1A4661
:1086300067E71B68C4F83C31002554E7494BD4F880
:108640003C111A68337E03EB830303EB8303521A56
:10865000B2EB830FFFF647AF022584F8265142E7BD
:108660001889C0F30B0046F00FFE092860DD317D4C
:10867000002284F8262184F82721002900F0808038
:10868000394B1970B388728894ED4E8A13FB01F34D
:1086900012FB01F2717C9BB28B4292B2A4F828319A
:1086A00086BF5B1A9BB200238A42A4F82A2186BFA8
:1086B000521A92B20022A4F82E21642284F83121A9
:1086C0000022A4F82C31C4F83421F8E691B9012035
:1086D000C4F8348184F83001C3F1640301FB03F072
:1086E000254B83FB0013C017A0EBA350643084F824
:1086F000310111E7D4F834112048A8EB010181427F
:10870000EADB84F8313107E7BDEC028B0820BDE8D5
:10871000F84F08F0AFB9337C83420FD301239D4259
:108720002A4684F8273138BF1A46EAE60025DAE6F9
:10873000032D3FF46EAF94ED4E8AD4E6002384F807
:1087400027312A46DDE61889C0F30B0046F09CFD70
:1087500009283FF714AFEEE720080120A4C6002047
:108760006CAF0020A0180020B4C60020B5C60020C1
:10877000ACC52737000000006BCA5F6B809698007D
:10878000224832880068B7FBF2F20132082A90F9D9
:108790007600DFF88490CABF0822D1B21146904219
:1087A00089F800103FF46EAF00283FF46BAF184813
:1087B00090F800E00EF1010505F0030575453FF462
:1087C00061AFDFF858B04FF0FF304FF0EA0A0AE02F
:1087D000002803DABCF1000F08BF2846013505F078
:1087E000030575450ED00AFB05BC9CF976C094457F
:1087F000EED12846C0B2F9F783FC064B99F8001079
:108800001F883FE70028FFF63DAFF3E760AE00208A
:10881000ACA50020A4C60020B4C60020E4A6002019
:108820002DE9F047A84C2DED048BA368204698470E
:10883000002800F0BB80B4F90E30A17D06EE903A1E
:10884000B4F9103007EE103AB4F9123007EE903A4E
:10885000F8EEE66AB8EEC77AF8EEE77A0929C4EDD1
:10886000126A84ED137AC4ED147A00F0A380974E57
:1088700004F1480027F0C4FDB28DB36A002A40F02D
:10888000A580934A934D1268520700F1E880B3F92E
:108890000020D4ED147A94ED128AD4ED138A06EEFA
:1088A000102AB3F90220B3F9043006EE902A07EE3D
:1088B000103A894B894A93F80080B4F8443092F812
:1088C0008273B8EEC66AF8EEE66AB8EEC77A38EE9A
:1088D000468A37EEC79A78EEE68A07EE903A3388F2
:1088E00084ED128AF8EEE79AC4ED138A84ED149AA7
:1088F000002B40F0FF80B8F1040F00F0D88195ED17
:108900005F6AD5ED606A95ED617A85ED5F8A38EE34
:10891000466A78EEE66A39EE477A26EE296A66EE0E
:10892000A96A27EE297A84ED156AC4ED166AC5EDA9
:10893000608A84ED177A85ED619A94ED137AD4ED0F
:10894000167A94ED126AD4ED156A27EE077A67EE6F
:10895000A77AA6EE067AB8F1040FE6EEA67A94EDB1
:10896000146AD4ED176AA6EE067AE6EEA67AB1EEA0
:10897000C70AB1EEE77AD4ED006A26EE800A26EE49
:10898000878A84ED180A84ED198A0CD1DFED548AA8
:10899000544D20EE280A45F08FFE28EE280AA880C4
:1089A00045F08AFE2881012384F86830BDEC048BF1
:1089B000BDE8F087454E04F1200104F1480027F09E
:1089C000B9FCB28DB36A002A3FF45BAFB2F5C87F41
:1089D00000F051813F4DD4ED127A95ED547AD4EDEB
:1089E000136A94ED146AB8EEC77A4FF0000C37EEB4
:1089F000277AD5ED557AC4F848C0F8EEE77ABDEE8F
:108A0000C77A77EEA67AD5ED566A85ED547AF8EEF8
:108A1000E66AFDEEE77A76EE866A17EE901AC5ED05
:108A2000557AFDEEE67A4FF0000E012AA3F800E039
:108A300017EE100AC4F84CC017EE907AA3F802E0C3
:108A4000C5ED567AC4F850C0A3F804E000F01682D1
:108A5000013AB2851E4A126852077FF518AFB5F881
:108A60005C71322F00F0C180002F40F0828195F8B8
:108A70007A21002A3FF40BAFDFF870C0D5F87421DB
:108A8000B4F80CE0D5E95B178CFB0298D217C2EB67
:108A90002812A2EB0E029A808CFB01E2C917C1EBEF
:108AA000221119808CFB0721FA17C2EB21125A8080
:108AB0000D4B00200122D881C3F80A2085F87A01E5
:108AC000F9F7E0FCB36AE2E684BE002090B3002030
:108AD00068AF002020080120A0350020B0AA0020A7
:108AE00000007A44A4350020B0AF00201F85EB5170
:108AF0000AD7233C002F00F0B380D6ED027A96ED22
:108B0000037A96ED010A38EE678AE8EE077A95ED6A
:108B10005F8AC6ED027A77EEC06AA6EE870A30EE6B
:108B2000488A86ED010A28EE298A84ED120A84ED2E
:108B3000158A85ED5F0A002F7FD0012F00F0798123
:108B4000D6ED057A96ED067A96ED040A95ED608AE3
:108B500078EEE78A012FE8EE877A77EEC06AC6EDF5
:108B6000057AA6EE870A30EE488A86ED040A28EEDA
:108B7000298A84ED130A84ED168A85ED600A00F0D7
:108B80003A81022F00F04A8196ED087AD6ED096A03
:108B900096ED070A95ED618A79EE477A022FA6EEE7
:108BA000A77A77EE407A86ED087AA6EEA70A30EE2D
:108BB000488A86ED070A28EE298A84ED140A84ED96
:108BC000178A85ED610A7FF4B8AEB8F1040F7FF41F
:108BD000B4AE45F071FD1FED3A0ABB4D28EE000A18
:108BE000688045F069FDE880A7E6B84AD4ED126ACE
:108BF00094ED137AD4ED147AD268C5F868211A6816
:108C0000C5F86021FDEEE66A9A88A5F86421BDEEFC
:108C1000C77AFDEEE77A00210022A164C5ED5B6A08
:108C20001A8085ED5C7AE164C5ED5D7A5A80216534
:108C30009A807A1EA5F85C2119E7B8F1040F7FF439
:108C40007FAF45F039FD9FEDA20ADFF87C9228EE58
:108C5000000AA9F8020045F02FFDA9F806006FE709
:108C6000B8F1040F7FF449AFB0EE480A45F024FD97
:108C7000954B188041E7D4ED126A94ED137AD4ED48
:108C8000147A944DFDEEE66ABDEEC77AFDEEE77A02
:108C900000200021A064C5ED546A198085ED557A45
:108CA000E064C5ED567A598020659980D0E697B387
:108CB000D5ED5F7A85ED5F8A38EE678A012F28EE61
:108CC000298A84ED158A00F0BF80D5ED607AC5ED64
:108CD000608A78EEE77A022F67EEA97AC4ED167AF9
:108CE0003CD1B0EE490A45F0E7FCD5ED617A9FED45
:108CF000780A754E85ED619A79EE677A00B267EE73
:108D0000A97A308027EE800AC4ED177A708045F08A
:108D1000D3FCF08011E6B0EE480A45F0CDFCD5ED6D
:108D20005F7A9FED6B0A684E85ED5F8A78EE677A11
:108D300000B267EEA97A308027EE800AC4ED157A7A
:108D4000708045F0B9FCD5ED607AF08078EEE77A76
:108D5000C5ED608A67EEA97AC4ED167AD5ED617A21
:108D600085ED619A79EE677A67EEA97AC4ED177A94
:108D7000E3E5D5ED5B6A94ED127AD4ED137A94EDC8
:108D8000146AF8EEE66A002176EE876A95ED5C7A61
:108D9000A164B8EEC77AFDEEE66A37EE277AD5ED24
:108DA0005D7AC5ED5B6AF8EEE77ABDEEC77A77EEDD
:108DB000867A0022FDEEE77A012F1A8085ED5C7A33
:108DC000E164C5ED5D7A5A8021659A807FF431AF08
:108DD0000B2085F8782185F8797107F04BFEB36A8E
:108DE000D5F860111960394AB5F864119980D5F841
:108DF0006811D1601DE7B8F1040F7FF4C5AE45F0EE
:108E00005BFC9FED330ADFF8C09028EE000AA9F85A
:108E1000020045F051FCA9F80600B5E6B8F1040FD0
:108E20007FF4B2AEB0EE490A45F046FC264B1880FE
:108E3000AAE6B8F1040F7FF483AEB0EE680A45F0FD
:108E40003BFC214B18807BE6B0EE680A45F034FC11
:108E5000D5ED607A9FED1E0A1B4EC5ED608A78EE57
:108E6000E77A00B267EEA97A308027EE800AC4ED77
:108E7000167A708045F020FCF0806FE7DFF858C06C
:108E8000B4F80C80C8378CFB07A9FF17C7EBE917AC
:108E9000C830A7EB08079F808CFB0087C017C0EB8A
:108EA000E710C83118808CFB010CC917C1EBEC111D
:108EB0005980064BC3F80A20A3F80EE0F9F7E2FA4E
:108EC000B28DB36AC4E500BFA4350020B0AF002066
:108ED0000AD7233C200801201F85EB51CE4B1B688D
:108EE0001A0700D470472DE9F0432DED108BCB4FBE
:108EF000CB4C3A78D4F89831D4F88811582A83B0FA
:108F00000546C4F88801187800F0D281012800F0E5
:108F10005C82C449D4F89031A1F1B400984797F825
:108F20000080B8F1580F08BFBF4B80F00100C0B2FD
:108F300008BF5881002840F0A782B4F9403294F865
:108F4000081207EE903AB4F94232F8EEE77A07EEEB
:108F5000103AB4F94432C4ED937A07EE903AB8EE81
:108F6000C77AF8EEE77A0123092984ED947AC4EDF3
:108F7000957A84F8483200F04881AC4827F040FAEE
:108F800094F85892B9F1000F00F05A81D4F85C328D
:108F900094F859225B1B002B40F3DA81D4ED987AC8
:108FA000D4ED996A94ED9A7A002A00F02A82A04EB4
:108FB000A04B1A6852B1A04B91881B781268DB4312
:108FC00003F001031B0101FA03F3936194ED941A7A
:108FD00094ED934AD4ED959A94EDA40AD4EDB47A25
:108FE000D4ED9C2AD4EDA9DA94EDA53A94EDAEEA3D
:108FF00094EDAA2AD4EDB5EAD4EDA64AD4EDAFCAD1
:1090000094EDABCAD4EDB33A94EDB6FA94EDA7BAA9
:10901000D4EDB7FA94EDA18AD4EDA08A21EE017ABD
:10902000B0EE62AAA4EE047A64EE2D6AA9EEA97AE3
:1090300021EE0E6A67EE005AE7EE036A25EEA75AA4
:10904000A4EE026AA5EE85AA66EEAE1AC7EE8A5AAB
:10905000F0EE4A0AC4EDB45AC6EE8A5AA7EE246A64
:10906000E6EEA10AF0EE436A86EE209AE5EEC56AC6
:1090700061EE2C7AF0EE455AE4EE0C7AC4EDA56A66
:1090800066EEA16AE3EE215A69EEA33AE0EE056AC4
:1090900026EE0F5A73EEA77AB0EE600AA6EE050A26
:1090A000B0EE646AE7EE0B7AA9EE656AF0EE40AACC
:1090B000E6EE056A84EDA66A27EEAF6AE4EE855A0D
:1090C000E7EE86AAF0EE624AE3EE864AB0EE613A37
:1090D000F7EE003AA2EE053AA9EE612A83EEAA9ACB
:1090E00062EEAAAAC7EE80BA80EE2ADA22EE800AE1
:1090F000D4EDA27A84EDAA2AC0EE80AA60EEA20A7C
:109100002AEE8F0A61EE277A84EDB60A8AEE200AEB
:10911000E4EE087A60EE2E0AB0EE6C0AABEEC50AF9
:1091200073EEE77A84EDAF0A26EE000AC4EDB50AC5
:10913000AEEE050AF0EE450AE1EE004AB0EE4C1A3A
:10914000ABEEC31AB0EE4B0AABEEE50A84EDAB1AF8
:1091500026EE011AE6EE006AADEEA11AE7EE264A07
:10916000A2EE051AE6EE0B5AE4EE014AE6EE2C0AF0
:10917000C2EEA46AA6EE0C3A26EEA65AD4EDA36A75
:1091800084EDA70AE9EEE67A2DEE2FDAE7EE687AAB
:1091900084EDB7DA67EEA55A27EE833AE9EE258A21
:1091A00067EEA00A83EEA84AC4EDA08A67EE867A2D
:1091B00094EDA26AB0EE667AA9EE277AA0EE896AEB
:1091C000A9EE038AD4ED9B6A84EDA26A73EEE63AB7
:1091D000FEEE007A66EE275A68EE274AE3EE856ACD
:1091E00067EE277A24EE846A67EE847A84EDA37AA8
:1091F00025EE847A84EDA18A84ED9D6A84ED9E7AC1
:10920000C4ED9F7AC4ED9C6A1BE00C4901F140005B
:1092100027F090F8B4E600BF80BE0020A035002003
:1092200020080120600A0120A43500206C0A0120DA
:1092300088AF0020702C00207C2C00202C0A0120FC
:10924000994EB6F9083094ED939A94ED948AD4ED42
:10925000958A07EE903AB6F90A30F8EEE77A07EE0B
:10926000103AB6F90C3039EE679A07EE903AB8EE3C
:10927000C77AF8EEE77A38EE478A78EEE78AB8F1EF
:10928000570F84ED939A84ED948AC4ED958A18D093
:10929000B8F1580F7AD0854B1B68012284F83C2224
:1092A000002B40F0F78003B0BDEC108BBDE8F083DD
:1092B0007F4E691A0128B18100F0CA8000233381F2
:1092C00027E6B0EE490A45F0F7F9794E94ED9D0A8C
:1092D000308045F0F1F9B0EE480A308145F0ECF904
:1092E00094ED9E0A708045F0E7F9B0EE680A70814F
:1092F00045F0E2F994ED9F0AB08045F0DDF928EEE3
:10930000080AB081A9EE090AA8EEA80AB1EEC00ABF
:1093100045F0D2F9F080B9F1000F13D094F859322A
:1093200083B1D4ED9B6A9FED637A9FED636AD4EDC0
:109330009C7A37EE667A77EEE67A86EE070A20EEBA
:10934000270A01E09FED5D0A45F0B6F9F081A2E73A
:10935000002A78D094ED9D0A534E45F0ADF994ED76
:109360009E0A308145F0A8F994ED9F0A708145F07E
:10937000A3F9B081012007F07DFBF9F783F84FF0E6
:10938000000997F8008084F858925AE7D4F8E06210
:10939000C4F8E052F0F74CF93B78582B7FF47BAFE0
:1093A000AE1B07EE906ADFED466A414BB8EEE77AF6
:1093B0002822C6EE877A1A80401B9E80D880FCEE59
:1093C000E77A17EE902A5A8065E793F904003D4B3F
:1093D000542101FB003191F83660002E47D091F8FE
:1093E0003610112943D0012384F83C324FF4FA732C
:1093F000354A12681268136103B0BDEC108BBDE8EA
:10940000F08367EEA77A9FED316AE6EEA67AE7EE83
:10941000077AF4EEC67AF1EE10FA7FF711AF224E1A
:1094200001920D2007F026FB019AB260012384F817
:109430005932B281F0F7FCF8254B97F800800344CD
:10944000C4F85C32B4E50C2007F014FB164E96E726
:1094500093F904001B4B542101FB003191F836C0F5
:10946000BCF1000F03D091F83610112909D1542115
:1094700001FB00339B699B691B040FD5582AB2D1AD
:109480000B4E01233381AEE7012384F83C324FF4C5
:109490007A73ADE7642BB8BF6423A9E7582A7FF439
:1094A00038AD034E0AE700BF88AF00200805002052
:1094B000A43500200800803F0000FA4400000000AE
:1094C00000247449543C00201C080120FF41EF4750
:1094D00080C3C9012DE9F04F2DED048BDFF8D4B323
:1094E0009BF8E43295B0022B0393059040F0E481A1
:1094F000E649DBEDBB7A4C8ADFEDE56A07EE104A00
:10950000B8EEC76A012377EEC67A9FEDE27A8BF850
:10951000E532F4EEE67AF1EE10FA9BF8E83288BF15
:10952000F0EE667AF4EEC77A06EE903AF1EE10FAB3
:10953000B8BFF0EE477AF8EE666AB0EEE77AF4EE7E
:10954000C76AF1EE10FA00F39584F5EEC07AF1EEF9
:1095500010FAB4BF76EEA77A77EEE67A9BEDBC7A86
:109560009FEDCB5ADFEDCB5ACBEDCD7A37EE467A75
:10957000B4EEC57AF1EE10FA88BFB0EE457AB4EEDB
:10958000E57AF1EE10FAB8BFB0EE657AF0EEC75AA0
:10959000F4EEE56AF1EE10FA00F39185B5EEC07ACB
:1095A000F1EE10FAB4BF36EE877A37EE667ADBED6D
:1095B000BD6ADFEDB75A9BF8EA328BEDCE7A76EED4
:1095C000C66A9FEDB46AF4EEE56AF1EE10FA88BF60
:1095D000F0EE656AF4EEC66AF1EE10FAB8BFF0EE8E
:1095E000466A0BB9F1EE666A9BF8E93206EE103A6C
:1095F000B8EE466AF0EEE65AF4EEC65AF1EE10FA0C
:1096000001F11D81F5EEC06AF1EE10FAACBF36EE45
:10961000C66A36EE266AA04BDBEDBE6A1A688BED91
:10962000CF6AFDEEE66A12F4805216EE903A00F030
:109630000B85B3F5FA6FA8BF4FF4FA63B3F57A7FE1
:10964000B8BF4FF47A73A3F57A739BF830110029F1
:1096500040F0388703EB830103EB410342F6F72028
:109660008342194600F3528513F57A7F00F30C8785
:10967000BBF9343906EE903AF8EEE66ACBEDD06AE3
:10968000002A40F04E85BBF848335F0640F1D88091
:1096900040F62B021A40814B08BFDBEDCF2A93ED39
:1096A000043AD3ED053AD3ED0A5A93ED062AD3EDE9
:1096B000036A93ED074A93ED086AD3ED094A18BF90
:1096C000DFED772A36EEA30A33EE021A76EEC31ADE
:1096D00076EE839A72EE638A33EE425A76EEE36A4E
:1096E00032EE232A74EE253A36EE643A66EEA36A29
:1096F00074EE650A25EE035AF0EE663AE0EE203A83
:10970000B0EE453AA0EE203A34EE069A34EE464AE0
:1097100036EE246A34EEE58AE1EE463AA1EE063AE8
:1097200074EEA54AF0EE455AD1EE065A73EEC53AEC
:10973000B6EE001A36EE833A63EE813A21EE433AF2
:10974000E8EE883AB0EE658AA9EE893AA0EE608A22
:1097500035EEE66A23EE035AA0EE206A76EE886ABA
:10976000F0EE455A66EE816AD3EEA35AA3EEA35AF1
:1097700026EE016AE2EE046AA1EEA46AB0EE454A62
:10978000B0EE655AA6EEE65A23EE061A26EE262A13
:10979000A6EE464AB0EE418AF0EE420A63EE261A81
:1097A000A3EEA68AA6EE065AE3EEC30AA3EEE61AD5
:1097B000E6EE465AA6EEE64A77EE074AB0EE610AB2
:1097C000A3EE860A25EE075A60EE870A64EE884A01
:1097D000E6EEA65AE3EEC61AA3EE832A31EE011A8C
:1097E000E4EE274AB0EE457AB0EE605AA7EE817AF1
:1097F000A0EE275A71EEA11A65EEA27A32EE022A85
:10980000B0EE004AF0EE645AE2EEA15AA2EE227ADD
:10981000E5EE047AC3ED0B3A83ED0C3A83ED0D6A65
:10982000C3ED0E6A1F4BCBEDCD5AC3ED005A83ED4D
:10983000017AC3ED027A8BEDCE7A0AB9CBEDCF7AFD
:1098400010F0F8FA184B049300221446049B8BF88E
:10985000E4221B78002B41D0144B1B78472B08D1F6
:109860000399134A0BEB8103D3F868399B1122F853
:1098700011300BEB8403D3F868399B11CBF87439A2
:1098800015B0BDEC048BBDE8F08F00BF6CAE0020BE
:109890000000FA430000FAC368AF0020080500206A
:1098A000000000007C110120C4B30020A03500207E
:1098B000A4350020200801200124A3428BF83C425B
:1098C0002DD019F027F80028BCD0384B0493049B06
:1098D0001B7822468BF8E422002BBDD1EFF7A8FEBF
:1098E000059B039AC3F101031844314B1B68DD69E2
:1098F0000BEB8203E909D3F868399E11B6EBD51F4B
:109900001CBF8B019911920088425A44CBBF800141
:1099100003F1FF33C2F86809C2F868399CE718F010
:10992000C1FF9BF845339FED237A07EE903AF8EE9E
:10993000E77A9BF8C13067EE877A13F0010FFCEEEF
:10994000E77A1D4B069317EE904A054640F05A847D
:10995000059B1C44CBF84C43DBF85823550700F11A
:109960008D829BF85C33002B00F0A382069BD3F81A
:109970000090124B07930D4B049319F0040F40F025
:109980001084DBF878230DAF00230D93CDE90F335E
:109990007B601193002A4FF00403129354DD084EAC
:1099A000084D931901934FF0010813E0C4B3002050
:1099B0001C0801200024744968AF002080BE0020EC
:1099C0009C0B0120CCAF00202F2840F2A981019BE5
:1099D0009E4236D016F8014B04EB440105EB4103DF
:1099E00015F8110000934FEA501C14AB03EB8C03E5
